:020000040800F2
:1000000000000220211506083D9D00080572020827
:10001000D1150608D1150608D11506080000000004
:100020000000000000000000000000005DB20008B9
:100030005FB200080000000061B200082D1901083D
:10004000D1150608D1150608D1150608D1150608E0
:10005000D1150608D1150608EFFF0008F3FF0008C8
:10006000D1150608F7FF0008FBFF0008E5A300080C
:10007000F9A300080DA4000821A4000835A4000875
:1000800049A400085DA40008D1150608000000007E
:10009000000000000000000000000000FFFF00085A
:1000A0001DA3000845A300086DA3000807A30008CE
:1000B00095A30008A9A30008BDA30008D115060850
:1000C000D1150608D1150608D1150608D115060860
:1000D000D1150608599E0008659E00080000000022
:1000E00003000108D115060863B2000800000000F3
:1000F00000000000000000000000000071A40008E3
:1001000000000000D1150608D1A30008D11506088B
:1001100000000000000000000000000000000000DF
:1001200085A4000899A40008ADA40008C1A4000893
:10013000D5A400080000000000000000000000003E
:10014000000000000000000000000000ADB2000848
:10015000E9A40008FDA4000811A50008D1150608AF
:10016000D1150608D11506080000000000000000A7
:10017000000000000000000000000000000000007F
:1001800000000000D115060800000000000000007B
:08019000D1150608D11506087F
:080198008806060001000000CA
:1001A0001C6A012002010000020014003C6A0120C8
:1001B00002020000020014005C6A0120020B000031
:1001C000020014007C6A01200206000002001400F4
:1001D0009C6A01200207000002001400BC6A012092
:1001E0000203000004001400DC6A01200208000081
:1001F00004001400FC6A0120010C000000007700DC
:100200001C6B0120010D0000000076003C6B0120FA
:1002100001110000000076005C6B0120010E01005E
:10022000000077007C6B01200113000000007600C5
:100230009C6B01200115000000001E00BC6B01201A
:10024000011B000000000D00DC6B0120011D0000FF
:1002500000000E00FC6B0120011E000000001E00CB
:100260001C6C01200118000000000C003C6C0120F7
:100270000119000000000E005C6C0120012A010041
:10028000000018007C6C01200122000000004800E2
:100290009C6C01200123000000004900BC6C01207F
:1002A0000124000000004A00DC6C01200125000050
:1002B00000004B00FC6C01200126000000004C00F7
:1002C0001C6D01200127000000004D003C6D012045
:1002D0000128000000004E005C6D01200129000093
:1002E00000004F007C6D0120012D0000000029005E
:1002F0009C6D0120012E010000002900BC6D012031
:10030000012F010000007000DC6D012001310000B0
:1003100000003100FC6D012001300100000052009E
:100320001C6E012001320100000028003C6E0120FB
:1003300001330000000076005C6E012001340100F2
:10034000000028007C6E01200238040000012C000F
:100350009C6E01200137000000003C00BC6E0120B3
:08036000013A0000000020003A
:10800000D0E907239A423CBFC1685218D01A704782
:10801000D0E9092300699A4238BF1218D31A0138EF
:10802000C01A7047D0E90902131A584258417047E4
:10803000036A41690246C85CD16801338B4228BF9C
:10804000002313627047436A8269D154436A02690C
:108050000133934228BF0023426B4362D36843F04D
:108060008003D3607047436B188810F010001EBF68
:108070001A889B8801207047436B99891A88890662
:1080800010B592B2044607D5900605D5E26A2AB328
:108090009888216B80B29047636B99891A8809068A
:1080A00092B210D510060ED5D4E909128A4223D017
:1080B000A169895CC9B2998021690132B2FBF1F0F2
:1080C00001FB1022A262998A1A88C90592B204D5CE
:1080D000D20744BF4FF6F7721A8010BD9B88E26941
:1080E0006169DBB28B54E369E2680133B3FBF2F1FF
:1080F00002FB1133E361CFE7DA6822F08002DA6035
:10810000E1E7036942681F2B70B54FF0200185BF7E
:10811000A3F1200554681468A94098BF99402142F2
:108120000DD08069017C03290AD11F2B4FF020015B
:1081300085BF203B99409940D16098BF916070BD48
:108140004568002101742C686E79074DA18935F8C6
:10815000165089B221EA0501A181C16888680168C9
:1081600021F001010160E0E7C84606080E4BDA681D
:10817000D20310D4DA68D1060FD4DA68D2050ED44F
:10818000DA6812F0E00F0CD1DB6813F0020F0CBFBD
:108190000920082070470120704706207047022000
:1081A00070470720704700BF003C024007B5092315
:1081B0008DF80730FFF7DAFF8DF807009DF80730DC
:1081C000012BF7D09DF8070003B05DF804FB838A0C
:1081D000028B9BB243EA024399430CBF012000206B
:1081E000704782B000230193009301230090019314
:1081F000019B63B1009A21F07F4314320092009AF0
:1082000012681A4214BF0120002002B07047009A81
:108210001832F3E7024B01F001011970704700BFFB
:108220000000002070477047704701207047034BE3
:1082300018685B68C01AC0F30A0070474019002034
:10824000064B986830B19B68052B05BF044B187826
:108250000020C0B200F00100704700BF40190020AC
:1082600000000020012380F849307047054BD86892
:108270001B69984234BF03F1FF3303F2FF73181AEE
:10828000704700BF4019002010B5D0F8E83504460B
:108290001B699847032384F81231002010BD08B5EC
:1082A00090F8123180F81331042380F81231D0F89D
:1082B000E835DB689847002008BD08B5D0F8E435FC
:1082C000DB6903B19847002008BD08B5D0F8E43554
:1082D0001B6A9847002008BD08B5D0F8E4355B6AF2
:1082E0009847002008BD70B504460D46164658F064
:1082F000F1FAC3B201335B0033802B7003236B7040
:10830000601E0223002410F8011F01B970BD5A1C21
:10831000D2B2E9540233AC54DBB2F4E710B5064CE8
:108320006068FF2806D005494A69183100F080F8D6
:10833000FF236360002010BD0000002040190020D2
:10834000432301480B807047080000201223014896
:108350000B8070474B000020042301480B807047BE
:108360005D00002010B5044C04480A462146FFF782
:10837000BAFF204610BD00BF6019002090EB060830
:1083800010B5044C04480A462146FFF7ACFF2046CE
:1083900010BD00BF60190020A3EB060810B5044C07
:1083A00004480A462146FFF79EFF204610BD00BF45
:1083B00060190020A8EB060810B5044C04480A46D2
:1083C0002146FFF790FF204610BD00BF6019002036
:1083D000B2EB060810B5044C04480A462146FFF7E4
:1083E00082FF204610BD00BF60190020BDEB0608CB
:1083F00070477047704770477047024B00229A6081
:10840000704700BF401900207047054B002005222F
:108410009A60C3E948001860586083F828017047E3
:1084200040190020014B002098607047401900203F
:10843000212838B50C461BD022282BD0202815D156
:10844000A1B1072A12D11A4DD5F8243113B1096808
:10845000002098472368C5F82931237985F82D3104
:10846000637985F82E31A37985F82F31002038BD46
:108470000029FBD0072AF9D10D4BD3F829210A6036
:1084800093F82D210A7193F82E214A7193F82F3118
:108490008B71EBE70029E9D0022AE7D1044AD2F830
:1084A0002031002BE2D00988D2F830019847DDE76F
:1084B000401900202DE9F843194D2C68C4F50069D6
:1084C000894507460E4605F59A7818D30A460146AF
:1084D00008EB04005BF0AAFE3444C4F30A042C60E9
:1084E0006B6803F2FF731B1BC3F30A03802B9DBF52
:1084F000012385F8283102200020BDE8F8830146D9
:1085000008EB0400A4F500644A4634445BF08EFE98
:10851000224607EB090140465BF088FEDFE700BF1B
:1085200040190020034BD3F8340908B103691847F8
:10853000704700BF40190020034B93F85C090038D6
:1085400018BF0120704700BF40190020034B93F86B
:108550005C09032894BF00200120704740190020C7
:1085600000487047A0220020837B042B0DD0074BCE
:10857000D3F898200132C3F8982042600422827315
:10858000D3F89C200132C3F89C207047785D00200E
:10859000202301480B80704761000020122301480E
:1085A0000B80704781000020042301480B80704736
:1085B000930000200A4608B5044920B90448FFF793
:1085C00092FE024808BD0348F9E700BFD022002010
:1085D000CBEB0608E3EB060810B5044C04480A464A
:1085E0002146FFF780FE204610BD00BFD0220020AC
:1085F000FBEB060810B5044C04480A462146FFF779
:1086000072FE204610BD00BFD02200200EEC0608EE
:1086100010B5044C04480A462146FFF764FE204684
:1086200010BD00BFD022002019EC0608002370B551
:108630004D1C1E46040FB0F1204F34BF3034373488
:1086400001F8134005F813600133DCB2A2424FEA8F
:108650000010EFD870BD1A2310B50B80094BD3F86A
:10866000E807D3F8EC2780180AD0D3F8EA47064980
:108670000822FFF7DBFF042210312046FFF7D6FF68
:10868000024810BD00F0FF1F990000209700002055
:1086900008B5FFF747FF013840B208BD002070471A
:1086A0000020704770477047D0ED007AD0ED036A24
:1086B00030EE677AE6EE877AB0EE670AC0ED007AB0
:1086C000704790ED017AB5EE407AF1EE10FAF0EED7
:1086D000407A09D19FED0E7A60EE870AF7EE006AC4
:1086E00086EEA07A80ED017A90ED017A90ED000A95
:1086F00080ED021A31EE077A77EEC07AC1EE076A92
:10870000A6EEA70AC0ED036A80ED000A704700BF1D
:10871000DB0FC940D0ED056AD0ED017A90ED026A19
:10872000D0ED045AB0EE407A26EEA70AD0ED007ADA
:1087300080ED057AA7EE870AD0ED067AC0ED066ACD
:10874000A6EE270AD0ED077A90ED036AA6EE670A37
:1087500090ED086AC0ED087AA5EEC60A80ED070A1A
:108760007047B0EE407AD0ED007A90ED050AD0ED7A
:10877000016AA7EE870AD0ED037A67EEC07AE6EECB
:10878000877AD0ED066A76EEA77AD0ED026AC0ED60
:10879000057AD0ED047A67EEC07AE6EE877AC0ED0E
:1087A000067A704703685A1C0260197070472DE9F9
:1087B000F04F87B083680193D0E90032511C91FBE0
:1087C000F3F403FB1411416000EB820181ED200AF8
:1087D000B1EE400A00F18005009281ED400A00F5FB
:1087E0008070A3F1020E4FF0010C019A6245009ACD
:1087F00017DA01991A44521A92FBF3F103FB112282
:1088000005EB820500EB8200D5ED007A90ED007A51
:1088100077EEC77AB6EE000A27EE800A07B0BDE809
:10882000F08F0EEB020494FBF3F103FB1144611C87
:1088300091FBF3F603FB161105EB840600EB8404B1
:1088400094ED007A03940CEB0104D6ED007A0296C5
:1088500094FBF3F603FB1644F246F14626460F4618
:10886000A3EB0C0BD9450CDB029AD2ED007A039AEC
:1088700092ED007ADA454EDB0CF1010CAEF1020EFE
:10888000B3E7BB42D8BF002705EB8702D2ED006AF1
:108890000492B342D8BF002600EB8702F4EEE76AE9
:1088A00092ED006A0592F1EE10FA00EB8602D2ED2D
:1088B000005A4FEA860811DDA84498ED005AF4EEFC
:1088C000C56AF1EE10FA09DDB4EEE75A049AF1EE4A
:1088D00010FA58BFF0EE457AC2ED007AB4EEC76ADE
:1088E000F1EE10FA0EDDB4EEE56AF1EE10FA09DDF4
:1088F000F4EEC75A059AF1EE10FA58BFB0EE657A59
:1089000082ED007A0137013609F10109B0EE467AAD
:10891000F0EE667AA6E78B42D8BF002105EB81080E
:10892000D8ED006AA342D8BF0024F4EEE76A00EB5A
:10893000810700EB8409F1EE10FA97ED006AD9ED9A
:10894000005A4FEA840610D52E4496ED005AF4EEF4
:10895000C56AF1EE10FA08D5B4EEE75AF1EE10FA56
:10896000D8BFF0EE457AC8ED007AB4EEC76AF1EEF2
:1089700010FA0DD5B4EEE56AF1EE10FA08D5F4EE72
:10898000C75AF1EE10FAD8BFB0EE657A87ED007ADB
:10899000013101340AF1010AB0EE467AF0EE667A4E
:1089A00068E703690133012B036108D1DFED107A19
:1089B00080ED010A80ED000AC0ED027A704790ED6B
:1089C000006A07EE903A70EE466AF8EEE77A86EEB5
:1089D000A77AD0ED027A37EE067A30EE470A80EDBC
:1089E000017AE6EE807AB0EE470AC0ED037AE1E75D
:1089F0000000000003685A1C02601970704700797B
:108A000070470079C0F34010704700794009704703
:108A10002DE9F843D0F8148007468946B8F1000FD5
:108A200057D10568C5F30D0606B3D9F80060FFF706
:108A3000BDFB092840F08680444C236923F4407331
:108A40002361236943F400732361236943F0010325
:108A500023612E60FFF7AAFB2369092823F0010395
:108A600023616FD13B6804333B6032E0384B9D4259
:108A700029D303F580439D4224D303F580439D42CF
:108A80002AD3344B9D4229D903F580339D4227D9FF
:108A900003F500339D4225D903F500339D4223D9C8
:108AA00003F500339D4221D903F500339D421FD9C0
:108AB00003F580239D421DD9B5F1016F1CD305201C
:108AC0000BF05AFA0826FFF771FB092816D04FF071
:108AD000FF384046BDE8F8831026F4E71826F2E791
:108AE0002026F0E72826EEE73026ECE73826EAE7EE
:108AF0004026E8E74826E6E75826E4E7134C2369D2
:108B000023F440732361236943F4007323612369D1
:108B100023F0F80323612369334343F00203236105
:108B2000236943F480332361FFF740FB236923F07B
:108B3000020323612369092823F0F80323613FF42A
:108B400074AFC4E76FF00108C3E700BF003C024008
:108B500000400008FFFF000803682DE9F0410D46C2
:108B6000416813448B42044619D8AE1800F10C0733
:108B70004FF00008B54202D16069BDE8F081236979
:108B80005A1C2261234415F8011B1973042AF1D1E0
:108B900039462046FFF73CFFC4E90480EAE74FF07E
:108BA000FF30EAE72DE9F0479846444B914603EB46
:108BB000800205469468002C51D02833636004F18C
:108BC0003E03A36104F59F73E3614FF48073C4E92E
:108BD0000433236894F83D00E160A36307F03EFB93
:108BE000064694F8440294F83CA0271D08B154F0BE
:108BF00045F894F8450208B154F040F8D4F84032F2
:108C00001BB12F4A116B0B43136318F0080F2FD0C1
:108C10000135EDB21EB140F20673F380357218F0E3
:108C2000100F94F846221DD00221304607F0D6FAE4
:108C3000D4F8482294F9471294F8473212010029D7
:108C4000D2B236DB1F49C81880F800235809012228
:108C500003F01F0302FA03F341F820303C4620469C
:108C6000BDE8F08718F0200F0CBF32211221DCE79D
:108C700019F0020F0CD06B1CDBB21EB140F2065291
:108C8000F280337294F846220221304607F0A6FAA9
:108C900019F0010FCCD0504607F0E0FA0135EDB2E3
:108CA00018B140F20663C380057294F8462202218F
:108CB000BCE7054903F00F03CA54CFE7C8460608CE
:108CC0000038024000E100E014ED00E02DE9F3413E
:108CD000038A8689B6B205460C461E404FF000480E
:108CE00016B902B0BDE8F081B6FA86F328FA03F2AD
:108CF000D24391B2298216401B3B002C3ED0042B5C
:108D0000EED8DFE803F037312B250300E368EF6A84
:108D100023B19B6813B1B9B2201D9847636A2BB188
:108D20009B681BB1B9B204F11C009847E36B2BB1EF
:108D30009B681BB1B9B204F134009847636D002BF6
:108D4000CED09B68002BCBD0B9B204F14C0003E02D
:108D5000E368696B5B68201D9847C1E7636AA96B8C
:108D60005B6804F11C00F7E7E36BE96B5B6804F1F7
:108D70003400F1E7636D296C5B68E6E7042B06D8E5
:108D8000DFE803F00D0B09070300EB6A0193019B79
:108D9000A6E76B6BFAE7AB6BF8E7EB6BF6E72B6CD0
:108DA000F4E7F8B5174C002504F68F2662682368AF
:108DB0009A4224D063682344012793F834516368AE
:108DC0000133C3F30A0363606368236894F82831AE
:108DD0008BB16368226803F2FF739B1AC3F30A0323
:108DE000802B08D9002384F82831074840233246D5
:108DF000012156F0D1FE002FD8D02846F8BD00271B
:108E0000E4E700BF4019002010240020282303FBC2
:108E1000010110B5B1F88C1304460648FFF74AFB70
:108E200028B9044A40230121204656F0B5FE00200F
:108E300010BD00BFCF23002090F84820531C0244EF
:108E4000DBB280F8483082F8341090F849200AB13B
:108E5000132B01D957F098BA7047002280F84920A7
:108E600057F092BA2DE9F041184E56F8348C04466A
:108E700016F8303C33B9164F6518A54213D10020BF
:108E8000BDE8F08156F8343CA3EB0803322BEFD950
:108E90000220F5E756F8343CA3EB0803322BF7D851
:108EA00001200AF001FDFB683A690133C3F30A03AC
:108EB0009342EFD0FB6814F8012B334403F82F2CB6
:108EC000FB680133C3F30A03FB60D6E7382A0020AE
:108ED00040190020F8B50D461446FFF7B1F998B1D6
:108EE0000A4E56F8347C002C0EDD21462846FFF74A
:108EF000B9FF00280CBF23460023E41A1D4456F88E
:108F0000343CDB1B322BEED9F8BD00BF382A0020E1
:108F100070B50E4BD3F8DC2793F8D157044632B125
:108F200093F8E0372B4302D1012156F069FC8121EF
:108F3000204656F065FC022D07D12046044ABDE8C4
:108F400070401F23012156F027BE70BD382A002033
:108F50000C32002010B5044671BB90F81131032B80
:108F60001BD1D0F89023D0F87C339A4217D9C1781E
:108F7000012908BFD0F88013A2EB030204BFC9186F
:108F8000C0F88013934228BF1346C0F890239BB2C9
:108F9000D0F88023002156F0FFFD002010BDD0F84E
:108FA000E4351B6923B190F81221032A00D19847B8
:108FB000204656F041FDF0E7D0F8E4359B69002BE0
:108FC000EBD090F81221032AE7D19847E5E770B576
:108FD0000A7812F0600305460C4626D0202B2BD1D0
:108FE000CB884E78DBB112060AD51C491A463046AA
:108FF000FFF71EFAE2881949284656F009FD0CE0F1
:10900000174A5660174A0321536180F81111C0E9CD
:10901000E4331832002156F0BFFD002070BD02225B
:1090200011443046FFF704FAF7E74B780A2B08D0D3
:109030000B2B09D0062BF0D1284656F013FC02204A
:10904000ECE709490122D8E78B781BB9074AC2F837
:10905000F437E2E756F006FCDFE700BF58190020BE
:1090600000000020401900202C320020382A002067
:10907000F0B585B0D0F8CC1590F8CC650291D0F859
:10908000D0150391012180F8111106F01F01B0F8ED
:10909000D22590F8CD75B0F8CE35B0F8D055C0F8DF
:1090A00040210129044600F00981022900F01A81BB
:1090B000002940F09381092F5ED8DFE817F0B60051
:1090C000F4005D00C8005D0057000A005D00A900C3
:1090D00076001D0A022DADF806200BD0032D25D0F9
:1090E000012D49D1D0F8EC351B68A0780DF10601AF
:1090F000984709E0D0F8E43580789B6A0DF10601C5
:1091000098474570C4F8F005BDF80620002A47D0FE
:10911000BDF80E30002B43D09A4228BF1A46ADF856
:1091200006200146204656F073FC39E0DBB2052BE1
:1091300022D8DFE803F003070B0F1317D0F8EC3544
:109140005B68D2E7D0F8EC359B68CEE7D0F8EC3519
:10915000DB68CAE7D0F8EC351B69C6E7D0F8EC3518
:109160005B69C2E7D0F8EC359B69BEE72A4303D1BF
:1091700090F81211032903D1204656F073FB0FE03B
:1091800003F07F05016980F8145163F30A120B683C
:109190001A430A6056F050FC2DB1022384F81231B4
:1091A000002005B0F0BD0123F8E7D9B28D4D0129AB
:1091B00085F8F817E0D890F81231022B0FD0032B66
:1091C000DAD1C1B9022380F81231D0F8E43580F841
:1091D00010115B689847204656F02EFCE0E7002906
:1091E000F9D00121032380F8101180F812312046B4
:1091F00056F0FAFAEFE790F810110129EBD0D0F809
:10920000E4355B68984795F8F81784F81011EEE795
:10921000012AB1D190F81231022B04D0032BABD12B
:1092200000F588717EE770497CE790F81231023BC7
:10923000012BA1D86B4B0022C3F80028D0F81821CD
:1092400012B10222C3F80028684902226AE7012B02
:1092500008D1C4F81831D4F8E43502A99B68204637
:109260009847B8E7022B9BD1EBB2002B98D103694A
:109270002D0A023D5A68032D13D8DFE805F0020CD1
:109280000E10022363F30612564BC3F80428012381
:1092900084F816319FE70323F4E70423F2E705235C
:1092A000F0E70123EEE790F81221023A012A3FF697
:1092B00063AF012B7FF474AF0023CAE790F812313B
:1092C000032B7FF459AFEDB2012D3FF655AFD0F827
:1092D000E43502A99B689847BDF80E30002B7FF457
:1092E0005FAF78E706F06006202EE9B205D1D0F82E
:1092F000E43502A99B68984752E7012F35D0032F28
:1093000023D0002F7FF44CAF90F81231022B5FD0A6
:10931000032B7FF431AF15F0800F4FF028031BBFF4
:1093200001F07F0103FB010103FB010191F81E31F4
:1093300008BF91F876332B49003B18BF0123C1F8D1
:109340000838022201F60801ECE690F81221022A00
:109350003ED0032A7FF410AF002B7FF47CAF4A0687
:109360003FF479AF56F04CFA75E790F81221022AD3
:109370002ED0032A7FF400AF002B7FF411AF11F041
:109380007F023FF428AF6DB22823002DB5BF03FB49
:10939000020303FB010303F58E7303F55D730021E4
:1093A00099701A70E90F00EB82025970002DB4BF5A
:1093B0009269526DD9781368023923F40013012998
:1093C0008CBFC3F30071012161F31C73136042E78A
:1093D0004B063FF4E5AE56F013FAE1E606F08001E5
:1093E000F9E700BF382A002034320020383200204C
:1093F000002310B519460446402256F06BFA40226D
:1094000080212046002356F065FA012384F81231AA
:10941000D4F8E835A0785B689847002010BD38B5CF
:10942000402204460223812156F054FA20460223AA
:109430004022012156F04EFA2046032308228221C1
:1094400056F048FA084B0222002583F84F2083F893
:1094500050500121FEF7D9FF2046044A402356F020
:109460009BFB284638BD00BF00000020CF23002012
:1094700010B58121044656F003FA2046012156F02A
:10948000FFF92046822156F0FBF9FEF7CBFF0020C2
:1094900010BD10B58121044656F0F2F92046012195
:1094A00056F0EEF9024B002083F80C0810BD00BF07
:1094B000382A0020F8B5214D15F8302C012A034632
:1094C0002BD1D5F8104814B905F8304C21E0402CC8
:1094D00021D8A6B2402E02D1022205F8302C184F16
:1094E000184A39690A44C3E9542240F201110022A2
:1094F000A3F84411C3E9566203F5A271184656F069
:10950000B2FA3B693344C3F30A03A41B3B61C5F8B9
:1095100010480020F8BD4026E1E7022AF9D10024D6
:1095200040F20112C0E95444C0E95644A0F8442175
:1095300000F5A27156F097FAC6E700BF382A00205E
:1095400040190020092A0020F8B5234ED6F8143817
:109550000E2B04D80133C6F814380020F8BD0023C0
:10956000C6F8143816F8303C002BF6D11B4D2A698A
:10957000EB689A42F1D02A69EB689A4295BFEC6891
:109580002C692B69C4F5006498BFE41A402C1FD8DD
:10959000A7B2402F0CBF022301232A6906F8303CF2
:1095A0000F4B1344C0E9543340F201120023C0E9C9
:1095B0005673A0F8442100F5A27156F054FA2B69B5
:1095C0003B44C3F30A03E41B2B61C6F81048C4E70D
:1095D00001234027E1E700BF382A0020401900207E
:1095E000092A0020064BD3F88C391A79022A05D1B2
:1095F0009A68920702D5586954F0D8BE704700BFE8
:109600004019002038B5114D114CD4F88C0906F0E2
:10961000C3FB58B1013D15D194F850390133DBB289
:10962000072B84F8503901D984F85C59D4F88C0997
:109630000379022B08D183689B0705D5BDE8384024
:1096400008F0A4B900BFE0E738BD00BFA186010063
:109650004019002073B50A4E441C0025D6F88C0929
:10966000012300220DF1070156F0DEFE9DF80700F0
:10967000FF2802D10135A542F0D102B070BD00BF74
:109680004019002070B5044608200D46FFF7E2FFA0
:10969000FF2812D0FE2812D10A4E2B46D6F88C098C
:1096A0000022214656F0C0FE0022D6F88C09022383
:1096B000114656F0B9FE002070BD0120FCE70220E3
:1096C000FAE700BF4019002037B5124D4FF6FF539F
:1096D0000024D5F88C09ADF8043001AA02232146F4
:1096E000C5F8584956F0A0FE0120FFF7B3FFFF2848
:1096F00005D1042385F85C39022003B030BD09236D
:1097000085F85C39044B53F8343CC5F84C39204695
:10971000F3E700BF40190020382A002013B540F0BD
:1097200040038DF800300B0E8DF801300B0C8DF8D6
:1097300002300B0A8DF80330952304468DF804108F
:109740008DF8053056F096FE00B964B90748062337
:10975000D0F88C096A46002156F066FE0820FFF713
:1097600079FF02B010BDFF20FBE700BF40190020C9
:109770002DE9F041194C1E4694F85C39042B05463E
:10978000884617461CD1FFF72DFF94F85339FBB9D3
:1097900069021120FFF7C2FFE0B9052384F85C39A4
:1097A0000F4BC4F8388953F8343CC4F83C59C4F81A
:1097B0004479C4F84869C4F84C390120BDE8F08107
:1097C000082B03D1FFF780FF0228DCD00020F5E74B
:1097D0002946DEE7FFF716FFF8E700BF4019002033
:1097E000382A002038B500220D233821022006F047
:1097F000F3FE224CC4F88C0910B984F85C0938BD1A
:10980000002106F0DFF801200AF04EF8D4F88C5958
:10981000686906F0B0FC95F910301948194D14220A
:1098200002FB03000022D0F8B4000A23114656F0D0
:10983000D1FDD4F88C0906F0AFFA50B9124B84F878
:10984000500953F8343CC4F84C39012384F85C398E
:10985000D5E7013DEDD1D4F88C09022106F0B2F82C
:10986000D4F88C0906F082F894F85039C4F88C5971
:10987000013384F85C5984F85039C0E7401900205E
:1098800000000020A1860100382A002038B5134CC2
:109890000023A07BE0B125688D4219D1104C03F55F
:1098A00081751AB904EB0514A27138BD04F11801D1
:1098B00001EB43239A4209D1831E5842584104EBDD
:1098C000051455F093FE0123A371EEE70020F6E79F
:1098D0000133082B04F11004DBD1E6E7905D002092
:1098E000784D0020174838B5002380F8A03000F1EB
:1098F000180425688D421ED1A57B032D1BD1124C67
:1099000003F581754AB904EB05140423A371D0F85B
:109910009C300133C0F89C3038BD04F1180000EBD6
:109920004320131A5842584104EB051455F05EFECB
:109930000123A371F0E70133082B04F11004D8D1FF
:10994000EAE700BF785D0020784D0020F8B50446B6
:10995000144EFFF79EFD204602234022812155F040
:10996000B9FF402201212046022355F0B3FFD6F86B
:10997000183800251B6886F80C58284686F8D157F9
:109980009847E768384656F04BFB3846012156F0B9
:109990005DFB20461F2306F2D472012156F0FCF82D
:1099A0002846F8BD382A00202DE9F74F0F4601213F
:1099B00008460192984606F09FFFDFF87CA000243D
:1099C000A04532DD019B07EB442941F2893603EBC8
:1099D000040B0FE0FEF7A6FD013E08D10120002197
:1099E00006F08AFF4FF0FF3003B0BDE8F08F012092
:1099F00009F05AFFDAF83439002BEBD05B681D46CA
:109A000000231A4649465846A8470028E2D041F2AA
:109A1000893604E0013EE1D0012009F045FFFEF760
:109A200081FD0028F6D00134CAE70120002106F0AC
:109A300063FF0020D8E700BF401900202DE9F74F51
:109A40000F46012108460192984606F055FFDFF8BF
:109A500078A00024A04530DD019B07EB442941F2AA
:109A6000893603EB040B02E0012009F01DFFDAF850
:109A7000343933B941F28936FEF754FDB8B10134B7
:109A8000E8E7DB681D4600231A4649465846A847C2
:109A90000028EFD0FEF746FD013EE5D10120002170
:109AA00006F02AFF4FF0FF3003B0BDE8F08F013E13
:109AB000F4D0012009F0F8FEDEE70120002106F0D5
:109AC0001BFF0020F0E700BF40190020024BD3F835
:109AD0001C0807F089BE00BF382A00200068F02269
:109AE000FF2107F083BFCB4341EA0311CAB20068EC
:109AF000D22107F07BBF0068B422FF2107F076BFB8
:109B00000A460068A52107F071BF5521F8E70068F3
:109B10009622FF2107F06ABF0A460068872107F0F6
:109B200065BFCA01006802F08002782107F05EBFBD
:109B300038B50446154600680A46E12107F056FF8D
:109B400030B120682A46FF21BDE8384008F0DABE6F
:109B500038BD0A46E121EBE70A46C321E8E738B5FC
:109B6000021D0D46F0210446FFF7E2FF08B12379FC
:109B70002B7038BDF8B504460E461546071D206803
:109B80003A46FF2108F0BEFE30B116B12379DB075B
:109B9000F5D40DB123792B70F8BD00220121E9E73E
:109BA00010B50446FFF7A7FF18B12046BDE81040E6
:109BB000F3E710BD10B50446FFF7A2FF18B1204629
:109BC000BDE81040E9E710BD70B506460C468D189B
:109BD000AC4201D1012006E014F8011B3046FFF72A
:109BE000E9FF0028F4D170BDCC21E3E738B5044685
:109BF0000D46FFF78CFF40B12046FFF7CEFF20B1A6
:109C000029462046BDE83840A3E7002038BD70B59E
:109C100006460C468D18AC4201D1012006E02146D3
:109C20003046FFF7E3FF01340028F4D170BD38B5AA
:109C300005461446FFF770FF2846FFF7AEFF20B138
:109C40001CB12B79C3F34013237038BD10B5044603
:109C5000FFF7A6FF38B12046FFF7C6FF18B1204630
:109C6000BDE8104099E7002010BD73B50546CDE969
:109C70000023FFF795FFA8B12846FFF746FF88B1FC
:109C80002846FFF78AFF68B16E46082416F8011BC4
:109C90002846FFF78FFF28B1013C14F0FF04F5D1EF
:109CA00002B070BD0020FBE7C90138B501F08001AA
:109CB00004461546FFF735FF08B9002038BD0022DD
:109CC00001212046FFF756FF0028F6D023795B09D3
:109CD0002B70F3E710B5021D0446FF21006808F061
:109CE00011FE18B12079C04300F0010010BD0F49EA
:109CF000D1F8883043F47003C1F888300C4B1A68EF
:109D0000002042F001021A6098601A6822F0847202
:109D100022F480321A60074A5A601A6822F48022BC
:109D20001A60D860044B8B60704700BF00ED00E004
:109D3000003802401030002400000008704782B054
:109D40000023019300933C4B1A6842F480321A605E
:109D50001A6802F400320092019A01320192009ACC
:109D60001AB9019AB2F5A04FF2D11B6813F400336F
:109D700018BF01230093009B012B57D12E4B2F4975
:109D80001A6C42F080521A640A6842F440420A6037
:109D90009A689A609A689A609A6842F480529A60C7
:109DA000274A5A601A6842F080721A601A68900155
:109DB000FCD5244A40F2027111609A6822F0030235
:109DC0009A609A6842F002029A601B4B9A6802F00D
:109DD0000C02082AFAD19A6802F00C02042A27D051
:109DE000082A27D159685A685B684902C3F3881367
:109DF0004CBF1549154902F03F02B1FBF2F2534343
:109E00000D4A5268C2F3014201325200B3FBF2F331
:109E1000094A91680E4AC1F303110A4492F85C2082
:109E2000D3400C4AC2F8043102B0704700BFFDE7CE
:109E3000054BEDE7054BEBE70038024000700040B2
:109E400019304004003C024040787D010024F400B9
:109E5000C8460608000000200148FEF70DB900BF03
:109E60000C0100200148FEF707B900BF580300208D
:109E7000064A002352F83310814201D1D8B270470C
:109E800001330E2BF6D1FF20704700BF3447060880
:109E9000704770B5002828D04C684CB942681568E6
:109EA0005679AB8902229BB2B24023EA0203AB810E
:109EB0008A683AB943681D68AB8923F001031B0423
:109EC0001B0CAB81816044B1436819685D798C8952
:109ED0000223AB4023439BB28B8132B143681A68A3
:109EE00093899BB243F00103938170BD0B4B30B556
:109EF0001A4600241D79854208D1DD68294203D025
:109F0000142303FB042030BD0029F9D001340A2CAE
:109F100003F11403EED10020F5E700BFA0050020F7
:109F20000028ACBF00F16040064B4FEA0111ACBF06
:109F300000F5614000F00F00C9B2B4BF195480F8B9
:109F40000013704714ED00E038B503681B681C6807
:109F5000244B07EE902A93ED417AF8EE677AB8EE3B
:109F6000477A013987EE270A8DB2DFED1F7A30EE8E
:109F7000270A58F0B1F81D4A23880138944280B26C
:109F80009BB212D002F5806294420ED0B4F1804FA1
:109F90000BD0A2F58032944207D002F58062944241
:109FA00003D002F58062944206D123F070039BB285
:109FB00023F440739BB206E00D4A944203D002F5AD
:109FC00080629442F4D12380084BE5629C42208554
:109FD00003D003F580639C4201D100232386012333
:109FE000A38238BD000000200AD7233C00000140B6
:109FF00000100040F0B543689A795D7912F00400D2
:10A0000002F0020C11BF0022E6464FF48072844633
:10A010000FBF0124964604201446032D38D8DFE8EC
:10A0200005F0023872AC1B681D8C25F001052D046B
:10A030002D0C1D841D8C9F881E8B25F002052D0480
:10A0400044EA0E042D0C26F073062543634C3604B7
:10A05000360CA342BFB246F0600603D004F580641C
:10A06000A34209D14FF6F3742C4044EA0C0427F4C0
:10A07000407744EA000517439F801E8359631D847F
:10A080001A8B22F008021204120C42F008021A8302
:10A09000F0BD1D682B8C23F010031B041B0C2B84BC
:10A0A0002B8CAF882E8B23F020031B0444EA0E0474
:10A0B0001B0C26F4E64643EA0413484C3604360CDF
:10A0C000A542BFB246F4C04603D004F58064A54261
:10A0D0000CD123F0800343EA0C1323F040039BB21E
:10A0E00027F4406743EA001347EA8207AF802E83D4
:10A0F000A9632B842B8B23F400631B041B0C43F4F8
:10A1000000632B83C4E71D682B8C23F480731B042E
:10A110001B0C2B842B8CAF88AE8B23F400731B0499
:10A1200044EA0E041B0C26F0730643EA04232B4C6E
:10A130003604360CA542BFB246F0600603D004F5E3
:10A140008064A5420CD123F4006343EA0C2323F47A
:10A1500080639BB227F4405743EA002347EA021783
:10A16000AF80AE83E9632B84AB8B23F008031B0421
:10A170001B0C43F00803AB838AE71B68188C20F4A0
:10A1800080500004000C1884188C9E889D8B20F44D
:10A190000050000444EA0E04000C25F4E64540EAB1
:10A1A00004300E4C2D042D0CA342B6B245F4C0452C
:10A1B00003D004F58064A34203D126F4804646EA26
:10A1C00082169E809D83196418849A8B22F4006203
:10A1D0001204120C42F400629A8359E70000014015
:10A1E00043685A79032A0FD8DFE802F00205080B0A
:10A1F00018683430704718683830704718683C3039
:10A2000070471868403070470020704710B54368A9
:10A210001A685879084B0344012093F8DC40138CEA
:10A22000A0409BB223EA00031384138CA14019437E
:10A2300089B2118410BD00BFC846060870B5EFF39F
:10A240001184102383F3128845682A686E79134DB0
:10A25000938935F816509BB223EA05039381C368AE
:10A260009D682A6822F001022A601A695D681F2A27
:10A270004FF0200385BF203A93409340EB6098BF96
:10A28000AB60E3B283F31188C3689B6859601A68B6
:10A2900042F001021A600123037470BDC84606082B
:10A2A0000268137D012B04BF0223137592F82C1052
:10A2B0000CBF4FF400730023012904BF022182F870
:10A2C0002C1092F8441008BF43F48063012904BFA6
:10A2D000022182F8441092F85C1008BF43F4006336
:10A2E00001290DD1022182F85C1043F480534268A9
:10A2F000126800215162918989B20B43938101E078
:10A30000002BF4D17047034B0348D3F82018FEF715
:10A31000DDBC00BF382A00200000014010B5064C0B
:10A320000648D4F82018FEF7D1FCD4F840180448A9
:10A33000BDE81040FEF7CABC382A002000000140EA
:10A340000040014010B5064C0648D4F82018FEF72E
:10A35000BDFCD4F844180448BDE81040FEF7B6BC74
:10A36000382A0020000001400044014010B5064C8E
:10A370000648D4F82018FEF7A9FCD4F84818044879
:10A38000BDE81040FEF7A2BC382A002000000140C2
:10A3900000480140034B4FF08040D3F82418FEF7EB
:10A3A00095BC00BF382A0020024B0348D3F8281878
:10A3B000FEF78CBC382A002000040040024B034802
:10A3C000D3F82C18FEF782BC382A00200008004081
:10A3D000024B0348D3F83018FEF778BC382A002027
:10A3E000000C00400348D0F8743613B100F5CD607E
:10A3F00018477047000000200348D0F8943613B186
:10A4000000F5D16018477047000000200348D0F8DD
:10A41000B43613B100F5D56018477047000000202E
:10A420000348D0F8D43613B100F5D9601847704707
:10A43000000000200348D0F8F43613B100F5DD60C9
:10A4400018477047000000200348D0F8143713B1B4
:10A4500000F5E16018477047000000200348D0F87D
:10A46000343713B100F5E56018477047000000204D
:10A470000348D0F8543713B100F5E9601847704726
:10A48000000000200348D0F8743713B100F5ED60E8
:10A4900018477047000000200348D0F8943713B1E4
:10A4A00000F5F16018477047000000200348D0F81D
:10A4B000B43713B100F5F56018477047000000206D
:10A4C0000348D0F8D43713B100F5F9601847704746
:10A4D000000000200348D0F8F43713B100F5FD6008
:10A4E00018477047000000200348D0F8143813B113
:10A4F00000F6080018477047000000200348D0F815
:10A50000343813B100F628001847704700000020C7
:10A510000348D0F8543813B100F648001847704784
:10A5200000000020036823F00103036000230360A0
:10A5300043608360C3600361212343612A4B9842D7
:10A5400003D13D2243F8082C7047284B984204D190
:10A550004FF4746243F8202C7047254B984204D185
:10A560004FF4741243F8382C7047224B984204D1B0
:10A570004FF0746243F8502C70471F4B984203D140
:10A580001E4A43F8642C70471D4B984203D11D4A64
:10A5900043F87C2C70471C4B984203D11B4A43F86C
:10A5A000942C70471A4B984204D14FF03D5243F817
:10A5B000AC2C17E0174B9842C3D0174B9842C7D02A
:10A5C000164B9842CCD0164B9842D1D0154B98429E
:10A5D000D6D0154B9842DAD0144B9842DED0144BAB
:10A5E0009842E2D0704700BF1060024028600240ED
:10A5F0004060024058600240706002403D00002010
:10A6000088600240400F0020A060024000003D2012
:10A61000B860024010640240286402404064024076
:10A62000586402407064024088640240A0640240A2
:10A63000B86402402DE9F0410022012603250B6891
:10A6400006FA02F737EA030334D10368540005FA27
:10A6500004FE23EA0E0303600B79D0F800806FEA52
:10A660000E0C03FA04FE013B4EEA080E012BC0F863
:10A6700000E014D883680CEA030383604B79D0F8B8
:10A6800008C0A34043EA0C038360436823EA07033E
:10A6900043608B79476893409BB23B434360C368F8
:10A6A00005FA04F723EA0703C360CB79C768A34020
:10A6B0003B43C3600132102AC1D1BDE8F081204B79
:10A6C0009A6802F00C02042A10B534D0082A34D15A
:10A6D00059685A685B684902C3F388134CBF19492B
:10A6E000194902F03F02B1FBF2F25343144A526897
:10A6F000C2F3014201325200B3FBF2F3104C03608B
:10A70000A168124AC1F30311114491F8E010CB4043
:10A710004360A168C1F38221114491F8E01023FA4B
:10A7200001F18160A168C1F342310A4492F8E0204E
:10A73000D340C36010BD034BE0E7034BDEE700BF2F
:10A740000038024040787D010024F400C846060825
:10A75000F0B5446B8668A38923F400531B041B0CDB
:10A76000A3818579290201F4806C417901F001030C
:10A770008907218A4FEA053289B221F4405102F457
:10A78000005242EA01022282A289C5F3800722F424
:10A79000B0524FEA83034FEA073722F00C0248BF5A
:10A7A00043F008034CEA07011204120C0B43134355
:10A7B000A381A38A23F440731B041B0C85B0A382DE
:10A7C0006846FFF77CFF204B9C4203D003F5806373
:10A7D0009C4237D1039BA2891921170401FB03F383
:10A7E0004FF064014CBF7600B600B3FBF6F3B3FB49
:10A7F000F1F001FB10330201A08900044BBFDB0024
:10A800001B01323332334BBFB3FBF1F3B3FBF1F334
:10A8100003F0070303F00F0313439BB22381A38AC2
:10A820002A0755BF23F008039BB21B0443F008031B
:10A8300058BF1B0CA382A3899BB243F40053A3818E
:10A8400005B0F0BD029BC6E7001001402DE9F843BA
:10A850001E46204B9DF820509DF824709842894652
:10A8600090462CD13B462A4631460020FEF79AF905
:10A8700004460020C4E90700C4E90900C4E90B98B4
:10A880006571A660A7712046FFF762FFEA0707D54A
:10A89000636B4FF6DF721A80DA6842F02002DA60EA
:10A8A000626BAB0742BFD36843F08003D3609389E8
:10A8B0009BB243F4005393812046BDE8F883064BD6
:10A8C000984204D13B462A4631460120CEE7002477
:10A8D000F2E700BF0010014000440040816037E70C
:10A8E000417135E7817133E72DE9F043654F07EB9F
:10A8F000C00985B005464FEAC00899F86C0805F014
:10A90000ADFC064699F86D0805F0A8FC044699F8D8
:10A910006E0852F0B3F96B1CDBB21EB140F60C129C
:10A92000F28033721CB140F60C22E28023720422C2
:10A930003A21304605F052FC204604223A2105F027
:10A940004DFC07EB0803D3F868484F4B9C4263D19A
:10A9500003F5F2331A6A42F400121A621A6A22F4F8
:10A9600000121A62474497F86F38022B6ED0032BFF
:10A970006ED0464E464A012B18BF1646A78827F0D0
:10A980003F0768463F04FFF79AFE3F0C029A414B8F
:10A99000B2FBF3F398B20743A780218821F00101AD
:10A9A0000904090C21803C498E4253D13B4BB2FB38
:10A9B000F3F2013091B2042980B238BF042120841F
:10A9C000A18323889BB243F001032380238823F4CF
:10A9D000816323F002031B041B0C43F48063238078
:10A9E0004FF480432381238823F080031B041B0C36
:10A9F000238023889BB243F001032380284B03EB81
:10AA00004513012283F85928002283F8585883F807
:10AA10005A2805B0BDE8F083224B9C4209D103F5CA
:10AA2000F0331A6A42F480021A621A6A22F480022F
:10AA300097E71D4B9C4295D103F5EE331A6A42F419
:10AA400000021A621A6A22F400028AE7124E95E79F
:10AA5000124E93E706EB4606B2FBF6F291B2C2F352
:10AA60000B020AB941F001014FF4967253434FF4BF
:10AA70007A72B3FBF2F301339BB241F400412384B9
:10AA80009EE700BF000000200054004000350C008D
:10AA9000801A060040420F00A0860100400D03000E
:10AAA000382A002000580040005C00402DE9F047A3
:10AAB000BC4E440106EB401908F004FE99F95828F1
:10AAC000B94B8846D10003EBC2020746D2F868585A
:10AAD00099F85A28013A142A00F28380DFE812F02C
:10AAE00079008900A200BB00C900D300DF00F80094
:10AAF00006010F011D0170018F01B9012A023E02FA
:10AB000050025C027002930215005F184FF0090AB0
:10AB100097F86C0805F0A2FB054697F86D0805F05C
:10AB20009DFBB6F8B83801339BB207462846A6F815
:10AB3000B83805F020FB384605F01DFB11212846EA
:10AB400005F023FB1121384605F01FFB4FF0650887
:10AB500003E00520002108F007FE284605F002FB6F
:10AB600010B9B8F10108F4D1284605F009FB00211D
:10AB7000052008F0F9FD284605F0FDFA0520002122
:10AB800008F0F2FDBAF1010AE0D1284605F0F8FA22
:10AB90000021052008F0E8FD384605F0F1FA002113
:10ABA000052008F0E1FD284605F0E5FA0520002122
:10ABB00008F0DAFD384605F0DEFA331993F9580843
:10ABC000431C01D0FFF790FE3319002283F85A2866
:10ABD00007E02B8813F4007340F0ED81321982F8FE
:10ABE0005A38331993F85A38002B7FF465AFBDE813
:10ABF000F0872B8823F400631B041B0C2B802B880D
:10AC00009BB243F480632B802B889BB243F4807308
:10AC10002B803319032283F85A28644B1A191F51C9
:10AC2000C2F8048062492846FDF7D1FA002800F0F6
:10AC3000C281331993F86A285AB993F86B28FF2A0E
:10AC400004D193F868280AB10A22BFE73319042215
:10AC5000BCE70F22BAE7321992F8693803F0FE0315
:10AC60002B82052382F85A38504B1A191F51C2F80B
:10AC7000048050492846FDF7AAFA002800F0938185
:10AC800033190622A2E7331993F86B282A82072288
:10AC900083F85A28454B1A191F51C2F804804649B7
:10ACA0002846FDF794FA002800F07D813219D2F889
:10ACB0006C385BB92B889BB243F400732B803B4B01
:10ACC00019191F51C1F80480012388E7082386E77A
:10ACD0002B889BB243F480732B803319092283F8AD
:10ACE0005A28324B1A191F51C2F80480304928469D
:10ACF000FDF76DFA002800F05E813319A4E73219E0
:10AD000092F8693843F001032B820B2382F85A38FA
:10AD1000264B1A191F51C2F8048028492846FDF70E
:10AD200056FA002800F03F813319D3F86C38012B14
:10AD30001DD12B8823F480631B041B0C2B80EFF3A5
:10AD40001182102383F312882B8B2B889BB243F440
:10AD500000732B80D3B283F311880C23321982F84D
:10AD60005A38124B1A191F51C2F8048039E7022BC6
:10AD700015D12B889BB243F400632B80EFF3118233
:10AD8000102383F312882B8B2B8823F480631B04FE
:10AD90001B0C2B80D3B283F311880D23DEE72B8BA2
:10ADA0000E23DBE7382A0020000000209832002024
:10ADB0000100030082000700840007000200030076
:10ADC00098492846FDF70DFA974A002800F0A2801E
:10ADD0003319D3F87018481CC3F87008288A087013
:10ADE000D3F86C1801391019C3F86C1801211751E8
:10ADF00083F87418C0F8048083F85A18F1E68B4978
:10AE00002846FDF7EEF9884A002800F08380EFF32A
:10AE10001181102383F312882B889BB243F40073B3
:10AE20002B803319C9B2D3F8700800F1010CC3F8B4
:10AE300070C8B5F810C080F800C081F31188D3F84D
:10AE40007018481CC3F87008288A08706FF0010158
:10AE5000C9E776492846FDF7C4F9734A002859D056
:10AE60003319D3F86C18032930D1298821F4806173
:10AE70000904090C2980EFF31180102181F3128855
:10AE8000D3F8701801F1010CC3F870C8B5F810C000
:10AE900081F800C0298889B241F400712980C1B2CB
:10AEA00081F31188D3F87018481CC3F87008288AF9
:10AEB0000870D3F86C180239C3F86C180C2183F8A9
:10AEC0005A1813191751C3F804808AE6022914D8B6
:10AED000298821F480610904090C2980298889B214
:10AEE00041F400712980298A1751002183F87418D0
:10AEF0001119C1F80480012268E6D3F87018481CC3
:10AF0000C3F87008288A0870D3F86C180139C3F8A0
:10AF10006C18D6E7131912595B68BA1A42F210710D
:10AF200068EB03038A4273F10003FFF45AAE33194E
:10AF300015224BE62B8823F4806332191B041B0C6B
:10AF40002B8092F8693803F0FE032B82102382F8DD
:10AF50005A38354B1A191F51C2F804803449284613
:10AF6000FDF735F9F8B1331993F86B28FF2A04D1AE
:10AF700093F868280AB1132228E63319112225E62E
:10AF8000331993F86B282A82122283F85A28264B09
:10AF90001A191F51C2F8048026492846FDF717F9EF
:10AFA00008B13319E7E724492846FDF71AF910B12B
:10AFB000331914220AE61C4B19191A594B68ACE7CD
:10AFC00033191949D3F86C2882B1D3F87008013AC3
:10AFD00010F801CBA5F810C0C3F86C280A190F515E
:10AFE000C3F87008C2F804801222EFE52A8892B2F2
:10AFF00042F400722A800A190F51C2F8048001221B
:10B0000083F87428E2E52B889BB243F400732B800D
:10B010004FF6FF33AB82044B1A191F51C2F804805C
:10B02000331968E740000010983200200400001037
:10B0300082000700840007000004001038B5114C9E
:10B0400004EB401494F85958D5B1C4F86C38049BFB
:10B05000C4F87038002384F874380223490084F857
:10B060006B2884F85A3801229DF8143084F8691846
:10B0700084F86A2884F86838FFF718FD94F8745843
:10B08000284638BD382A002038B5114C04EB40144E
:10B0900094F85958CDB1C4F86C38049BC4F8703892
:10B0A0000223490084F86B2884F85A3800229DF85E
:10B0B000143084F8691884F86A2884F8742884F8AD
:10B0C0006838FFF7F3FC94F87458284638BD00BF81
:10B0D000382A002082B000230193054B0193019B85
:10B0E00003EB80030193019B196002B0704700BF1E
:10B0F0005028004082B000230193054B0193019B2F
:10B1000003EB80030193019B186802B0704700BFF6
:10B110005028004010B51C2005F0A0F8112104466D
:10B1200005F033F8204605F02BF8C82008F0BCFBEA
:10B130002046BDE8104005F01EB8436D064A1A616E
:10B14000C278012A06D100F2CC5058611A684FF03B
:10B1500080221A60704700BF1800086038B50446A6
:10B1600000296DD190F81131022B28D1D0F8382167
:10B17000D0F824118A4230D9C378012B02BFD0F80D
:10B1800028315B18C0F82831521AD0F82831C0F89D
:10B1900038214FF48071002592B2A0F81C11C0E94B
:10B1A0004A33C0F83451C0F8302100F58E7154F0A4
:10B1B000DBFB2B462A462946204654F0EDFC94F84A
:10B1C0001631012B07D1244A2369D2F804285A608A
:10B1D000002384F81631002038BDD0F83C31B3FB91
:10B1E000F1F501FB1535A5B9994212D8D0F84021E7
:10B1F00093420ED24FF48073C0E94A55C0E94C55D2
:10B20000A0F81C3100F58E7154F0AEFBC4F840512B
:10B21000CFE7D4F8E435DB682BB194F81221032A88
:10B2200001D120469847052384F811310023204698
:10B230001A46194654F0B0FC2046FFF77EFFBEE7E1
:10B24000D0F8E4355B69002BC5D090F81221032AB1
:10B25000C1D19847BFE700BF382A00207047704728
:10B26000704710B50F4C94F8DA3AB3B14FF0E022C2
:10B27000D2F8103D23F00603C2F8103DFEF737FD6B
:10B28000D4F8E03A9B68DB0707D5D4F8DC2B1368C9
:10B2900023F0030161F307031360034B4FF4802293
:10B2A0005A6110BD40190020003C01402DE9F04FCB
:10B2B000B14CD4F8DC3A5A69D0078BB000F19681D2
:10B2C0005A699B6912EA030A00F09081CAF30743A6
:10B2D0001AF4002F01930FD0D4F8E03ADFF8A082DF
:10B2E0009E69DB691E40360C04F6243B04F52D698B
:10B2F0000027002E40F07D81019B59070DD5D4F821
:10B30000E03A9E4D9F69DB691F40BFB205F1180608
:10B310004FF00008002F40F0AD811AF0020F1FBF60
:10B32000954BD3F8DC3A02225A61BAF1000F5FFA6A
:10B330008AF51BDA904B93F8DA2A3AB1D3F8DC2B72
:10B34000136823F0030161F307031360D4F8E02AC4
:10B350008A48536823F001035360894BD3F8983827
:10B360009847D4F8DC3A4FF000425A611AF4006F63
:10B37000CAF307262FD000238DF8173094F8E23B4C
:10B380008DF817307E4B7D48D3F894389847D4F821
:10B39000DC2AD4F8E03A4FF400619B68516194F8DC
:10B3A000DA2AC2B1DB0716D594F8E53B012B12D19E
:10B3B0009DF81730032B0ED1D4F8DC3B1A6842F00D
:10B3C00001021A601A6842F003021A606D4A13699A
:10B3D00043F0060313612F0708D5694B6748D3F87C
:10B3E0008C389847D4F8DC3A08225A61ED0614D517
:10B3F000D4F8DC1A8B6923F010038B610B6AC3F35A
:10B400004342022A03F00F0500F0E981062A00F00A
:10B410000D828B6943F010038B61F00633D5D4F8AD
:10B42000E05AD4F8DC8A6B68002723F001036B60D4
:10B430003946404654F00AFE94F8D1CA5249B946FA
:10B440003B46FF206345C0F000824FF0FF33AB6105
:10B450004FF00113EB610B2363F3070763F3070955
:10B460006F61C5F810902B68444823F4FE632B608D
:10B47000FFF763FE4FF48053C8F81430404B3F4849
:10B48000D3F890389847B1066DD5D4F8E06AD4F86F
:10B49000E82AB3681168C3F34103022B14BF0023E9
:10B4A000032363F30A011160736843F480737360CC
:10B4B00006A8FFF704F9D4F8DC5A0799E86820F4E5
:10B4C0007050E860B36813F0060FC3F3410200F058
:10B4D000C3812E4B2E4A0B44934240F2C1812D4A28
:10B4E000A1F57403A3F51053934240F2BD812A4B9A
:10B4F0002A4A0B449342C0F0BB81294AA1F18C73C4
:10B50000A3F54343934240F2B781264B264A0B44AE
:10B510009342C0F0B581254B254A0B449342C0F0BD
:10B52000B381244AA1F1B773A3F558539342C0F0F5
:10B53000AE81214B214A0B449342C0F0AC81204B99
:10B54000204E0B4401224021B34234BF0623052381
:10B55000094E63F38D204FF40053E86086F8D22A39
:10B56000A6F8D41A6B61019BDA0632D5044B034866
:10B57000D3F89C38984727E0401900201024002079
:10B580000000002000ED00E024240020401E1BFFEE
:10B590003F420F00DFC810002013FBFE20D613002F
:10B5A000FF69180000D3CEFE40771B00C05BB3FEDE
:10B5B000C091210040AC2700C01D6AFE40E133006D
:10B5C000803C36FEE09C4100D4F8DC3A4FF4801217
:10B5D0005A61019B9B0609D5B14BB248D3F8A038FC
:10B5E0009847D4F8DC3A4FF400125A610BB0BDE82A
:10B5F000F08FF10737D5DBF80010D4F8E03A8D680A
:10B600005B691D40EA071ED594F8D33A0125AB4289
:10B610008D6007D10969D9F87C33C1F312015B1A37
:10B62000C9F88C33D8F880389E48F9B2984794F816
:10B63000D33A012B07D137B994F8E13B052B02D15E
:10B640009848FFF77AFDAB0742BFDBF800300225D0
:10B650009D60280707D5D8F8883892489847DBF8C6
:10B66000003008229A60013776080BF1040B09F1CB
:10B6700028093EE6FA0772D5D4F8E03A326818692C
:10B68000D3F83490916829FA08F94FEAC9195FFA9A
:10B6900089F949EA000909EA010919F0010F1FD0E7
:10B6A000596B012000FA08F021EA000159637C4B34
:10B6B0007C48D3F884384FF00109C2F808905FFA4B
:10B6C00088F1984794F8D33A4B4509D1B8F1000F67
:10B6D00006D194F8E13B042B02D17248FFF72DFD0F
:10B6E00019F0080F1EBF33684FF00809C3F808901F
:10B6F00019F0100F1EBF33684FF01009C3F80890FF
:10B7000019F0400F1EBF33684FF04009C3F808908E
:10B7100019F0020F1EBF33684FF00209C3F80890FA
:10B7200019F0800F1BD0D5E94C329B1AD5F8242193
:10B73000D6F800B0934228BF13465B4ADBF81800E6
:10B7400092F8D3CAD2F8E09A03339B080293029B83
:10B7500080B2984203D9D5E94C03984205D808F144
:10B7600001087F0828350436D4E5C01AD5F82431FD
:10B77000984228BF1846C31C9B080293BCF1000FD7
:10B780001BD0D5F82811D5F834210144C5F828116B
:10B79000D5F8301102448A42DBF81800C5F834218C
:10B7A000D5D195F81C11D9F83420012303FA01F101
:10B7B00022EA0102C9F83420C9E782B2D6F8B810EB
:10B7C000D5F828E10332931003930A466146039BA0
:10B7D0008B42D6D05EF8213013600131F7E747F68F
:10B7E000F0721A423FF415AE282202FB0542C3F361
:10B7F0000A13D2F8507ED4F8A0CBDA1C92100020A5
:10B8000082420DD1282202FB0542D2F8500E184484
:10B81000C2F8500ED2F85C0E1844C2F85C0EF8E57F
:10B82000DCF800E047F820E00130E9E7D4F8A00BAD
:10B830001E4A0768C2F89C700068C2F8A00028225F
:10B8400002FB0542C3F30A13E4E751F8042F9060AA
:10B85000CA6B01339060F5E54FF40071092377E678
:10B86000012240210E2373E6012240210D236FE6C1
:10B87000012240210C236BE6012240210B2367E6C5
:10B88000012240210A2363E601224021E6E701224A
:10B89000402108235CE601224021072358E600BF2F
:10B8A0000000002010240020401900204029002022
:10B8B000034BD3F8880908B104F054BC0120704749
:10B8C0004019002008B5FFF7F3FF0A4A18B9002312
:10B8D00082F85C3908BD92F850390133DBB2072B8E
:10B8E00082F85039F3D8044B53F8343CC2F84C3941
:10B8F0000123EDE740190020382A0020F0B5C54C9F
:10B90000D4F88C0985B0002861D094F85C39013BEB
:10B91000082B44D8DFE813F009005D00DF00430086
:10B92000AA01300186014300E601FDF75BFE00211C
:10B930000846FDF7F3FE0546FDF764FE012D29D10B
:10B94000002684F85269FDF74DFE40F2AB11082045
:10B95000FDF7E4FE05280AD184F85259FDF752FE9E
:10B9600094F85239A3B1022384F85C39CDE7012859
:10B97000F4D10423D4F88C093246694654F054FDBE
:10B980009DF80330AB2B04BF022384F85239E5E75E
:10B9900084F85C39D4F88C09022104F013F894F887
:10B9A0005C39013B022B09D89B4BD4F84C2953F846
:10B9B000343C9B1AC82B01D9FFF784FF94F85C092B
:10B9C000042800F0A081A0F108035842584105B0B6
:10B9D000F0BDFDF707FE94F85259AA1E5542554195
:10B9E000AD0700213720FDF799FE29462920FDF7F4
:10B9F00095FE0546FDF706FE002DCBD194F8523991
:10BA0000022B17D1FDF7EEFD29463A20FDF786FE01
:10BA1000042306462A46D4F88C09694654F004FDEE
:10BA2000FDF7F0FD16B1FFF74DFF6EE7009D2DBA53
:10BA3000C5F3807584F85359FDF7D4FD0021092022
:10BA4000FDF76CFE10B1FDF7DDFDA3E77348102193
:10BA5000FDF718FE06460028F5D101217F2050F0A1
:10BA600075FF01280546EED10221304650F06EFFE9
:10BA700050B10128E7D116213A2050F067FF01307C
:10BA80008002C4F8600918E004212C2050F05EFF09
:10BA9000032107464E2050F059FF0C210646362060
:10BAA00050F054FF0236431CB340BD40A3FB0535A4
:10BAB0005B0A43EAC553C4F86039FDF7A3FDFDF7FF
:10BAC00091FD00210A20FDF729FE08B903234BE769
:10BAD000FDF798FDA7E710216846FDF7D3FD002884
:10BAE0007FF458AF9DF8003084F86639BDF8013016
:10BAF0005BBAA4F864399DF8033084F86739019B78
:10BB0000C4F868399DF808301A0903F00F0384F867
:10BB10007139DDF8093084F870291BBAC4F86C3922
:10BB20009DF80D309DF80E201B01DBB243EA121385
:10BB300003F5FA6302F00F02A4F8723984F874294D
:10BB4000FDF760FD94F853394BB1D4F88C0902210C
:10BB500003F038FF0023C4F85839042304E7FDF745
:10BB600041FD4FF400711020FDF7D8FD0546FDF7AB
:10BB700049FD002DE9D056E794F84019D4F838294A
:10BB8000D4F88C09802302EBC112002154F04CFC44
:10BB900094F840390133DBB2042B84F840397FF448
:10BBA000FEAE1F4AD4F88C090223002154F03CFC5D
:10BBB0000123D4F88C090022694654F035FC9DF825
:10BBC000003003F01F03052B15D1072384F85C39DF
:10BBD000114BD4F8445953F8343CC4F84C39002D77
:10BBE0003FF4DDAED4F84839D4F83829D4F83C19FC
:10BBF0000120A847D3E6FFF765FED4F84459002D8D
:10BC00003FF483AED4F84839D4F83C19002201201F
:10BC1000A8477AE640190020382A0020B8220020E0
:10BC2000B847060854F026FC002862D0002384F8A8
:10BC30005039D4F85839012B0BD9013BC4F8583985
:10BC4000D4F854390133C4F85439082384F85C39E2
:10BC5000A5E607D1FDF738FD02287FF4A0AEFDF779
:10BC6000D1FC9CE6042384F85C39F8E7D4F8380961
:10BC70004FF40071FDF706FD0128054619D0022892
:10BC800020D000287FF48BAEFDF7BCFCD4F84469CB
:10BC900084F85059042384F85C39002E3FF47FAEB9
:10BCA000D4F84839D4F83829D4F83C192846B04794
:10BCB00075E6164B53F8342CD4F84C396433934260
:10BCC000BFF46DAEFDF79EFCFFF7FCFDD4F84459C0
:10BCD000002D3FF41AAE0022D4F84839D4F83C19AC
:10BCE000104695E754F0C6FB18B1FDF78BFC042312
:10BCF000ACE7064B53F8342CD4F84C39FA33934262
:10BD0000FFF491AE4BE6012061E600BF382A002027
:10BD10002DE9F341284C05460E4690461F4694F8FF
:10BD20005C39042B0DD0082B07D1D4F85439AB4221
:10BD300019D0FDF7C9FC0228F1D0012002B0BDE8FE
:10BD4000F081FDF74FFC94F8533953B9690218207C
:10BD5000FDF7E4FC38B1FDF755FCFFF7B3FD032018
:10BD6000ECE72946F3E794F85C39D4F88C09082B02
:10BD700014BFFE23FC23FF228DF804208DF805302C
:10BD800001AA0223002154F04FFBD4F88C09802330
:10BD90003246002154F048FB012384F84039062341
:10BDA000C4F83869C4F83C59C4F84489C4F84879DF
:10BDB00084F85C390020C1E74019002070B51C4CA4
:10BDC00094F85C39042B05460E4610D1FDF70AFCA9
:10BDD00000213720FDF7A2FC31461720FDF79EFC1D
:10BDE00090B1FDF70FFCFFF76DFD032002E0082B7B
:10BDF00001D0012070BDD4F85439834214D0FDF72E
:10BE000063FC0228F5D1E1E794F8533973B969026C
:10BE10001920FDF783FC0028E3D1082384F85C395E
:10BE2000C4F85869C4F854590220E3E72946EFE7FB
:10BE300040190020034BD3F8340908B1436918476F
:10BE4000704700BF40190020034BD3F8340908B1F4
:10BE500083691847704700BF40190020002110B5C2
:10BE6000084604F049FDFFF7EFFF40B90F4B104AB9
:10BE700003F6AC01C2F83419D3F8AC389847002463
:10BE800003E00120013407F00FFDFCF74BFB10B974
:10BE9000B4F57A7FF5D10121002004F02DFDB4F531
:10BEA0007A7F4FF0FF3018BF002010BD0000002047
:10BEB00040190020034BD3F8340908B1C36918476F
:10BEC000704700BF4019002038B50D461446FFF7F3
:10BED000F1FF03682B604FF400732360002038BD2E
:10BEE000034B1B78032B14BF4FF4807080207047E6
:10BEF000784D002008B50B4A68B1816811B107235D
:10BF0000937008BDFFF7ECFFC2E90311C2E901001D
:10BF100011750423F4E702F58051012381F8B4314F
:10BF20005370EEE7784D002010B502784368022A7E
:10BF30000B4A06D1D2E9802102EB410202EB5320E9
:10BF400010BD0169D2F81802D2F810421840023927
:10BF5000D2F80C32400A04FB01001844F0E700BF9D
:10BF6000785D0020064B1B78022B0BBF030AC0F341
:10BF7000D413C0B200F07F000B601060704700BFA8
:10BF8000784D002090F91A305A1C0AD003F58172BE
:10BF9000124B03EB0213DA7922F00102DA71FF236C
:10BFA000837690F91B104B1C16D00C4A01F5817159
:10BFB00002EB011302EB0112DB79D179C3F34503E4
:10BFC000012B86BF03F1FF3303F03F03002363F32C
:10BFD0004601FF23D171C376704700BF784D002022
:10BFE00008B5FFF77DFF034BD3F8103258434002EA
:10BFF00008BD00BF785D00200378022B09D10E4BED
:10C00000D3F820224368B3EB422F2CBF012000203D
:10C010007047006970B1094B1B78032B0EBF084BAA
:10C0200080B24FF6F773984294BF0020012000F0D1
:10C03000010070470120FAE7785D0020784D00206C
:10C04000F7FFFF0F4368F7B5C3F308020A44B2F5E0
:10C05000007F04460D4604D22B446360012003B0E8
:10C06000F0BDFFF78FFF0378022B01D16368F3E780
:10C07000154BD3F81022B5EB422F4FEA422706DCCE
:10C08000D3F8183246681E407342AB4201DD0020EF
:10C09000E5E7AB19BB4210D30169007E01AA53F05A
:10C0A00085FB0128F3D123696361019B23616368E8
:10C0B0003B449B1BEF1B6360BD192046FFF79CFFB1
:10C0C0000028CBD1D2E700BF785D002070B50446D0
:10C0D0000E461546FFF7B6FF20B10DB12046A84722
:10C0E000012070BD94F82800022320B9C4E90B5642
:10C0F00084F82830F5E71846F3E738B5174D05F50D
:10C100008054014694F8E00130BB49B191F82830E1
:10C110002BB9442204F5DC7058F088F8012038BDB2
:10C1200044220F4858F0C6F84FF6FF73A4F8D231F6
:10C13000032384F8D0312B780948022B18BF03233E
:10C1400084F8B831D4F81C32C4F8DC31102384F8F8
:10C15000D13150F0C5FDE1E70020E0E7784D002047
:10C16000305F0020044A92F8B411012309B982F823
:10C17000B431024A53707047785D0020784D00203A
:10C180002DE9F74F12F002098A461546019304D0B3
:10C1900018B9FFF7E7FF02200CE0684AD2F80862FE
:10C1A0005EB1D2E9831404FB0611884205D3FFF780
:10C1B000D9FF002003B0BDE8F08F4FF0FF31604E93
:10C1C000DFF880B18C468E46884600243368B77B02
:10C1D000984221D1002F46D0D2F89810594E013103
:10C1E000C2F8981004F581721201B1502146554CE5
:10C1F00001F5817604EB06129279042AC9D801A7C9
:10C2000057F822F09BC20008F1C20008B3C1000831
:10C21000F1C2000805C300080FB3012F10D104F5C7
:10C2200081770BEB0717FF79FB0709D417F07E0F17
:10C2300006D1FF0915D1B76847453CBFA446B846AB
:10C240000134082C06F11006C0D100290CDABEF129
:10C25000000F20DABCF1000FABDB614604E02146A1
:10C26000EEE7A646ECE72146364E41F2180406EB0F
:10C2700001173851D2F898400134C2F8984041F281
:10C280001C02BC5001F58172170106EB0212F45139
:10C2900000245460ABE77146E6E715F0010213D0C5
:10C2A000294BD3F83439002B83D0284F5D68284AB6
:10C2B000002307EB4121A84700283FF47AAF04EBA5
:10C2C00006140223A37174E704EB0610019B90F897
:10C2D00007C0EF1067F3C71C032B80F807C02BD9EA
:10C2E0004FF6FF72934228BF134604EB0612938069
:10C2F000B9F1000F06D004EB011000F580501830A2
:10C30000FCF732F96A0741BF04EB0612D37943F018
:10C310000103D371EB0608D504EB0614E379C3F3EC
:10C320004502013262F34603E371084B03EB4123FC
:10C33000CAF8003001203DE71346D6E7785D0020BB
:10C34000905D0020784D002040190020904D002085
:10C350008D9800087FB50F4D01AA0C4602A9FFF782
:10C3600001FE05F58053029ED3F80002032200234C
:10C3700003A93044FFF704FF012808D12978039B63
:10C38000019A02290CBF23F8124043F8224004B05E
:10C3900070BD00BF784D00202DE9F04FD1F800901E
:10C3A00085B01646074601AA48460D4602A9FFF782
:10C3B000D9FD374A0299D2F8003201EB0308019BFC
:10C3C000013B9C19FFF78CFDA4EB09040444A2F582
:10C3D000805AB4FBF0F408EB04092B68B342A9EBD4
:10C3E000080103D3012005B0BDE8F08FDDF804B0EB
:10C3F0000BEB0604E41AFFF773FD844228BF0446E2
:10C40000BBF1000F1AD1A0428CBF0B220A220B46AF
:10C41000404603A9FFF7B4FE0128E4D19AF80010C2
:10C420002B68039A022903F1010358460CD0A0425D
:10C430000CD242F8203001300133F8E70B22E6E756
:10C4400022F8103001300133A042F9D32B68A3EB5E
:10C450000B032344012F2B6014D1B34212D10229C4
:10C460000BBF04F1004404F1804304F1FF3403F1F5
:10C47000FF330BBF4FF6FF734FF0FF3122F814303C
:10C4800042F82310002308F101080193A5E700BF3B
:10C49000785D00202DE9F04F85B00546FFF720FDBF
:10C4A0000C461746814601AA206802A9FFF75AFDEB
:10C4B0006B1E012B66D9019B4BB94E46DFF8C88035
:10C4C000012D8CBF00250125A8F5805A1BE0FFF740
:10C4D00049FE02202BE0D8F87831C3B1D8F8941186
:10C4E000914214D1D8F81022013B500203EB4223B1
:10C4F000B3FBF0F30B44B3FBF6F206FB12320AB1C6
:10C5000033449B1A23602268BA42E4D32BE0DDF85F
:10C5100008B0D8F800020023092203A95844FFF705
:10C520002FFE012806D00228D3D00028EBD105B079
:10C53000BDE8F08F9AF80010019A022907D003296C
:10C54000C7D1039B53F8223023F0704302E0039BD2
:10C5500033F81230D4F800C0B3FA83F35B09AB426E
:10C5600004D16745E3D827600320E0E732440CEBB1
:10C57000060391452360E0D80BF1010302930023E9
:10C580000193C0E7012699E7785D002037B504469E
:10C59000C0690D4610B9012003B030BD002303224D
:10C5A00001A9FFF7EDFD0128F6D1B4F92030002BE9
:10C5B00017DB019A012D4FEA431102EB431316D00A
:10C5C000022D12D0E268DA612278032A04D1002217
:10C5D0001A775A779A77DA77626A5A83110C9982B6
:10C5E000D9E7FFF7BFFD0220D6E7E5205054A26847
:10C5F000E9E738B5044694F83430052B2FD8DFE846
:10C6000003F00727353C444D022084F83400F2E75C
:10C61000294DD5F8082204F1300102320120FFF73C
:10C6200039FF012805D00238C0B2012817D80520EB
:10C63000EBE7D5F81012E268236BC5F8143202EB71
:10C640004122E260E26A2361002ADED16362DCE714
:10C65000206B4FF0FF31FFF77DFE012801D0002055
:10C6600038BDE36A002BCFD10320CEE7D4E90B011C
:10C67000FFF770FE0128F7D0F1E700212046FFF711
:10C6800085FF0128EBD10420BFE794F82830082B60
:10C6900004BF002384F828300120E1E794F8283013
:10C6A000082B04BF002384F82830034B012283F8B1
:10C6B000B5210220D4E700BF785D00202DE9F341C9
:10C6C000044694F83830032B0ED8DFE803F0061147
:10C6D000767F032084F83800F3E72046FFF789FFD0
:10C6E0000128F7D00228F4D0002002B0BDE8F08184
:10C6F00023786568DFF8E480022B1CBF374BD3F842
:10C700001832204618BF1D40FFF70EFCC5F34F2519
:10C710002D1A0646ADB20023022201A93046FFF7CA
:10C720002FFDAF190128BFB2DFD101984FF400727D
:10C73000002157F0BFFDE3692BB363681BBB019B6E
:10C740004FF020322E211970C3F80120C3F80520C4
:10C75000A3F80920606A58834FEA104C102083F830
:10C76000201083F82110D872C3F82220C3F82620A5
:10C7700083F82A20E26BA3F814C022FA00F199860C
:10C780005A8783F82B00D8F810124B1E9F4208D20C
:10C790004FF400712046FFF755FC52F027FF013699
:10C7A000B9E7C1EBC151490201F500712046FFF71D
:10C7B00049FC52F01BFF02208CE7002384F828304C
:10C7C000236C0BB12046984701208EE7236C002094
:10C7D00084F8280003B19847022086E7785D00209E
:10C7E00010B5044694F83830032B53D8DFE803F033
:10C7F0000631434D022384F83830F3E72649D1F857
:10C8000094212261FFF7ECFBE3680344E360FFF748
:10C8100067FB1044C1F89401FFF7E2FBD1F87831CF
:10C820001B1AC1F87831FFF7DBFBD1F87C311B1AFA
:10C83000C1F87C312263FFF753FBE36A1044606365
:10C8400013B962620123D6E7FFF74AFB121A22638B
:10C85000F8E712480021FFF799FE0128CAD0431ECD
:10C86000DBB2012B06D894F82830062B04BF002336
:10C8700084F8283010BD626B04F130010120FFF70D
:10C880008BFD0128EBD10323B5E700212046FFF7FC
:10C890007DFEE4E70220E2E7785D0020E85E00200C
:10C8A0002DE9F74306460C464FF6F77596F83C30EF
:10C8B000042B73D8DFE803F0290736416300032017
:10C8C00086F83C00F2E73A4FDFF8EC8007F5805934
:10C8D0003B78306B032B4FD140454BD801A950F02A
:10C8E00011F8012857D1306B0021FFF733FD0128E3
:10C8F00051D1019B3363D9F81422013B934294BF79
:10C90000C9F81432C9F81422E2E7610001F0FE010F
:10C910003046FFF73BFE01280CD1736B002B18BF8C
:10C920000220CDE7726B06F130010020FFF734FDE5
:10C930000128C4D002282ED131E01E48F26AD0F876
:10C940009431C0F894219B1AD0F810225343D0F8A8
:10C95000782102EB4322C0F87821D0F87C2102EB49
:10C960004322C0F87C21002100F5B870FFF70EFECD
:10C970000128DFD10420A3E783B2AB42ADE796F8EC
:10C980002830042B04BF002386F82830B36B0BB18A
:10C9900030469847012003B0BDE8F083022096F8A6
:10C9A0002830042B04BF002386F82830F3E700BFAB
:10C9B000784D0020785D0020F7FFFF0F70B50378F9
:10C9C000027E023B012B04461CD8237E990622D40A
:10C9D0002046FFF7D7FA237E1A070AD51E4D95F891
:10C9E0009801C31F5842584152F000FE002385F8B9
:10C9F00098310023237084F82830E36A53B1BDE8EE
:10CA00007040184712F0060FDFD00121FFF7BEFD7E
:10CA10000128DAD070BDE2691049002318010858D6
:10CA2000824211D10E4903F5817201EB0213DB79C9
:10CA3000C3F34503012B0BD8002301EB0212D1797C
:10CA400063F34601D171C3E70133082BE6D1BFE799
:10CA5000013B03F03F03F0E7785D0020905D00208C
:10CA6000784D002010B580B1027872B190F828207E
:10CA70006AB9D0E9012494422CBF84608260032209
:10CA800080F82820C162FFF799FF012010BD002027
:10CA9000FCE7B1F904300F2B2DE9F34104460D46B4
:10CAA00016460BD14FF40071FFF7CCFA18B90020ED
:10CAB00002B0BDE8F0814FF6FF73AB802046FFF770
:10CAC00033FA94F91B20531C074624D0244B41F21F
:10CAD000180103EB021041588F4212D1183303EBB7
:10CAE00042230193019A72B1AB8801331BB202EB6E
:10CAF0004312AB8020463260FFF716FA286001200F
:10CB0000D6E7FFF72FFB2046FFF776FA0028CED0B6
:10CB100000233360F3E72046FFF76EFA80460028D3
:10CB2000F1D1381E18BF012052F060FD434611229A
:10CB300001A93846FFF724FB0128E4D1094A019BEB
:10CB40009B1A48BF03F2FF13B3F5805F4FEA6322DD
:10CB500003D3FFF707FB4FF0FF32E276C2E700BFD7
:10CB6000784D0020904D00202DE9F0414FF0FF312D
:10CB7000304A314C0D460023107804280ED103F5BD
:10CB8000817004EB0010C079C60707D4681C52F806
:10CB90000A0C01D0884201D201461D460133082B00
:10CBA00002F11002E8D1002D41DB234CDFF8988020
:10CBB00005F5817704EB07132E01998841B1D8F868
:10CBC00034392BB1A01941F218029B68805898475C
:10CBD00041F218032644F058D8F834396BB1174E97
:10CBE000D3F80C80164A002306EB4521C04720B13C
:10CBF000022810D00020BDE8F081124BD3F89C2011
:10CC000004EB0714013AC3F89C200322A27101220D
:10CC100083F8A020EEE706F6E87604EB0714D6F8D2
:10CC20009C30013BC6F89C300123A371E2E7012050
:10CC3000E1E700BF9E5D0020784D0020904D002070
:10CC4000E5980008785D00204019002070B5124D6D
:10CC5000124BC5F8BC3840F20112002385F80C389D
:10CC6000A0F84421C0F85C3105F6BC020D23C0E9F0
:10CC70005422044685F8C818C0F8583100F5A2714E
:10CC800052F0F1FE05F2D47220461F23BDE8704039
:10CC9000012152F081BF00BF382A00205553425372
:10CCA00070B50B7813F06002044638D0202A1ED1EC
:10CCB0004A78FE2A05D0FF2A1DD052F0D3FD02206B
:10CCC00016E04A88AAB9CE88012E12D11A0610D5CC
:10CCD000314DD5F818389B699847C0B285F8CC0813
:10CCE00038B1324605F6CC01204652F091FE0020C4
:10CCF00070BD2046E1E74A88002AFAD1C988002998
:10CD0000F7D11B06F5D4244A82F80C18012182F8C9
:10CD1000D1171F2302F2D47252F03EFFE7E74B789F
:10CD20000A2B24D00B2B25D0012BE0D191F90460E4
:10CD30000D79C068002E22DA05F07F0153F086F9E4
:10CD40002946204652F09CFD2946134D02234022DD
:10CD5000204652F0BFFD95F8D137022B12D1812128
:10CD6000204652F04DFD002385F8D137BFE70B492F
:10CD70000122BAE7084B4A8883F8CD28B7E753F079
:10CD80004FF9DDE7002EB2DA012BB0D001212046A9
:10CD9000FFF75CFFABE700BF382A00200533002017
:10CDA00010B50B4A92F80C38022B044607D0033B0F
:10CDB000012B02D80021FFF749FF002010BD92F897
:10CDC000E11752F007FF0028F7DA01212046F2E7C9
:10CDD000382A002070B5314C94F80C6805461EB115
:10CDE000012E50D0002070BDD4F8D837C4F8C03818
:10CDF000D4F8DC37C4F8C438B0F8B4331F2B0DD1E5
:10CE0000D4F8D427264B9A4208D194F8E117012987
:10CE100004D894F8E237013B0F2B0AD920210520D2
:10CE200052F064FB022384F8D1372846FCF770F8EF
:10CE3000D8E752F0CFFE0028F7DB94F80C38013B1E
:10CE4000022BCFD9B4F8CE1821B3D4F8DC3784F84C
:10CE5000C868994228BF1946D4F8C4385B1AC4F888
:10CE6000C438042384F80C3840F20113A5F8443187
:10CE70000C4BC5E95616C5E9543305F5A271284691
:10CE800052F0F1FDAEE794F8E11752F0A3FE00284E
:10CE9000A8DA31462846FFF7D9FEA3E7382A002052
:10CEA00055534243763D0020F0B59C0827010E46BD
:10CEB000154600EB0414A04206F1100605F110051A
:10CEC00008D103F0030339443A4404EB83039C4242
:10CED00023D1F0BD84469CED006A16ED045AD0EDD6
:10CEE000016A56ED037A90ED027A56ED025A26EE6B
:10CEF000056A66EEA76AD0ED037A05ED046A16EDC1
:10CF0000016A45ED036A27EE257A67EE867A1030CE
:10CF100005ED027A45ED017ACDE7F4EC017AB1EC4A
:10CF2000017A67EE877AE2EC017AD0E74A090123B9
:10CF300050F8222001F01F018B40134214BF012042
:10CF40000020704710B54C09012250F8243001F040
:10CF50001F018A40134340F8243010BD80EA0120AD
:10CF6000082241F2210103B2002BB5BF81EA43033D
:10CF7000400098B280B2013AF5D1704738B50C46FE
:10CF80008D18AC4200D138BD14F8011BFFF7E6FF45
:10CF9000F7E74840082243B2002BBBBF5B0083F099
:10CFA000D5034000D8B2A8BFC0B2013AF3D1704750
:10CFB00038B50C468D18AC4200D138BD14F8011BB1
:10CFC000FFF7E7FFF7E770B5066805460C46002057
:10CFD000B44203D3731C2B60307070BD14F8011B76
:10CFE000FFF7D7FFF4E7DFED0A7AC0ED020A20EE83
:10CFF000270AB7EE007AC7EE007A00230360C0ED7F
:10D00000017A70EEA77A80EEA77A80ED037A7047F6
:10D01000DB0FC94090ED017AD0ED007AC0ED020A35
:10D0200030EE877AC0EE876A30EE677AE6EE877A6E
:10D03000B0EE670AC0ED007A704701230370002349
:10D04000C3648364036503644364436583628365E7
:10D050007047DFED157A80ED010AF4EEE70AF1EE94
:10D0600010FAC0ED020A80ED031AC0ED051A18DDB2
:10D07000B4EEE70AF1EE10FA08DC9FED0C7A80EDD1
:10D08000047A80ED0F2AC0ED0E2AD6E781EE007AF1
:10D09000C0EE207AF0EE006A77EE877A86EEA77A05
:10D0A000EDE700238360E8E7BD3786350000000028
:10D0B0000F29A8BF0F21012970B5B8BF01214C006D
:10D0C000013400260460A4000546816046602246C3
:10D0D0003146803057F0EEF82246314605F5807033
:10D0E000BDE8704057F0E6B8FDEEC07A17EE903A12
:10D0F0002033402B43D8DFED237A9FED237AB4EE23
:10D10000E70AF1EE10FA28DCDFED207A9FED1E7AB7
:10D11000B4EEE70AF1EE10FA22D4DFED1D7AB4EE98
:10D12000E70AF1EE10FA1EDD30EE670A37EEC00AAC
:10D1300060EE007ADFED176A9FED177AA7EEA67A08
:10D14000DFED166AE7EE876A9FED157AA7EEA67AFD
:10D1500020EE276AA6EE070A704730EE470ACEE7B0
:10D1600030EE070AD4E79FED0F7AB4EEC70AF1EE6E
:10D1700010FA44BF30EE270A37EE400AD8E79FED99
:10D180000A0A7047DB0F4940DB0FC940DB0F49C07B
:10D19000DB0FC93F9A7C2E36FAAF4FB93587083C72
:10D1A000A4AA2ABEDB0FC9BF00000000DFED027A8F
:10D1B00030EE270A98E700BFDB0FC93F10B51C46C9
:10D1C000334BB3FBF2F399429FED325AF0EE404AF3
:10D1D000F7EE005A53D207EE901A9FED2F7ADFED4B
:10D1E0002F6AF8EE677AF8EE002A67EE877A07EE84
:10D1F000102AB8EE477A27EE267AC5EE876A87EEC0
:10D20000A64AB0EE440AFFF76FFFF0EE403AB0EEE8
:10D21000440AFFF7CBFF74EEA44A012C83EEA43A34
:10D220001CBF35EEC04AF6EE006A33EE257A12BF17
:10D2300064EE266AF0EE656A20EE224A86EE876A80
:10D24000C4EE074A60EE227A75EEC35AC7EE876ACB
:10D25000C5EE877AF0EE465AC0ED005AC0ED014A9D
:10D2600080ED026AC0ED036AC0ED047A80ED065AD3
:10D2700080ED055A80ED085A80ED075A10BDF0EE9A
:10D28000454AB0EE456AF0EE456AF0EE457AE3E7CE
:10D2900020A1070000000000DB0FC940BD37863524
:10D2A0009FED010A002389E7F304353FB0EEE06A01
:10D2B000F0EEC07AB4EEE76AF1EE10FAF0EE406AF2
:10D2C0004BDCB5EE400AF1EE10FA4BD0B4EEE76A53
:10D2D000F1EE10FAF0EE675A41D5B0EE465A85EEFF
:10D2E000257ADFED225A9FED225ADFED224AA7EE82
:10D2F000255ADFED215AE5EE075A9FED205AA5EE9B
:10D30000875ADFED1F5AE5EE075A9FED1E5AE7EEEA
:10D31000054AB7EE005AA4EE875AB1EE657A87EE59
:10D32000050AB4EEE76AF1EE10FA48BFDFED167AAF
:10D33000F5EEC00A48BF37EEC00AF1EE10FA48BF5A
:10D34000DFED127AF5EEC06A48BF37EEC00AF1EEA3
:10D3500010FA48BFB1EE400A7047F0EE465AB0EE00
:10D36000675ABCE79FED0A7ABBE700BF39094E3D1B
:10D37000E3B59EBE69A2163E88FA16BE45FE7FBF83
:10D38000A7DFA8B499FB243FDB0FC93FDB0F49405F
:10D390000000000044F25063984203DDA0F50C4009
:10D3A000A0387047034B9842BCBF00F50C40A0303A
:10D3B000704700BFB0B9FFFF48F69F43984203DDB6
:10D3C000A0F50C40A03870470028BCBF00F50C4009
:10D3D000A030704791ED005A08B5B0EE450AFFF74E
:10D3E000E5FEF0EE405AB0EE450AFFF77DFE91ED06
:10D3F000015AF0EE404AB0EE450AFFF7D7FEF0EED4
:10D40000403AB0EE450AFFF76FFE91ED023AB0EEFA
:10D41000405AB0EE430AFFF7C9FEB0EE404AB0EE04
:10D42000430AFFF761FE25EE806A63EEC07A24EEC0
:10D43000847AC0ED017AF0EE467AE5EE077A25EEC1
:10D44000843A64EE806AC0ED037AF0EE437AE5EE4A
:10D45000667AA5EE067AE5EE436A23EE844A64EE28
:10D46000E34A65EEA35A80ED004A80ED025AC0ED12
:10D47000047AC0ED054AC0ED066A80ED077AC0ED7A
:10D48000085A08BD034600F1400100221A615A61A2
:10D490009A61DA6110338B42F8D11022002156F0E4
:10D4A00009BF91ED007AD0ED047AE7EE077AC0ED7E
:10D4B000047AD1ED006A91ED017AD0ED057AE6EEBD
:10D4C000877AC0ED057AD1ED006A91ED027AD0ED50
:10D4D000067AE6EE877AC0ED067A91ED007AD0ED15
:10D4E000077A77EE877AC0ED077AD1ED016A91ED80
:10D4F000007AD0ED087AE6EE877AC0ED087A91EDF1
:10D50000017AD0ED097AE7EE077AC0ED097AD1ED1C
:10D51000016A91ED027AD0ED0A7AE6EE877AC0EDE3
:10D520000A7A91ED017AD0ED0B7A77EE877AC0ED29
:10D530000B7A91ED007AD1ED026AD0ED0C7AE6EE2D
:10D54000877AC0ED0C7AD1ED026A91ED017AD0EDC7
:10D550000D7AE6EE877AC0ED0D7A91ED027AD0ED84
:10D560000E7AE7EE077AC0ED0E7A91ED027AD0EDF1
:10D570000F7A77EE877AC0ED0F7A91ED007AD0EDD1
:10D58000107A77EE877AC0ED107A91ED017AD0EDBE
:10D59000117A77EE877AC0ED117A91ED027AD0EDAB
:10D5A000127A77EE877AB7EE007AC0ED127AD0ED74
:10D5B000137A77EE877AC0ED137AD1ED017AD1ED47
:10D5C000006A91ED027A67EEA77AE6EEA67AE7EEB8
:10D5D000077A90ED007AA6EEA77A80ED007AD1ED79
:10D5E000016A90ED017AA6EEA77A80ED017AD1ED7D
:10D5F000026A90ED027AA6EEA77A80ED027A90EDAB
:10D60000037A77EE277AC0ED037A70472DE9F0436D
:10D61000034685B000F11007054600261C46AC46BF
:10D6200012E0F8EC016A1EED047AD4ED007AE6EE21
:10D63000C77AC4ED007A98450EF1100EF1D104348A
:10D64000BC420CF1040C03D0A7F11008E646F2E747
:10D6500001361C46B646BEF1040F1DD000EB0E1C71
:10D66000A84604F1100907E0FCEC016A18ED047A01
:10D67000E6EEC77AC4ED047ACC45D4ED047A08F11D
:10D680001008F1D1D3ED006A87EEA67A0EF1010EF3
:10D6900084ED047A6446DEE7042E03F1140305F1F9
:10D6A000040507F11007B9D10023009301930293F9
:10D6B00003936C4600231427F2EC017A00EB031568
:10D6C00007FB030C6E466545C4ED007A1FD101339C
:10D6D000042B04F10404EFD104AD103100F1400239
:10D6E00075ED017A00EB03170E461446BC4241ED7E
:10D6F000017A13D152ED016A87EEA67A013BA2F1BD
:10D70000140221ED017AEBD105B0BDE8F083F5EC10
:10D71000016AB6EC017AE6EEC77AD4E7F4EC016A66
:10D72000B6EC017AE6EEC77AE0E71FB50C46024692
:10D7300069461030FFF76AFFDDED007AB6EE007A39
:10D7400067EE877A0120C4ED007ADDED017A67EE9D
:10D75000877AC4ED017ADDED027A67EE877AC4ED4F
:10D76000027A04B010BDB5EEC00AF1EE10FA08B5A9
:10D7700006DB54F013FCB4EE400AF1EE10FA01D7C8
:10D780009FED010A08BD00BF000000002DE9F04137
:10D79000044626461C3004F1640250ED017AB1ECD7
:10D7A000010A77EE807A40ED017AFBF7FAF818303B
:10D7B0009042F2D12C4F626857F8343C25699B1A8D
:10D7C000A2680135934225612BD904F13008F36A30
:10D7D000012BC3BF03F1FF3307EE903A96ED0A7AAF
:10D7E0009FED220AC4BFF8EEE77A87EE270AFFF71B
:10D7F000BAFF4645D4ED057A15D0F4EEC07AF1EEC5
:10D8000010FA06F11806E2D5237B4BBB57F8342CEF
:10D81000626000222361A261E36222636364A26406
:10D82000E365BDE8F081F4EEC07AF1EE10FAEBD4D6
:10D8300007EE905AD4ED066AF8EE677A022386EE78
:10D84000A77AD4ED0C6A84ED067A86EEA77AD4ED39
:10D85000126A84ED0C7A86EEA77A84ED127A00E0E3
:10D8600003232370DDE700BF382A002000000000FA
:10D8700070B52DED028B0378012B04463CD1056970
:10D88000254E25B9426812B956F8342C426094ED01
:10D89000068A30EE088A013584ED068A256104F196
:10D8A0001C00FBF77EF8626856F8343C9B1AA268AD
:10D8B000934221D9E36A012BC3BF03F1FF3307EE83
:10D8C000903A94ED0A7A9FED150AC4BFF8EEE77A14
:10D8D00087EE270AFFF747FFD4ED057AF4EEC07A0A
:10D8E000F1EE10FA0ED5237B4BB956F8342C62605A
:10D8F00000222361A261E362BDEC028B70BD0323B1
:10D900002370F9E707EE905AF8EE677A022388EE63
:10D91000277A84ED067AF3E7382A00200000000019
:10D9200008B52DED028BF0EEC08AB0EE408AB7EE5E
:10D93000000A30EE680AFFF716FF9FED0E7ADFED62
:10D940000E7AE8EE877A9FED0D7AA7EEA87ADFEDE2
:10D950000C7AE7EE287AB5EEC08ABDEC028BF1EEC8
:10D9600010FA20EE270A44BFDFED067A37EEC00A30
:10D9700008BD00BF306E99BC2716983D843459BE4F
:10D98000A40DC93FDB0F494060EEA00AE0EE000A9B
:10D99000B0EE600AE7E660EEA00AE0EE000AE1EE13
:10D9A000010AB0EE600ADEE62DE9F74F90469DF8D9
:10D9B0003020002A0CBF4FF0200A4FF0300A0D9A99
:10D9C0001C1E05460F46BABF64424FF0010B4FF0D4
:10D9D000000B12F8011B01B14CB9BBF1000F2DD1A6
:10D9E000264636B9A1464FF0FF340D9E0FE0013CAC
:10D9F000EFE7BD4202D251462846C047013EF0E75C
:10DA0000BD4203D201922846C047019A16463246CB
:10DA100012F8011B0029F3D10D9BA9EB03094E4419
:10DA2000BBF1000F06D0A146B9F1000F09DC002CB4
:10DA3000A8BF3619304603B0BDE8F08F4FF000099B
:10DA4000D3E7BD4202D251462846C04709F1FF390B
:10DA5000EAE70FB437B50C4D06ABD5F8D41853F838
:10DA6000042BD5F8D008019352F034FD0446D5F8C4
:10DA70001C0803F0E3FE0028F9D0204603B0BDE8FF
:10DA8000304004B0704700BF382A00200EB403B500
:10DA900003AB084953F8042BCDE9003001A852F03C
:10DAA00019FD019B00221A7002B05DF804EB03B06F
:10DAB000704700BFF58900080CB430B52D4CD4F880
:10DAC000D838A5B01BB9D4F8DC38002B3FD094F877
:10DAD000E038994206D9012303FA00F0D4F8E4387B
:10DAE000184234D054F8341C4FF47A7304A8B1FBB4
:10DAF000F3F203FB12132049FFF7C8FF04AB034402
:10DB0000289A1E490393054629AB03A8029352F0B5
:10DB1000E1FC039B591C03910A211970039B591CBA
:10DB20000391002119700246D4F8D808A0B1036807
:10DB30005B6A4BB9D4F8D85804AC14F8011B31B166
:10DB4000284603F051FEF8E798470028F2D125B0A7
:10DB5000BDE8304002B07047D4F8DC38002BF6D076
:10DB600015440222009204A9AA18FD2029F00AFFF8
:10DB7000EDE700BF382A002027EC0608A58700083B
:10DB8000174A38B5D2F8E858033005EB9003B3F5DF
:10DB9000007F19D802F6EC04C2F8E838114A02EB0B
:10DBA000810120F0030051F80C2CC3F500730244EE
:10DBB00041F80C2C9B000C4A0421002004EB850446
:10DBC000FFF77AFF204638BD0021084A0846FFF7D4
:10DBD00073FF074A136843F0007313600024F1E7F2
:10DBE000382A0020303B002033EC060857EC0608AA
:10DBF000E06E01202DE9F0470368214F054600241F
:10DC000057F83420934213D11E4E06EB84094FEA95
:10DC10008408D9F820A8BAF1000F21D10721642087
:10DC2000FFF7AEFF0146C9F8200860B9164A04E0C4
:10DC300001340E2CE4D1154A00210520FFF73CFFEA
:10DC40000020BDE8F0876422514656F033FBD9F836
:10DC5000203807EBC407C3E90073DB615B63DB6457
:10DC600046446879D6F82038182404FB0032002195
:10DC70001046C2E90311956011750430E1E700BF59
:10DC800034470608382A00208AEC060865EC0608A6
:10DC900003685A1C026019700368090A5A1C026062
:10DCA0001970704703685A1C0260197003685A1C87
:10DCB00002600A0A1A7003685A1C02600A0C1A7081
:10DCC0000368090E5A1C02601970704738B5044683
:10DCD0000068154656F0AAFA23682B44236038BD25
:10DCE00003685A1C02601878704703685A1C026067
:10DCF0001A4612F8021B0260587841EA0020704769
:10DD0000026810B5531C0360134613F8021B03602E
:10DD1000D31C5478036093781B0443EA04230B4319
:10DD2000111D0160D07843EA006010BDD1E90032D6
:10DD30009A4206D05A1C0A6008B11B780370012071
:10DD4000704700207047D1E900239B1A012B10B5C2
:10DD50000446084604DDFFF7C8FF2080012010BDFF
:10DD60000020FCE7A0F16103192B98BF2038704711
:10DD700038B505460024284652F0ACFDA04200D834
:10DD800038BD2B5DA3F16102192A9CBF203B2B55A6
:10DD90000134F0E730B50A440546914201D1002034
:10DDA00011E015F8013B11F8014BA3F141001928CE
:10DDB000A4F1410098BF2033192898BF2034181BC4
:10DDC00001D1002CE9D130BD6FF00042E2E710B57F
:10DDD0000388827803F003010C24013A04FB01223A
:10DDE0001149847901EB4202A3F5FA63B2F8F220FB
:10DDF00040F2B5519B0801FB0323C278013A13445A
:10DE00000279182101FB0323427900893C2101FB9F
:10DE10000322064B234401FB02334FF47A720021A4
:10DE2000C3FB020110BD00BFC846060880436D3821
:10DE3000F8B519460446002310464FF47A7253F0A1
:10DE400005FB244B3C25034493FBF5F005FB103305
:10DE500090FBF5F105FB110060711820A37191FB97
:10DE6000F0F300FB131140F2B550217193FBF0F178
:10DE700000FB1133B3F5896F4FEA810526DA40F2D2
:10DE8000DA218B4224DCB3F5B77FB4BF0020012038
:10DE9000114E182101FB00660B2136F811709F42CC
:10DEA00001DD0139F9D105F5FA65054425804D1CE0
:10DEB000A5700C2505FB00110848228100EB4101EB
:10DEC0000133B1F8F2105B1AE370F8BD0320DFE70D
:10DED0000220DDE780BC92C7BA470608C84606089C
:10DEE000F0B5294D07460E460FCD8DB06C460FC4D8
:10DEF0000FCD0FC495E80F0084E80F0017F003035F
:10DF00003FD1642197FBF1F201FB127242B94FF449
:10DF1000C87297FBF2F302FB1373003B18BF012397
:10DF20007A1EC3F11D03002A019340F26D131146BE
:10DF300007FB03F3B8BFB91C03EBA1036FF0630148
:10DF400092FBF1F10B444FF4C87192FBF1F21344D0
:10DF50002533072493FBF4F2C2EBC2029B1A013E65
:10DF60006D46002155F8040F01310344B14293FB83
:10DF7000F4F2C2EBC202A3EB0203F3D1C01A0DB05C
:10DF8000F0BD0123CCE700BF1C480608084BD3E9CD
:10DF9000201251EA020309D0064B53F8343C5B18B7
:10DFA00042F10002C0E900320120704700207047B2
:10DFB000303B0020382A002037B505466846FFF779
:10DFC000E5FF044638B1DDE900232846FFF730FFBE
:10DFD000204603B030BD40F2011328806B80A8803A
:10DFE000A8712881F4E737B50546FFF7E5FF044639
:10DFF00050B1074B0DF10602B3F88830ADF806308A
:10E00000294628464EF0EEFB204603B030BD00BF47
:10E01000303B00202DE9F041044686B094F83030C2
:10E02000042B13D8DFE813F0150005005D00E900AC
:10E030003601DFF8688204F11C0701AA3946404620
:10E04000FEF727FD01280CD002282AD006B0BDE833
:10E05000F08192484EF044FE4FF6FF732384012373
:10E060003CE0019D0DB12B7863B98C48FDF78AFF28
:10E07000237EDD0618D54EF033FE4FF6FF73238462
:10E0800002232BE0EE7A3007D7D40B2204F13101C2
:10E09000284656F053F90028CFD1637E7340D90645
:10E0A00004D57E48FDF76EFF042317E0AA8A6B8B28
:10E0B00043EA02437A4A6362D2F81022EB69A36012
:10E0C0005202B3FBF2F102FB113109B113445B1AA6
:10E0D0007248E3606676FDF755FF032384F830301D
:10E0E0009CE76F4E96F8E031002BAFD104F11C088D
:10E0F00006F5DC7701AA41463846FEF7CAFC01283E
:10E1000059D1019D002D38D02B78E52B01D0002B63
:10E11000F0D1644BEB1A48BF03F2FF13B3F5805FF5
:10E120004FEA632003D3FEF71DF84FF0FF305E493E
:10E1300001EB0010FAF718FA01F5D070FDF722FF95
:10E1400020220021284656F0B5F8D4F831302B6053
:10E15000D4F835306B60B4F839302B8194F83B300B
:10E16000AB72637EEB7203A8FFF73DFF38BB6FF025
:10E170007E032B7447236B743AE096F8B831022B78
:10E1800092D096F8E031002B8ED10922C6E97D337A
:10E1900086F8E02186F8F031D6F8CC2186F8EC310B
:10E1A0003E48D6F81432C6F8E421C6F8E831FEF746
:10E1B00085FA01289ED002283FF476AF46E79DF805
:10E1C0000E209DF80F3043EA4213BDF80C20A2F256
:10E1D000BC7243EA42232B829DF811309DF8122035
:10E1E0005B0143EA52039DF8102043EAC223EB810E
:10E1F0002B8A2B83EB89EB826FE7237E9A0608D567
:10E20000E0690023112202A9FDF7BAFF01287FF47B
:10E210001DAF20464EF064FD2269237E9AB91B078C
:10E2200008D51F4B93F89821002A7FF40FAF0722DF
:10E2300083F89821002384F82830E36A204606B04A
:10E24000BDE8F041184703F0F70213F0040322760B
:10E250000AD0E26AA1680023204684F8283006B07C
:10E26000BDE8F041FDF732BF122AE3D1E26AA263B2
:10E27000626A84F83C3004212046C4E90B22C4E9D8
:10E28000023384F828106363636206B0BDE8F0418E
:10E290004EF026BD0020E36A2070D0E7305F0020FA
:10E2A000785D0020904D0020905D00202DE9F34125
:10E2B00003780446002B76D090F82830013B082BD9
:10E2C00071D8DFE803F00509475B4C6170666B00AD
:10E2D00002B0BDE8F0419DE6344B4568D3F81072BA
:10E2E000D3F818327F021D40216B2046FDF784FED3
:10E2F00005EB01084745064626D880B1D4E901322E
:10E300009A422CBFA260A360002384F82830E36AFD
:10E31000002B48D0204602B0BDE8F04118472169E3
:10E32000207E01AA51F042FA01283CD123696361A1
:10E33000019B236163683B445B1B6360236BDB1BB6
:10E340002B4423633546CFE70028D7D163680B44BD
:10E350006360D3E702B0BDE8F041FEF72FBB0121B7
:10E36000FEF79EFA01281ED1216C0023204684F876
:10E37000283002B0BDE8F041FEF774BB002102B0C6
:10E38000BDE8F041FEF78CBA02B0BDE8F041FEF7FF
:10E3900027BA02B0BDE8F041FEF72BB902B0BDE8E4
:10E3A000F041FEF78BB902B0BDE8F081785D002046
:10E3B000F0B50124B0FBF4F58D4203D200261CB960
:10E3C0001C70F0BD4C43F5E7B0FBF4F5B4FBF1F77E
:10E3D00004FB15002EB9002D03DC8C420CD33C4607
:10E3E000EDE7092D08DD002A0CBF572437242C4403
:10E3F00003F8014B0136F2E73024F8E700280B461A
:10E40000BEBF2D2203F8012B404200220A21CFE794
:10E4100003463038C2B2092A0FD9A3F16102052A96
:10E4200002D8A3F157007047A3F14102052A02D890
:10E43000A3F1370070474FF0FF30704770B50446C6
:10E44000944208461546B4FBF2F602D33046FFF775
:10E45000F5FF05FB1644024B1B5D00F8013B70BD48
:10E46000AFEC0608B5EEC00ADFED2D7AF1EE10FA3A
:10E47000CCBF30EE270A30EE670ADFED2A7A20EEB5
:10E48000270A30B5FDEEC07A87B017EE904A0546F0
:10E4900084EAE470002303A9A0EBE470CDE9003323
:10E4A00002934EF00DFC002CB4BF2D23202303A8B3
:10E4B0008DF8003052F00EFA012822D130238DF869
:10E4C000013043F23003ADF8023003A9684655F03D
:10E4D000F9FE684652F0FEF9C41EE4B222466946CF
:10E4E000284655F0A3FE00232B550F49284655F02A
:10E4F000E9FE0DEB0401284655F0E4FE284607B07E
:10E5000030BD022805D130238DF801308DF802305E
:10E51000DBE7032804BF30238DF80130D5E700BFC7
:10E520006F12033A00007A44E325070830B50278F9
:10E53000202A034600F10100F9D0092AF7D02D2A3C
:10E540004BD10346BFEE000A9FED3C7A1A46F2EE2D
:10E55000046A134612F8010BA0F13001CCB2092C69
:10E5600041D92E280BD1F2EE046A1146B0EE666A4C
:10E570000B4611F8012B303AD0B209283CD91A7851
:10E5800002F0DF02452A53D15A782D2A3FD10233B7
:10E590000120013B00220A2513F8011F3039CCB2BB
:10E5A000092C3AD9B2F59A7F1346DFED256A28BFC8
:10E5B0004FF49A731A46F7EE007A072A30D8DA0831
:10E5C0006FF0070101FB0233F2EE046A63BB88B30C
:10E5D000C7EE276A20EE260A30BD2B2A08BF034665
:10E5E000B7EE000AB0E707EE901AF8EEE77AE7EE2A
:10E5F000267AB0EE677AACE707EE902AF8EEE77A73
:10E60000C7EEA65A66EE866A37EE257AB0E72B2A61
:10E6100014BF013302330020BBE705FB0212BBE746
:10E6200067EEA67A083AC8E767EEA67A013BCDE71F
:10E63000F7EE007A67EE276ACCE700BF0000000023
:10E6400020BCBE4C70B5034610F8012B202AFAD02E
:10E65000092AF8D02D2A0ABF034601254FF0FF35BD
:10E66000591E00240A2611F8010FFFF7D1FE0928D0
:10E6700002D905FB04F070BD06FB0404F3E710B5F6
:10E680000023802804D893420AD2C854581C10BDD5
:10E69000934205D060F07F04CC54C0090133F0E709
:10E6A0004FF0FF30F3E7F8B5144D2B787E2B23D1D4
:10E6B000012229460020FEF761FC114F6C1C2288C4
:10E6C00062B1A31DBB4217D2A618BE4214D2052ABE
:10E6D00012D92146FEF752FC3446F0E702222146C9
:10E6E000FEF74CFC6388074AC31A0434641B584283
:10E6F000A2F822425841F8BD0020FCE70040000883
:10E7000000800008303B00202DE9F04F01208FB041
:10E7100002F0D8FCDFF8E0B1724BA3EB0B02CDE9BD
:10E7200001234FF00308102200210AA855F0C2FD72
:10E73000019B0993029B08936B4BCDF81CB01A699F
:10E74000002ABFBF694A5A6002F188325A60012428
:10E75000F322DA604FF000097E23224604A907A8BD
:10E760008DF83440CDF830908DF81030FAF7F4F988
:10E770004845C0F2A180224604A94846FEF7FEFBA8
:10E780005B4CADF812005B4B9C423CD30024022250
:10E7900005A907A8ADF81440FAF7DEF9A042C0F2C7
:10E7A0008B80BDF81200022205A9FEF7E7FB0222CA
:10E7B000ADF812000DF1120107A8FAF7CDF9A04249
:10E7C0007ADB0B9880B1079B089A0344934273D875
:10E7D0000AABC0F104022146184455F06BFD0AA9AA
:10E7E00007A8FAF715F90C900C9C002C64DB9DF837
:10E7F000343023B13C4A136943F000431361B4FA47
:10E8000084F4640959E062888DF81990C2F30B060C
:10E81000B31DADF814302388C3F30B011B0B8DF827
:10E8200018301304ADF816101ED4062205A907A847
:10E83000FAF792F900283FDBBDF81200062205A97D
:10E84000FEF79CFB676805463246394607A8FAF78B
:10E8500083F9002830DB324639462846FEF78EFB26
:10E86000ADF8120014348EE700273D460135EDB2B5
:10E87000062205A907A88DF81950FAF76DF90028A6
:10E880001ADBBDF81200062205A9FEF777FB6168C6
:10E8900082463944324607A80391FAF75DF9002809
:10E8A0000ADB039932465046FEF768FB032DADF8AC
:10E8B00012003744DAD1D5E70024B8F1010802D0BC
:10E8C000002C3FF430AF002002F0FCFB14B905200F
:10E8D00005F052FBFFF7E7FE0028F8D00FB0BDE8C7
:10E8E000F08F00BF00800008003C02402301674514
:10E8F000C45107081457070800400008034AD2F81B
:10E90000243223EA0003C2F824327047303B00204F
:10E91000034606490648884201D300207047028812
:10E92000C2F30B029342F9D01430F4E714570708EE
:10E93000C451070870B544880B460546C4F30B0460
:10E9400022460021184655F0B5FC2969084A914233
:10E95000034607D3074A914205D22246BDE87040DC
:10E9600055F064BC19B1BDE870401846084770BD49
:10E97000145707082B5C070810B4B0F9024042880E
:10E98000002C0B4641685DF8044BBEBFC2F30B027E
:10E99000DBB203FB0211CDE730B5094B094CA342B2
:10E9A00000D330BDB3F902205988002A06DA5A682C
:10E9B000DD68C1F30B0100FB01222A601433EEE78E
:10E9C000C45107081457070830B502460144002017
:10E9D00012F8015B082480EA050343F3000323F0E7
:10E9E000730383EA5003D8B2631E13F0FF044FEAA7
:10E9F0005505F0D19142EBD130BD2DE9F04F87B0F4
:10EA0000CDE903230025804601910095039B4046F4
:10EA1000EC0003EBC50AFBF7C3F8002800F0978071
:10EA2000002201214046FBF7A5F80290002800F0E3
:10EA30008E8098F804309A0706D4029A049B1046F8
:10EA40001D7007B0BDE8F08FF0214046FBF7B2F82B
:10EA500000287CD0039BA4F108024FF0000B012694
:10EA6000134434465F460593019BB3B3082C34D856
:10EA700004F1FF3943FA09F909F001094946404612
:10EA8000FBF74FF8002862D0002201214046FBF737
:10EA900071F8024600285AD098F8041001F0600C72
:10EAA000BCF1600F4FEAD11037D0019B1BB1082C8D
:10EAB00001D88145C1D120B31AF80710314376003F
:10EAC000013416F0FF060AF80710E4B2CCD1013782
:10EAD000FFB2082F21D00126C6E75DB1009BA342FB
:10EAE00008D9059BDA5D164214BF4FF001094FF0BB
:10EAF0000009C3E7009B1B1BD3F1000949EB030985
:10EB0000BCE7880940EA511111F0010F1AF807100B
:10EB100008BFA34621EA0601D1E7402C11D90721FD
:10EB200050460292FFF750FF9AF80740029A84423B
:10EB300007D10135EDB2BBF1000F3FF47FAFCDF847
:10EB400000B0049B1B78AB423FF660AF76E7002233
:10EB500074E700BF0000000090F83C20034602F07C
:10EB6000FF0012B1002283F83C2070474FF480531D
:10EB7000838170474FF40063838170474FF40063D3
:10EB8000838170474FF40063838170474FF40063C3
:10EB9000838170474FF40063838170474FF40063B3
:10EBA0008381704710B5064A0423002152F8044BB4
:10EBB000844208BF42F8041C013BF7D110BD00BFDE
:10EBC000A05F0020324BF0B5188ADC8BB3F92850D7
:10EBD000B3F92270B3F918E0B3F93060001B9C8BD5
:10EBE0006043B3F9264005EBE035E40294FBF5F40D
:10EBF00004EBE034A4F57A60B3F91650DC6200FB54
:10EC000000FC4FEA2C3C45430CFB07F700FB0EFED3
:10EC1000ED12B3F9200005EBE725B3F914700CFBF6
:10EC200000F0001405EB8705B3F81AC05B6B00EB2E
:10EC30006E30B54002300235A3EBA50580104CF2D2
:10EC4000503300F5004033416B430CFB00F04FEABA
:10EC5000D03055BF5B00B3FBF0F3B3FBF0F35B00C8
:10EC600071B1181240F6DE3540436843094D001477
:10EC70005D4300EB254000F6CF6003EB20130B60F3
:10EC800022B10A235C430834241114600120F0BD32
:10EC9000A05F002043E3FFFF012070470120704781
:10ECA0002DE9F74F604E9046B38FB26BB6F94CC06A
:10ECB000B6F94A70B6F948B0C3EB22155B00C3EB56
:10ECC000E203B6F93E206D435343B6F940202D13BD
:10ECD0005543AD1305EBE325B36D0093A5F5FA306D
:10ECE000B6F946307565894680FB001EDA1703FBCE
:10ECF0000EF401FB0244A3FB01321444B6F9442094
:10ED000082FB00A21B0A120343EA046342EA1A527E
:10ED10004FEA0A3A13EB0A0342EB2422B6F842A068
:10ED200002F500420192A3FB0A23019A0AFB023A70
:10ED30004FEAEA734FEA6A0253EA6A0A4FF00004A4
:10ED40005ED087FB00704FEAEC7A0CFB0EFE4004AD
:10ED500001FB0AEE40EAD730ACFB011C7F047F18B0
:10ED60000099F4444CEB0000C1F5801C0CF000410C
:10ED7000E71941EA5C014FEACC7CBCEB070C40F69A
:10ED8000354400EBCB0061EB0001ACFB040C04FB51
:10ED900001C152F05BFB84460746430BB6F95200B3
:10EDA0004A1343EAC14300FB02FEC41703FB04EE0F
:10EDB000A0FB03407044624303FB0022A4FB034317
:10EDC0001A44B6F95030640E44EAC2144FEAE37EA6
:10EDD00003FB01F0E4190EFB0C00A3FB0C373844D5
:10EDE0004FEAD34343EA403341EB6262E41842EB1B
:10EDF000E042B6F94E30240A44EA026404EB0314FC
:10EE0000B9F1000F02D0240AC9F80040B8F1000F90
:10EE100005D005EB850580352D12C8F8005001207E
:10EE200003B0BDE8F08F00BFA05F002031B10A4BF6
:10EE3000D3ED1E7AFDEEE77AC1ED007A52B1064BB2
:10EE40009FED067AD3ED1F7A67EE877AFDEEE77ABB
:10EE5000C2ED007A01207047A05F00200000C84288
:10EE60002DE9F74FCDE90012574AB2F88E30D2F8AB
:10EE70008010B2F88A60B2F890701B02C91AB2F81A
:10EE80008C306EEB0E0EA3FB010403FB0E44B2F8B4
:10EE90008830C00940EA44601B04C018A6FB013555
:10EEA00006FB0E55B2F886604FEA132343EA05636A
:10EEB0004FEAC6364FEAE41444F100049B19A7FB5D
:10EEC000012607FB0E664FEAD25242EA46224FEA7B
:10EED000252545F10005F61512F5FA6C46F1000BF3
:10EEE000BCF5FA6F7BF1000750DA02FB06F8A2FBD3
:10EEF00002794FF0050A09EB4809A7FB0A780AFBDB
:10EF000009884FEA570949EAC879BF08B0EB0909EF
:10EF100047EA887764EB6804DF1B3B462B4F65EBC1
:10EF2000A805BC454FF0FF377BEB0707484622DAC0
:10EF300040F6AC57D21946F100065643A2FB0272C6
:10EF400002EB46024FEAC208FE00BE1B48EA5778B1
:10EF500062EB0808361844EB08044FF00B08304603
:10EF6000A7FB087608FB02627F0847EAC277DF1B2F
:10EF70003B4665EB620501FB0EFEA1FB011202EBB5
:10EF80004E02C90F41EA4201BCEB010C009A9AB152
:10EF90000D4AD2F89410A1FB033201FB05225B0D50
:10EFA00043EAC2231B1A4FEA625262EB0402DB0BF4
:10EFB00043EA4243009A1360019B0BB1C3F800C0BF
:10EFC000012003B0BDE8F08FA05F002024FAFFFF0E
:10EFD00001207047B0F900305943084B994208DBD3
:10EFE000B1F5000F07DA0029B8BFFF31081200B2EF
:10EFF00070470348FBE747F6FF70F8E701FF7FFF24
:10F000000080FFFF064B0022C3F89820C3F89C2025
:10F01000C3F8A0200022C3F8A4200120704700BF3D
:10F02000A05F0020104B1A68104BD3F8A410521A9E
:10F03000FA2A16D8D3ED267AFDEEE77A17EE902A53
:10F04000D3ED277AC286FDEEE77A17EE902AD3ED4C
:10F05000287A0287FDEEE77A17EE903A438701207F
:10F0600070470020704700BF042A0020A05F0020E6
:10F0700090F85F3230B53BB990F85D1290F85E328F
:10F080000124DAB2914200D830BDB0F8665204FAD9
:10F0900003F22A43A0F866220133F2E743790246DD
:10F0A00013F0010006D0D2E90731D2685B1A013AA9
:10F0B00003EA020070474379024613F0020007D0CA
:10F0C000936A516A1269013B5B1A013A03EA020032
:10F0D000704710B5437913F0010304460ED0FFF7D3
:10F0E000DDFF034650B1226A6369E1689B5C01322F
:10F0F000B2FBF1F001FB1022DBB22262184610BD18
:10F1000043799B070AD5436A8269D154436A0269ED
:10F110000133B3FBF2F102FB1133436270474171DB
:10F12000704781717047D0E90920131A584258413D
:10F130007047024BD3F8A8305B681847A05F0020E7
:10F14000024BD3F8A83008309B681847A05F002016
:10F15000012070470120704701207047012070474F
:10F160000120704731B10C4BD3ED2B7AF8EEE77AE2
:10F17000C1ED007A7AB1084BDFED086AD3F8B03000
:10F18000A3F5D543333B07EE903AF8EEE77A87EEE6
:10F19000A67A82ED007A7047A05F00200000C84286
:10F1A0000120704701207047094A30B505460A24FE
:10F1B00000201368AB4205D1D3688B421EBF431CAD
:10F1C000D160D8B2013C02F11402F2D130BD00BFCF
:10F1D000A00500207047054B40F2FF7203EBC0030F
:10F1E0009142A8BF11469980704700BF083C00209B
:10F1F000112807D8044B03EB8003D3F8B4300BB1CC
:10F200009B681960704700BFA05F002008B5FFF73A
:10F21000EFFFBDE8084022F021BB0C4A13787BB118
:10F220000B4B93F8FC1059B193F8FD1059B150688D
:10F230000021FA2883F8FD10A8BF4FF0FF30704777
:10F240006FF0010070476FF002007047F810002067
:10F25000A05F00200B4B93F8FE206AB193F8FF20CB
:10F260006AB1002283F8FF20074B9868B0F5967FBB
:10F27000A8BF4FF0FF3070476FF0010070476FF08C
:10F2800002007047A05F0020F8100020024BD3F866
:10F2900000315B68184700BFA05F0020024BD3F825
:10F2A00000319B68184700BFA05F0020024BD3F8D5
:10F2B0000031DB68184700BFA05F0020014BD86811
:10F2C000704700BFF8100020044B93F8043113B1CD
:10F2D000034B186970476FF001007047A05F002072
:10F2E000F8100020014B5869704700BFF81000204B
:10F2F0002DE9F041062592F9007086B06B43144663
:10F3000012F80580A0EB080EA0EB070CBEF1000F71
:10F31000B8BFCEF1000EBCF1000FB8BFCCF1000CAD
:10F32000E645B8BF541905F10605B8BF4FFA88F78E
:10F33000AB421646E4D11A4433786588BB420BD100
:10F3400073884D1BCB1A002DB8BF6D42002BB8BF80
:10F350005B429D42C8BF34460636B242ECD1637967
:10F36000049323790393638802932378054ACDE9B4
:10F370000013034603210120FEF79EFB204606B042
:10F38000BDE8F08168ED06084B1EDBB2062BF0B538
:10F3900098BF204A204D98BFD25CA5F1580400F1D7
:10F3A000FF3388BF4FF48072012B88BF2C46234661
:10F3B00087B033F8086B1D88C5B9012827D0174BD3
:10F3C000174D022818BF2B46A0790590A0880490FD
:10F3D000A078039020880091CDE901200321114AF3
:10F3E0000120FEF769FB204607B0F0BDA2EB050C3B
:10F3F000971BBCF1000FB8BFCCF1000C002FB8BFB9
:10F400007F42BC45BCBF1C462E460833D3E7064BA3
:10F41000DAE700BF884806086C110020A8ED06084E
:10F42000A6040708AFED0608A1ED060808B50068B8
:10F430004EF0D3FF024BC3F88000012008BD00BF8F
:10F44000A05F002008B500684EF0C7FF024BC3F86C
:10F450009400012008BD00BFA05F002038B514460D
:10F460000D46002943D0344B9FED347AD3ED427AD8
:10F47000B3F92421F8EEE77A06EE102AC7EE876A80
:10F48000B3F92021D3ED437AF8EEE77AB8EEC66AF5
:10F49000C7EE875A07EE102AD3ED457AB3F91C213F
:10F4A000B8EEC77AB8EEE70AA6EE867AD3ED467ACA
:10F4B000F8EEE77AE6EE877AA6EEA70A07EE902A3C
:10F4C000B3F92221B3F91E3106EE102A07EE103AE5
:10F4D000B8EEC66AB8EEC77AF8EEE77AA6EE867A94
:10F4E000E6EE877AA5EEA70A52F0F6FD28600CB387
:10F4F000114BDFED126A93ED437AB3F91021B3F9A2
:10F500001231B8EEC77A07EE902A87EE260A07EE88
:10F51000103AB8EEC77AF8EEE77A20EE070AB6EEB0
:10F52000007AA7EE870ADFED067A20EE270A52F06E
:10F53000D3FD2060012038BDA05F00200000F04A0C
:10F540000000C842094B10B553F8304007EE901A3E
:10F550005CB1F8EEE77A94ED047A94ED030AA7EE35
:10F56000870A52F0B9FDA368186010BD083C00205E
:10F5700010B50C4B0C4C1B68D4F828011B1AFA2B45
:10F5800006D904201CF03AFC002084F82C0110BDA0
:10F5900011B1D4F830310B6012B1D4F834311360AA
:10F5A0000120F4E7042A0020A05F00202DE9F041AB
:10F5B0000C4DDFF834802C686B6901271C400CB9B6
:10F5C000BDE8F081B4FA84F3C3F11F0307FA03F630
:10F5D00008EB830324EA0604D3F83801036898474C
:10F5E0006E61ECE7003C0140A05F0020F8B5836845
:10F5F0001C686379DB0724D5A57994F85C3205F0A3
:10F6000001073D46F3B1E06B43681A68D36AC3F360
:10F610004E03536294F86D32012B07D094F8613297
:10F6200023B1B4F868320133A4F8683285F00101DF
:10F630004DF0ACF90023A4F866324FF08073C4F8A3
:10F640005C32F8BD94F85F62012E04BF94F85D321D
:10F6500084F85E322046FFF70BFD4EB9012384F893
:10F660005F3287EA0301E06BBDE8F8404DF08EB9E8
:10F67000002384F85F323946F5E7F0B52DED028BB3
:10F6800083B00E46154649F0CBF8002869D024F027
:10F69000B1F9354B354C1B6803F00203002845D007
:10F6A000002B59D0324F0DF1060024F0B1F9D7F8F4
:10F6B0006425BDF806309FED2F7A9B1A07EE903A2D
:10F6C000F8EEE77AF0EE408A67EE877A9FED2A0A35
:10F6D00027EE800AFDF76AFD07F5AF6797ED008A10
:10F6E000A0EE688A42F08EF854ED2E0AD0ED057A2D
:10F6F000B0EE480A70EEA70AFEF746F97EB1DFEDDC
:10F700001F7A9FED1F7A20EE000A20EE270AC0EE36
:10F71000077A9FED1C7A77EE877AC6ED007A0DB1F5
:10F72000194B2B6003B0BDEC028BF0BDA3B134F9D3
:10F730009C3C01EE103A34F99E3C00EE903A34F9CC
:10F74000A03C00EE103AB8EEC11AF8EEE00AB8EEAE
:10F75000C00AFEF720F9D1E754F8843C93ED330A50
:10F76000CCE79FED0A0AC9E7886F01209870002056
:10F77000A05F00200AD7233C35FA8E3CCDCC9C3FBD
:10F7800000409C4682E6C5473313904300000000CA
:10F7900070B50446012026F0F5FA58B103684BB164
:10F7A0001C4A237992F83D10994231D092F83C20BE
:10F7B0009A422DD0184B5E68730612D5002127207F
:10F7C000FAF794FB002105462620FAF78FFB1DB1BE
:10F7D0002A6823689A421BD018B1026823689A42AB
:10F7E00016D0F5030CD521680C4B0A22186881420B
:10F7F00002D1D868C0010BD4013A03F11403F5D14A
:10F800002079112804D0A0F121035842584170BD3D
:10F810000120FCE754030020886F0120A005002090
:10F8200000684EF01EBB154B53F8200070B508B3AE
:10F83000134D0C2202FB005212F97F3C591C1AD0C6
:10F8400012F8770CB0B1E9188C2411F82C6C12F86E
:10F85000781C0020142263435C1805EB4404013A31
:10F8600034F8284C314410FA84F0F5D11423B0FB5D
:10F87000F3F080B270BD0020FCE700BFA05F002065
:10F880009870002038B503200D461446FFF7CBFFD3
:10F8900007EE900A8DB19FED0B7AF8EE677AF0EEE5
:10F8A000006A67EE877AB8EE047AA7EEA67ADFEDF3
:10F8B000067A67EE277AC5ED007A0CB1034B236018
:10F8C00038BD00BF6740533A00007A443313904379
:10F8D000C28970B5002302F00F0602F47F42C28194
:10F8E000012519464C1030F81440002C18BF002593
:10F8F00011F0010F1ABFE4B2634083EA1423082415
:10F9000013F4004F18BF83F4C053013C4FEA430384
:10F91000F6D101311029E5D13243C28135B9C3F3A3
:10F920000330801B18BF4FF0FF3070BD4FF0FF3029
:10F93000FBE710B5427A044632B10146406851F8FF
:10F940000A3B98470023637210BD10B4447A621CCE
:10F950000444D2B24272A172037A934202D85DF893
:10F96000044BE6E75DF8044B7047EEE710B503681B
:10F970001A79022A044602D1987A4EF01FFD00231C
:10F980002371236010BDF0B50C4B0D4E0446B342FD
:10F9900001D30020F0BD587988420DD11D79A542D0
:10F9A00000D04CB9D879904206D118680779AF4297
:10F9B00002D105689D42EDD00C33E8E7A0010008B4
:10F9C0006803000837B503460079022830D11B4A86
:10F9D00093F91030009214225343194C194AE358FA
:10F9E000934227D0A2F57842934225D002F5806257
:10F9F00093421DD101F108020DEB02011A8811F8A2
:10FA0000085C22F040021204120C14211A8001FB3F
:10FA100000441A88E16822F0380231F825101204F7
:10FA2000120C0A431A801A8892B242F040021A80DD
:10FA300003B030BD0020DDE70120DBE70001020359
:10FA4000B400002000300140C36910B5044623B95A
:10FA500009211420FEF794F8E061E06910BD10B5AB
:10FA600004460068FFF7F0FF8378DBB1B0F90A3095
:10FA700007EE903AF8EEE77AC4ED057AB0F90C306B
:10FA800007EE903AF8EEE77AF1EE677AC4ED047A81
:10FA9000B0F90E3007EE903AF8EEE77A0120C4EDA7
:10FAA000067A10BD1846FCE710B504460068FFF75B
:10FAB000CBFF8378CBB1B0F9043007EE903AF8EE83
:10FAC000E77AC4ED047AB0F9063007EE903AF8EE22
:10FAD000E77AC4ED057AB0F9083007EE903AF8EE0F
:10FAE000E77A0120C4ED067A10BD1846FCE710B590
:10FAF00004460068FFF7A8FF8378CBB18388DBBAA0
:10FB000007EE903AF8EEE77AC4ED047AC388DBBAE0
:10FB100007EE903AF8EEE77AC4ED057A0389DBBA8E
:10FB200007EE903AF8EEE77A0120C4ED067A10BDB0
:10FB30001846FCE710B500680C46FFF785FF034642
:10FB4000807840B15B892222DBBA93FBF2F303F2A7
:10FB50006D132380012010BD38B500680D46144692
:10FB6000FFF772FFD0F8013007EE103ACDB1D0F8B0
:10FB70000530DFED176A9FED176A07EE903AF8EE51
:10FB8000677A77EEE67A77EEA77AC7EE866AF7EEBF
:10FB9000007A76EEE77ADFED106A67EEE67AC5ED79
:10FBA000007A9CB1DFED0D7ADFED0D6AB8EEC77A11
:10FBB00027EE277AC7EE267A9FED0A7A77EEC77A84
:10FBC0009FED097A77EE877AC4ED007A38BD00BFE1
:10FBD0009AC9CC449AC94C460E76D7450000484392
:10FBE00000E0FF4400004842339388432DE9F04190
:10FBF00000680E461546FFF727FF8446C068DCF80C
:10FC0000103030F07F4060D0002B5ED0BCF8082070
:10FC1000BCF80A70D2019B1A61EB0101EEB3BCF88B
:10FC200004E0BCF806809FED2A7AAEFB03420EFB8F
:10FC30000122BCF800E0BCF802C0E40944EA4264D6
:10FC40004FEACE3E14EB0E044FEAE212A4FB004E44
:10FC500042F1000200FB02E2600D40EAC2205415AE
:10FC6000A8FB032E08FB01EE52094FEADC3842EAFA
:10FC7000CE624FEA4C4C12EB0C0248EB6E1C801A21
:10FC800064EB0C04C00B40EA444007EE900AF8EE27
:10FC9000E77A67EE877AC6ED007AB5B1A7FB033243
:10FCA00007FB01225B0D43EAC22313F5FA6307EE5B
:10FCB000903ADFED086AF8EEE77A87EEA67ADFED94
:10FCC000067A77EE277AC5ED007ABDE8F08100BFAD
:10FCD0007B81303F0000C8423393884337B50068CA
:10FCE0000D461446FFF7B0FED0F805309FED237A9D
:10FCF00007EE903AF8EE677AF2EE046A77EEC77A8A
:10FD00009FED1F7AD0F8013067EE877AB3EE097A5B
:10FD100067EE877A07EE103AF4EEE67AF1EE10FA23
:10FD200006DCFAEE046AF4EEE67AF1EE10FA0CD58F
:10FD300017EE900A50F03AFF124ACDE90001042173
:10FD40000320FDF7B9FE03B030BD2DB1DFED0E6A23
:10FD500067EEA67AC5ED007A002CF4D0B8EE477AAB
:10FD6000DFED0A6ADFED0A7AE7EE267A9FED097A7F
:10FD700077EE877AC4ED007AE5E700BF0000004621
:10FD800000008038F6ED06080AD778430319C83D0D
:10FD9000000048C2339388430379022B0DD190F9B8
:10FDA000103014225343064AD3581A89920746BF8B
:10FDB0001889C0F3C010012070470020704700BFB1
:10FDC000B40000200368DB6B13B504462BB923682D
:10FDD0005B6B3BB9FF23E38202E098470028F6D132
:10FDE00002B010BD214601A898470028F2D0BDF806
:10FDF0000630013B9BB2EEE7036810B59B680446F2
:10FE0000984701236374FF23A37410BD036810B5E2
:10FE100004461B689847236820469B689847E37C04
:10FE20000133E37410BD036810B504465B6898475E
:10FE3000236820469B689847E37C013BE37410BD30
:10FE40002DE9F3410446184616460D461F4650F06C
:10FE500041FD2368E67328440022A0730092D3F882
:10FE6000148032463B4629462046C04702B0BDE8D2
:10FE7000F08130B5046885B0E469089D34B10DB9EE
:10FE80000DF10F050095A04705B030BD2046FBE7FA
:10FE900003685B6A184703689B6A184710B5037BC1
:10FEA00004460BB1437B13B92046FFF7F4FF2368E8
:10FEB0002046DB68BDE81040184703685B6C03B15F
:10FEC0001847704738B504468B6801600D4698475F
:10FED0000B4B2361002323752B6B13B120469847EE
:10FEE0002075084B93F820331BB1237D23F00103C9
:10FEF00023750023E3822046BDE8384062E700BF57
:10FF00000001FF009870002003681B6803B11847C8
:10FF1000704703685B6803B11847704703681B6A42
:10FF200003B11847704703685B6A03B1184770470D
:10FF300030B40468029DA46A1CB10295A44630BC8A
:10FF4000604730BC704730B40468029DE46A1CB15D
:10FF50000295A44630BC604730BC704703685B6CB8
:10FF600003B11847704703689B6C03B1184770478B
:10FF700003689B6F03B1184770470368D3F880305C
:10FF800003B1184770470368D3F8843003B11847AA
:10FF900070470368D3F8883003B11847704721B120
:10FFA0000B68D3F88C3003B118470020704738B580
:10FFB000094C052303FB0044A13C0025013514F83E
:10FFC000010FEDB24EF07FF8052DF7D1BDE83840B6
:10FFD00000204EF078B800BF8F48060810B5441EC8
:10FFE00014F8010F00B910BDFFF7E1FFF8E7FFF7C4
:10FFF000DDBAFFF7DBBAFFF7D9BAFFF7D7BAFFF7D9
:020000040801F1
:10000000D5BAFFF7D3BA18B103689B6803B1184794
:10001000002070470C4B93F8212370B506460D461F
:100020008AB9D3F8244374B123681B685BB12046B6
:10003000FFF7E9FF38B123683246196820462B469E
:10004000BDE87040084770BD9870002001207047DF
:1000500018B103689B6803B11847002070470B4B29
:1000600070B5D3F8284306460D4674B123681B6863
:100070005BB12046FFF7ECFF38B1236832461968C0
:1000800020462B46BDE87040084770BD98700020A0
:10009000034620B1026812B1D26902B1104793ED54
:1000A000017A084BB8EEC77AD3EDCC6AF6EE007A47
:1000B000E7EE267AFDEEE77A17EE900A00F30B00E2
:1000C000704700BF98700020034620B1026812B14B
:1000D000126A02B1104793ED027A084BB8EEC77A64
:1000E000D3EDCD6AF6EE007AE7EE267AFDEEE77AFA
:1000F00017EE900A00F30B00704700BF98700020C5
:10010000034628B102681AB1516A09B193691847C8
:1001100093ED037A074BB8EEC77AD3EDCE6AF6EECD
:10012000007AE7EE267AFDEEE77A17EE900A00F302
:100130000B007047987000204FF47A7300F5006050
:10014000584340F6FF7390FBF3F000F57A70B0F57A
:10015000FA6FA8BF4FF4FA60B0F57A7FB8BF4FF4DA
:100160007A70704730B1036882881B691A4214BFE5
:1001700001200020704710B1036882881A837047FD
:1001800010B1036882885A83704773B50C460546E0
:1001900000B30668104B06F13F4202F57E0203EB06
:1001A000922393F8AA024CF069FDAB88009304F007
:1001B00003038DF80430C4F381038DF805306946DC
:1001C000C4F30013304664098DF806308DF80740FB
:1001D000FAF730FA02B070BD88480608F7B50C4649
:1001E00015460746A8B306681B4B06F13F4202F5C9
:1001F0007E0203EB922393F8AA024CF03FFDB888ED
:100200000090B0FA80F3C3F11F0303F00702C3F3B9
:10021000CC0306EB83039200196A0F27974021EA6B
:1002200007011962196A95400D431D6204F003032A
:100230008DF80430C4F381038DF805306946C4F3AA
:100240000013304664098DF806308DF80740FAF740
:10025000F1F903B0F0BD00BF8848060838B50409BD
:10026000013C032C00F00F0219D80E4D05EB44039E
:10027000B3F8B01241FA02F313F001000ED00123DB
:100280009340013B03EA0100254454F0ABF895F894
:10029000B832034404480C2202FB030038BD00209E
:1002A000FCE700BF88480608D47300202DE9F04F12
:1002B000542204460021BE4891B053F0FBFFBD49D3
:1002C000621E0846033412F8013F5D1E052D88BFEB
:1002D0000023944240F8043BF5D1B64A002352F87B
:1002E000040B012800F05A810133042BF7D10023BD
:1002F00051F8042B022A00F047810133042BF7D177
:100300000320FEF74FFC0420FEF74CFC0520FEF70F
:1003100049FC0620A64EDFF8B882FEF743FC3446BF
:100320004FF01A0B4FF0000A08F52F79277B57B3CF
:10033000384694F90D50FFF791FF28B105238371DA
:10034000002380F807B003721321FFF71EFF00237C
:1003500019F83310B94240F0DE8008EBC303D3F83C
:10036000C032954A2361182303FB0525D5F8E830F0
:100370002375591C0723A3750123C5F8E81063757D
:1003800085F8E4309A440BF1010B5FFA8BFBBBF16B
:10039000200F04F10C04C9D1BAF1000F00F0B880AD
:1003A000864DDFF8308200272B7C002B00F0A880E0
:1003B00068794CF063FC28794CF060FCD5F808A013
:1003C0005046FAF7AFF82C68D5F81490CDF80C80A9
:1003D0000023CDE90C33CDE90E330493069304F1E9
:1003E0004C030293EB680193142303FB09F34FF4CE
:1003F000806205934FF40063CDE907234FF4005169
:100400004FF48073CDE9091350464FF4003301A92E
:100410000B934CF045FBDAF80030694A43F00103D6
:10042000CAF800305168674B0B4043F440335360C7
:100430006268B9F1010F22F04072D4BF002301239A
:1004400022F4807242EA03226260A2685E4B13408B
:1004500043F00203A360E26A09F1FF3322F4700261
:10046000DBB242EA03530122E362304694464FFA7C
:1004700087FE437D6BB390F90D30734529D1037C22
:1004800090F81690092B4CD9A3F10A01D4F80CA0CE
:1004900001EB41014FF0070B0BFA01FB2AEA0B0AB3
:1004A00009FA01F141EA0A01E160062A48D8511E21
:1004B000D4F8349001EB81014FF01F0A0AFA01FAD7
:1004C00029EA0A0903FA01F141EA090161630132EB
:1004D000D2B20CF1010CBCF1070F00F10C00C8D135
:1004E000A36843F40073A360A36843F48073A3601C
:1004F000A36843F00103A360A36843F08043A360B3
:100500000137032F05F1180508F58C787FF44CAFFF
:1005100011B0BDE8F08F0133102B7FF419AF002329
:100520001FE7216903EB430B4FF0070A0AFA0BFAA6
:1005300021EA0A0A09FA0BF141EA0A012161B4E74A
:100540000C2A10D8D11FD4F8309001EB81014FF064
:100550001F0A0AFA01FA29EA0A0903FA01F141EA33
:1005600009012163B3E7A2F10D01D4F82C9001EB4E
:1005700081014FF01F0A0AFA01FA29EA0A098B40A1
:1005800043EA0903E362A2E7104B212203F8682C37
:1005900013F82C2C013203F82C2CB1E60B4B112252
:1005A00003F8742C13F82C2C013203F82C2C9EE643
:1005B00018700020A05F0020F8100020CC1100204F
:1005C00000230140E030FCFFFDF7FFC098700020E1
:1005D00088480608707000202DE9F04F85B0B04DB6
:1005E0000293B04B9D4220D26C798C4240F07081D6
:1005F0002C79844202D0002840F06A81EC79944240
:1006000040F066812C6884B11C220021201D53F02B
:1006100051FE25602B792371AA79A2600192012BEA
:100620002A7AE26006D0022B0DD00024204605B0C5
:10063000BDE8F08FE87AFFF711FE6B7A2374AB7A8E
:10064000A0616374F2E7E87AFFF708FE95F9098084
:10065000A06184F81080A87AFFF700FE0746606169
:10066000002800F0318114238F4E03FB08F3F218A9
:10067000F558002D00F02881937C002B40F0CB80B2
:1006800092F8089048464CF0F9FA09F01F024FEA38
:1006900059190123A9F102099340B9F1030F08D8B0
:1006A000DFE809F07872026C80490A6922EA0303E4
:1006B0000B61142303FB086308F101095879FFF764
:1006C000CDFD5FFA89F9034620B140F60A32C280B7
:1006D00080F80890142202FB08620393D079FFF798
:1006E000BDFD039B824620B140F60A52C28080F8CD
:1006F0000890142202FB086203939079FFF7AEFD85
:10070000039B834620B140F60A42C28080F80890DD
:10071000142202FB086292F80990019A12F0040276
:1007200001924A463CD04A211846FFF757FD4A46F7
:100730002A215046FFF752FD4A460A215846FFF744
:100740004DFD142303FB086393F804A0BAF1000FD6
:1007500006D05046FFF782FD4A460921FFF73EFDCD
:10076000534B9D4223D103F584335A6A42F480529D
:100770005A625A6A22F480525A6225E04B494A6909
:1007800022EA03034B6194E748490A6A22EA030319
:100790000B628EE745494A6A22EA03034B6288E707
:1007A0000A211846FFF71AFD4A460A21C1E7414BC4
:1007B0009D423ED103F500331A6A42F480421A6228
:1007C0001A6A22F480421A62019B002B65D1012231
:1007D00002212B880A4303F44153134343F4457326
:1007E0002B80AB8B23F400631B041B0CAB83072310
:1007F0002B822B889BB243F040032B80BAF1000F71
:1008000004D05046FFF72AFDFFF7B5FC142303FB85
:1008100008660123B374029BBB710E23FB71002396
:1008200038463B720921FFF7B0FC3846FFF7A3FCBE
:10083000FCE6214B9D4209D103F5FE331A6A42F4CE
:1008400000421A621A6A22F40042BCE71B4B9D4226
:1008500009D103F582335A6A42F400525A625A6A45
:1008600022F4005288E7164B9D4209D103F56843F4
:100870005A6A42F480125A625A6A22F480127BE762
:10088000104B9D42A0D103F564435A6A42F4001212
:100890005A625A6A22F400126EE70022114698E763
:1008A000A001000868030008B400002000380240DE
:1008B0000030014000380040003C0040003401405E
:1008C00000500140005401402046FFF74FF8ACE6CD
:1008D0000C3587E6074B03EB8003D3F83C333BB181
:1008E0009A881B6859690A4201D05A8370471A8353
:1008F000704700BF88480608064B03EB8003D3F817
:100900003C332BB11A689B8809B913837047538312
:10091000704700BF884806080A4B10B5D3F88845D1
:1009200024B1094A03212046F9F70EFB2046002195
:10093000F9F760FB20460549BDE8104040F62B4220
:100940004CF0D8B898700020009F24001488002034
:1009500038B5104CD4F8885525B10F4A6421284683
:10096000F9F7F2FA00212846F9F744FB6B681A6898
:10097000B2F844306FEA43436FEA53439BB2A2F8A4
:10098000443013889BB243F001031380012384F8A1
:100990008C3538BD98700020009F2400DFF8B0C16E
:1009A0002DE9F84F9CF88CE5BEF1000F40F0CC80AB
:1009B000DCF8889599F81030002B40F0C5809CF841
:1009C00090359CF891259CF89255ACF88EE50CF288
:1009D0009450F0463C268178C778C1F1FF0189B276
:1009E000002900F0AD80C1F1FF0179430488B4FB18
:1009F000F6FA0912BAF1050F20D8DFE80AF0030D64
:100A0000647283917A1A6243B2FBF6F252FA81F26F
:100A1000CDB2D2B23B460FE0B4FBF6F306FB134374
:100A20009BB2C3F13C037A1A5343B3FBF6F353FA78
:100A300081F3CDB2DBB23A464FF0010E1F0247EA16
:100A4000024747EA050B00210127C1F1170A07FAFF
:100A50000AFA08EB01041AEA0B0F04F12A0408BF92
:100A6000BA46A4B2394F01F1010118BF4FF0020A92
:100A7000182947F824A0E7D108F118081FFA88F8C8
:100A8000B8F5406F00F10400A5D18021ACF89417AF
:100A9000BEF1000F05D08CF892558CF891258CF89A
:100AA00090354FF44063ACF88E359CF89637002BA8
:100AB0004AD0484640F62B41F9F7C0FB4846BDE80E
:100AC000F84FF9F7EDBBB4FBF6F206FB12427D1AC4
:100AD00092B25543B5FBF6F555FA81F5CBB2EDB2BE
:100AE000A9E7B4FBF6F206FB124292B2C2F13C0255
:100AF0007C1A6243B2FBF6F252FA81F2CBB2D2B266
:100B00003D4699E7B4FBF6F506FB15447B1AA4B203
:100B10006343B3FBF6F353FA81F3CAB2DBB2EFE7F8
:100B2000B4FBF6F306FB13439BB27C1AC3F13C0300
:100B3000CAB26343B3FBF6F353FA81F1CDB269E76E
:100B40003D463A463B4677E7BDE8F88F14880020DB
:100B500098700020134B70B5D3F88845054604B350
:100B600093F88C15C9B96068026846790E48938974
:100B700030F816009BB223EA0003E0689381866890
:100B8000336823F001033360217413889BB243F070
:100B9000010313800177FFF7DBFE2046F9F720FB06
:100BA000056070BD98700020C846060838B5104C26
:100BB000D4F8880550B194F88C353BB194F8973748
:100BC000032B04D1F9F70CFB6423036038BD022B1F
:100BD0004FF0000503D1F9F703FB0560F6E784F851
:100BE0008C55FFF799FE0028F0D184F89607EDE7C1
:100BF000987000200346806B9B7903F001039942B3
:100C000001D0FFF7B8BAFFF7BBBA10B5837913F07C
:100C1000010F03F020020446C36B13D05B68002A67
:100C20001A7A08BF4221606B18BF0221FFF7D6FA7B
:100C3000012184F86012A4F85C12E06BBDE810405A
:100C4000F9F7E4BA5B68002A08BF22211A7AEAE7BA
:100C5000036C806B23B15B6801211A7AFFF7BEBA7F
:100C60000121FFF792BA2DE9F04183681C6866798B
:100C7000B1072FD594F86152C5B194F962528DB184
:100C8000B4F864124B08A4F86432204601F0010164
:100C9000FFF7B0FFA379013D6DB2580684F86252A8
:100CA00018D5BDB9002384F8613213E0A36A626AE3
:100CB00094F860129A4225D161B9A3791A0709D52F
:100CC000236CA06BD3B15B681A7AFFF787FA2046D2
:100CD000FFF79BFFF10740F1818094F85C32002B15
:100CE0007CD194F85D320133DBB2092B84F85D329C
:100CF00035D12046BDE8F041FEF7BAB91946FFF7F5
:100D000044FAE4E75A1CA069A262C35C2069A7798F
:100D10005B0043F40073A4F864320A23824228BFC4
:100D2000002284F862320123A26284F8613299B110
:100D30003B0711D5D4F83C8029464046F9F766FABE
:100D4000D8F80430606B1A7A2946FFF747FA84F81E
:100D500060522046FFF77CFF7D068ED4BAE70A2B4F
:100D60003CD194F85F322BB9B4F8663243F00103FA
:100D7000A4F86632B4F86602820501D4C3071AD417
:100D8000B4F86A320133A4F86A3294F85F5201234E
:100D90009D42A4F85C3221D1A179E06B002384F854
:100DA0005F3201F001014BF0F1FDE06B2946BDE837
:100DB000F041F9F72BBAE36AC0F3470013B1216B96
:100DC0009847E2E7E3696269D054E369E268013376
:100DD000B3FBF2F102FB1133E361D6E7BDE8F0812A
:100DE000F8B51E4B46681A6804461346B3FBF1F08B
:100DF000B0F5803F2ED281B22046F9F7A5F82368DE
:100E00001F687C7974B165B203212846F9F788F828
:100E1000002D07DB6109124A04F01F040123A340DF
:100E200042F82130BC7974B165B203212846F9F744
:100E300077F8002D07DB6109094A04F01F0401233C
:100E4000A34042F82130326813889BB243F001037B
:100E50001380F8BD012BCBD95B08C7E70401002044
:100E600000E100E08160C06BBAE7002ABCBF8018D7
:100E70005242002BBCBFC9185B420028BCBF121AEB
:100E80000020F0B584180029A4F11D04BCBF5B1834
:100E90000021002CC8BF121BCC180F3C002CC8BF6F
:100EA0001B1B0B4E02440B443C274FF0200C90427E
:100EB0000CDC06EB40050C4604E007FB04FE0134A5
:100EC00025F80EC09C42F8DD0130F0E7F0BD00BF10
:100ED0003078002008B5114B1A6C42F080521A6429
:100EE0000F4A012111620F4AFF215162CA2151624A
:100EF000532151625B6FDB0009D400210120FAF716
:100F0000E9F8BDE8084008490020FAF7E3B80020F6
:100F1000FAF7F0F8044B9842EFD108BD00380240D0
:100F200000000E420028004076614E6938B50C463C
:100F300005461946046014B12046F9F705F8BDF8D6
:100F400010102046F9F756F863681A68B2F8443072
:100F50006FEA43436FEA53439BB2A2F844301388CD
:100F60009BB243F0010313802046F9F739F90023BF
:100F7000A860036038BD2DE9F04F85B006469DF8A6
:100F80003CA0039289469846FCF734FE834648B15C
:100F9000214C94F8582B082A09D9204A0021042012
:100FA000FCF78AFD0025284605B0BDE8F08F531CEC
:100FB0005C21DFB284F8587B04F65C3501FB024407
:100FC00002FB01550022C4F85C2B84F8602B3079B9
:100FD000FFF744F9044620B1022280F80690C2715E
:100FE0000772BDF838300093039A434659462846A5
:100FF000FFF79CFFBAF1000F05D0327A022120469C
:10100000FFF7ECF8CFE720461121FFF7BEF82046A6
:10101000FFF7B6F8C7E700BF9870002018EE060883
:1010200030B51E4B2DED028B1C68B4FBF1F303F5BC
:101030007F4383B0FF331B0CB4FBF3F40023B4FBFA
:10104000F1F5019200932246ABB20221F0EE408A04
:10105000B0EE608AFFF78FFFE0B107EE904AB5EE81
:10106000408AF1EE10FAF8EE677A0ABF07EE105ADE
:1010700068EE270AF8EE470A9FED097AC0EE876A04
:101080000123037127EE667AC0ED046AA8EEA77A01
:1010900080ED037A03B0BDEC028B30BD040100206B
:1010A00000007A440023064910B51C46984200DC33
:1010B00010BD51F833200AB1926814600133F5E78E
:1010C000083C00202DE9F0414C4B1A784C4B03EBC7
:1010D00042035B783BB14B4B1E78C0B9DFF828C1A7
:1010E0000025AE4217DCBDE8F08154F832301BB960
:1010F00001329642F9DCF1E719790029F8D003F1C1
:101100001001503341F8045F9942FBD1F0E73E4CA7
:1011100000220725EDE75CF83530002B3CD01A792A
:10112000002A39D01A68002A36D0D368002B33D071
:101130009B68002B30D0EFF31187102383F31288C4
:101140005468DFF8C8E0216864798B893EF8144060
:101150009BB223EA04038B81D36899680B6823F060
:1011600001030B6042F21174D1688B68D3F80080E0
:1011700018F0010F01D0013C10D11C68E407FFB248
:101180000ED553681A685B7991893EF813300B438A
:101190009BB2938187F311880135A2E700BFE3E793
:1011A0000C69D1F804801F2C4FF0200185BF203C32
:1011B000A140A140C8F80C1098BFC8F808101968E1
:1011C00098B141F48071196012215960196821F0B9
:1011D0001001196003231374BFF34F8FD36899680C
:1011E0000B6843F001030B60CBE721F480711960B9
:1011F000196841F0100119601074EDE7BC3B002044
:101200004C480608846F0120083C0020C8460608A8
:1012100013B50F4C8DF80700D4E90423A16853439C
:101220008B4212D06368E0680DF10701184452F058
:10123000FDFF636822691344A268B3FBF2F102FB6D
:101240001133636063690133636102B010BD00BF95
:10125000E03B00200F4B1B78062B14D8DFE803F08F
:10126000041316070A0D10004FF4C87070470A4B9C
:10127000588870474FF47A6070474FF4FA507047BF
:101280004FF47A5070474FF47A7070474FF4FA6019
:10129000704700BFBC3B0020483D00202DE9F04FC7
:1012A0002DED028BA64FA74D3B78DFF8D4B299B055
:1012B00000240393AA462646A946DAF80080404651
:1012C000F8F7D6FD584490F8982E022A6FD0032ADA
:1012D00076D0012A09D1DAF80C2022F0807222F0AF
:1012E000080242F00402CAF80C205046FEF750FAF9
:1012F00070B9142202FB0692D16801F00C02042A94
:1013000006D14046FDF750FF0134E4B20444E4B294
:1013100001360A2E0AF1140ACFD18B4EA6F1C80865
:101320004046FEF735FAC0B9D8F80C104A0714D574
:1013300001F00C03042B10D0039B9C4247D221F0F8
:10134000080141F00401D8F80000C8F80C10FDF7BE
:101350002BFF0134E4B20444E4B208F11408B045B0
:10136000DED14FF000094C464E46C8462846FEF7EF
:101370000FFAA8B3754A434601210420FCF79CFBF1
:1013800008F10108B8F10A0F05F11405EED13E7815
:101390000C2E40F38F8001238BF8A63E6C4A0C2361
:1013A0000093334600210420FCF786FBA7E0DAF81F
:1013B0000C2022F0807222F0040242F0080292E730
:1013C000DAF80C2022F00C0242F080728BE721F058
:1013D0000401D8F80000C8F80C10FDF7E5FEBCE7E2
:1013E000E9684B070AD5039B9E4207D221F008010A
:1013F0002868E960FDF7D8FE0136F6B2EA68100702
:101400001AD5286805A900239C420DDC0823EB604F
:1014100018AB03EB890209F1010A082142F8245CA8
:10142000D146FDF7C1FEABE751F804CFDCF800C0B0
:10143000604501D00133E7E751071AD528680EA9A6
:1014400000234B450DDB0423EB6018AB04F1010ACC
:1014500003EB8404042144F8485CFDF7A5FE5446E0
:101460008EE751F804CFDCF800C0604501D00133AD
:10147000E7E7D30184D5286805AA00239C4202DC53
:101480000EAA00230EE052F8041F096888423FF4B8
:1014900077AF0133F2E752F8041F096888423FF43E
:1014A0006FAF01334B45F6DB4FF08071E960FDF71C
:1014B0007BFE65E7274B1979274B0329197035D92E
:1014C0000B1F022B34D8FFF7C5FE244A244B9FED97
:1014D0001A7B80B2B3FBF0F3136000235360214BFF
:1014E00083ED007B204BCBF8A83E204B13F8113046
:1014F000002B47D11E4A02210420FCF7DDFA22F01E
:1015000059F99BF8AC3E0446002B40F0C080194AC4
:1015100002210420FCF7D0FA9BF8A60EB0FA80F066
:10152000400919B0BDEC028BBDE8F08F124BDAE731
:10153000124BD8E7AFF3008000000000000000006D
:10154000846F0120A00500206806002053EE0608E5
:101550006BEE0608483D0020BC3B0020C83B002045
:1015600040420F00D03B0020D7F100084C4806084D
:1015700097EE060813EF060845F50008D5F10008B8
:1015800098700020A64217DC754F9FED768A0DF10A
:1015900014080024A642B2DD734B58F8045F5B6860
:1015A000C3F3007A714B1B78062B6CD8DFE803F08D
:1015B000621B220B2B2B2B0003238BF8A63E6C4ABD
:1015C00000943346EEE6FFF745FEDFED6A0A01467A
:1015D0005246B0EE600A2846FFF722FD47F8340075
:1015E000002845D125E0FFF735FEDFED630A01460F
:1015F0005246EEE7FFF72EFEDFED600A9FED600A30
:1016000001465246E7E7052B1DD05E4A5E49062B90
:1016100018BF0A46CDF804A04FF0000A2846CDF8BE
:1016200000A014230221FFF7A6FC054668B947F87D
:10163000340005238BF8A63E544A2346002104209B
:10164000FCF73AFA5BE7524AE4E700F11403194663
:101650000068039312224BF04DFA039B30B11846F9
:101660004822514652F026FE01232B7147F8345090
:1016700001348FE7FFF7EEFD9FED3A0A014652462F
:10168000F0EE480AA7E7002347F83430D1E71228E4
:101690000BDD02238BF8A63E3E4A12230093002165
:1016A00003460420FCF708FA36E79BF8B63E012B08
:1016B0000CD0022B0ED0384BCBF8BC3E9BF8B63E7C
:1016C000002B38D0022B09D0344A21E74CF004F922
:1016D000334BF1E74CF000F9324BEDE74B46122B60
:1016E000B8BF12239BB29C4227DC4C45A8BF4C4696
:1016F0002D4FDFF8B880DFF870900EAE0025A542C0
:10170000BFF60AAFD9F80420BBF8B03EB8FBF3F33C
:10171000C2F300720192BBF8AE2E00920321234A5D
:1017200056F8040F9BB2FFF726FC014670B147F84C
:10173000040B0135E3E74B46D4E704208BF8A60EF3
:101740001B4ACDF8009023460021ABE705238BF818
:10175000A63E184A2B460420FCF7AEF9DCE600BF93
:10176000083C00206F12833A886F0120BC3B0020A8
:10177000B5EE0608000000006F120339ACC5A737AC
:10178000ACC5A736001BB700C0C62D00EEEE06089C
:10179000808D5B002DEF0608F1F1000859EF060877
:1017A0005D1803080DF200085460002040420F004D
:1017B00095EF0608CBEF0608034AD2F8BC2E12B10B
:1017C000112800D8104770479870002040B10138A8
:1017D0000023FF2803F1010203D840EA032080B26E
:1017E000704740081346F4E703681B68184703680E
:1017F0005B68184703689B68184703681B6A70B5E5
:1018000006460C46154683B1BDE870401847304681
:10181000FFF7F0FF0028FAD014F8011B3046FFF75D
:10182000E3FF2B1B002BF2DC70BD0D44F9E7E4E76E
:101830000368DB68184703681B69184703685B691E
:1018400018470368DB6A03B11847704703681B6BCE
:1018500003B118477047164B1B6813F0100F154B58
:1018600005D0B3F8C02E12F0040F18BF002093F873
:10187000EE2E72B1D3F8F02ECAB1926838B1B3F837
:10188000F41E0D4BB3FBF1F35B1013607047106057
:101890007047D3F8F82E93F8FC3E0BB980F00100A6
:1018A0002AB11368928808B11A8370475A83704727
:1018B000E06E01209870002040420F00BFF34F8F70
:1018C0000549064BCA6802F4E0621343CB60BFF3DC
:1018D0004F8F00BFFDE700BF00ED00E00400FA05F8
:1018E00008B572B600224FF0FF31930003F1604358
:1018F00003F561430132082AC3F88010C3F8801150
:10190000F3D1FFF7DBFF08B50120F9F7F3FB01285E
:1019100009D10021F9F7DEFB034B1A6882F308882E
:101920005B689847FEE708BD0000FF1FEFF31183D7
:10193000102282F3128809490A6801320A604FF0C6
:10194000E02207499069C1F8000F0020C1F8040F98
:101950001269DBB283F31188704700BF042A0020AC
:1019600098700020074A084B5168D3F8083F584345
:101970004FF47A73B0FBF3F053685B1A8342FBD9E0
:10198000704700BF001000E09870002010B50446BA
:101990004FF4FA70FFF7E6FF6069BDE81040FEF70C
:1019A000EABB90F910302DE9F0411646142253435A
:1019B0000D4A52F80380836813F0020504460F466F
:1019C00002D140694CF0F2FC394640464EF06AFDC7
:1019D000314640464EF066FD15B92046FFF7D6FF6A
:1019E0000120BDE8F08100BFB40000207FB503797D
:1019F000012B0D460AD0022B19D18368DB0758BF93
:101A000001F07F0104B0BDE87040CAE781688DF83D
:101A10000F2001F001010DF10F0200920191417CB4
:101A200090F910002A46F9F709FB04B070BD0020B8
:101A3000FBE700682E22F421D8E7044B00681A8ED9
:101A40009201343202F0FC02F421CFE7A05F0020C3
:101A500008B53122F4210068FFF7C8FF012008BD56
:101A6000006801225821C1E7006801224821BDE732
:101A7000006802220821B9E7006801220821B5E7C1
:101A800010B50446002221210068FFF7AFFF20684F
:101A9000FC222021FFF7AAFF206840222421FFF723
:101AA000A5FF20680C222321FFF7A0FF2068002259
:101AB0002221FFF79BFF012010BD10B50122044633
:101AC0000B210068FFF792FF20B120681D22092139
:101AD000FFF78CFF00F0010010BD044B0246D3F865
:101AE0000C0F08B1802181E7704700BF987000207B
:101AF00010B5B020FFF7F1FF4020FFF7EEFF002008
:101B0000FFF7EBFF1020FFF7E8FF4FF48064013C84
:101B10000020A4B24CF0D7FA002CF8D110BD10B5BB
:101B20000446A1F15000C0B2FFF7D7FF04EB440018
:101B3000400004EB440400F00E00FFF7CEFFC4F3B6
:101B4000C3001030BDE81040C7E708B55038C0B238
:101B5000FFF7C3FF0020FFF7C0FFBDE808401020DB
:101B6000BBE738B500221F2337210120FEF734FDE3
:101B70003C4BC3F80C0F10B90024204638BDAE20F2
:101B8000FFF7ABFF04460028F6D0D420FFF7A5FFEF
:101B90008020FFF7A2FFA820FFF79FFF3F20FFF75D
:101BA0009CFFD320FFF799FF0020FFF796FF40200E
:101BB000FFF793FF8D20FFF790FF1420FFF78DFFB5
:101BC000A120FFF78AFFC820FFF787FFDA20FFF781
:101BD00084FF1220FFF781FF8120FFF77EFFCF20D7
:101BE000FFF77BFFD920FFF778FFF120FFF775FFA4
:101BF000DB20FFF772FF4020FFF76FFFA420FFF705
:101C00006CFFA620FFF769FFAF20FFF766FFA62055
:101C1000FFF763FFAE20FFF760FF2020FFF75DFFB7
:101C20000020FFF75AFFB020FFF757FF4020FFF7D3
:101C300054FF0020FFF751FF1020FFF74EFF4FF435
:101C40008065013D0020ADB24CF03DFA002DF8D189
:101C50008120FFF742FFC820FFF73FFFAF20FFF7CB
:101C60003CFF8AE79870002010B504460068FDF735
:101C7000EBFEC36820681B0EBDE810404FF0010268
:101C80000CBF48215821B1E608B5FFF7AFFE014B64
:101C9000187008BDF81000202DE9F0411E4690F99B
:101CA00010301546142253430E4A52F803808368BD
:101CB0009A0704460F4602D440694CF077FB394638
:101CC00040464EF0EFFB33462A46002140464EF098
:101CD00081FBA3689B0702D42046FFF757FE012033
:101CE000BDE8F081B4000020F7B50779012F164652
:101CF0000AD0022F15D18468E40758BF01F07F0194
:101D000003B0BDE8F040C7E7826802F00102CDE908
:101D100000620A46417C90F91000F9F78FF903B090
:101D2000F0BD0020FBE707B552BAADF8042002234E
:101D300001AAFFF7D9FF024B187003B05DF804FB4E
:101D4000F810002010B50A4C002384F8103F84F8E6
:101D5000111F84F8122F032304F57162FF21FFF78E
:101D6000C3FF00280CBF6FF00C00002010BD00BFA7
:101D70009870002010B50B4C002384F8103F130A14
:101D800084F8111F84F8123F84F8132F042304F5FC
:101D90007162FF21FFF7A8FF00280CBF6FF00C0055
:101DA000002010BD98700020024A006800235121D5
:101DB0009AE700BFA88000202DE9F0411E4690F967
:101DC00010301546142253430E4A52F8038083689C
:101DD0009A0704460F4602D440694CF0E7FA3946A8
:101DE00040464EF05FFB33460022294640464EF007
:101DF000F1FAA3689B0702D42046FFF7C7FD012034
:101E0000BDE8F081B4000020F7B50779012F164630
:101E10000AD0022F15D18468E40758BF41F0800131
:101E200003B0BDE8F040C7E7826802F00102CDE9E7
:101E300000620A46417C90F91000F9F725F903B0D9
:101E4000F0BD0020FBE713B5062304466A46006890
:101E50000221FFF7D9FFB8B1BDF9003007EE903A83
:101E6000BDF90230F8EEE77AC4ED077A07EE903A52
:101E7000BDF90430F8EEE77AC4ED087A07EE903A3F
:101E8000F8EEE77AC4ED097A02B010BD13B502236B
:101E900004466A4600680321FFF7B6FF10B9002028
:101EA00002B010BD9DF90130002BF8DA206807233D
:101EB0006A461221FFF7A8FF0028F0D09DF9022002
:101EC0009DF8013043EA022313EB430348BF033379
:101ED0009B1007EE903A9DF904209DF8033043EAE9
:101EE000022313EB4303F8EEE77A48BF03339B105A
:101EF0009DF90620C4ED047A07EE903A9DF805306E
:101F000043EA022313EB4303F8EEE77A48BF0333B7
:101F10009B10C4ED057A07EE903AF8EEE77AC4ED2F
:101F2000067ABDE738B504460068FDF78DFD0C2341
:101F30000546021D19462068FFF766FFA870B8B174
:101F4000B5F9043007EE903AF8EEE77AC4ED077A77
:101F5000B5F9063007EE903AF8EEE77AC4ED087A64
:101F6000B5F9083007EE903AF8EEE77AC4ED097A51
:101F700038BD38B504460068FDF766FD0D230546FB
:101F8000C21C0C212068FFF73FFFA870B8B1B5F95B
:101F90000A3007EE903AF8EEE77AC4ED077AB5F921
:101FA0000C3007EE903AF8EEE77AC4ED087AB5F90E
:101FB0000E3007EE903AF8EEE77AC4ED097A38BDB4
:101FC00013B503230C46006801AA2221FFF71CFF6A
:101FD00030B1BDF9053003EB83031B12E6332380D8
:101FE00002B010BD13B5062304466A4600681F21DF
:101FF000FFF70AFFD0B1BDF80030DBBA07EE903A28
:10200000BDF80230F8EEE77ADBBAC4ED047A07EEE9
:10201000903ABDF80430F8EEE77ADBBAC4ED057A01
:1020200007EE903AF8EEE77AC4ED067A02B010BDFA
:1020300013B5062304466A4600682521FFF7E4FE2F
:10204000D0B1BDF80030DBBA07EE903ABDF80230EF
:10205000F8EEE77ADBBAC4ED077A07EE903ABDF8FE
:102060000430F8EEE77ADBBAC4ED087A07EE903A6E
:10207000F8EEE77AC4ED097A02B010BD13B5022379
:102080000C46006801AA1D21FFF7BEFE98B1BDF8FD
:102090000430DFED0A6ADBBA07EE903AB8EEE77A71
:1020A000C7EE267A9FED067A77EE877AFDEEE77A1D
:1020B00017EE903A238002B010BD00BFCFF7534116
:1020C00000007A4370B5066805463046FDF7BCFC53
:1020D0000E230446021D3B213046FFF795FEA070FB
:1020E000B8B1A389DBBA07EE903AF8EEE77AC5ED0E
:1020F000077AE389DBBA07EE903AF8EEE77AC5EDA6
:10210000087A238ADBBA07EE903AF8EEE77AC5ED53
:10211000097A70BD07B50223006801AAF621FFF70E
:1021200073FE20B1BDF80430024A5BBA138203B0DB
:102130005DF804FBA05F002007B50323006801AA37
:10214000F621FFF761FE80B19DF805309DF804206F
:1021500007491B0243EA02439DF806201343B1F9E5
:102160003020C2F10802D3404B6303B05DF804FB9A
:10217000A05F002037B50623F7210068144C6A469B
:10218000FFF742FE1349D8B19DF801209DF80030B9
:102190009DF80350120142EA03329DF8023042EAF0
:1021A00013129DF804308A651B0143EA05339DF83C
:1021B000055043EA151344E93A238B6303B030BD5D
:1021C00054F8E83C8B6554F8E43C8B63F6E700BFB9
:1021D00090810020A05F002007B50323006801AABA
:1021E0001946FFF711FEA0B19DF804309DF80510C7
:1021F0009DF904201B0443EA01239DF80610002AE0
:10220000ACBF00224FF07F420B431343024AC2F897
:102210000C3103B05DF804FBA05F002007B5032379
:10222000006801AA0021FFF7EFFDA0B19DF804307E
:102230009DF805109DF904201B0443EA01239DF835
:102240000610002AACBF00224FF07F420B4313431D
:10225000024AC2F8083103B05DF804FBA05F002019
:1022600013B5044600680379022B0CBF43210321F8
:1022700006236A46FFF7C8FD18B9E086A06302B0DE
:1022800010BDBDF800305BBAE386BDF802305BBA22
:102290006387BDF804305BBA2387F0E713B50023EA
:1022A000C38683630446062300686A460321FFF75A
:1022B000ABFD78B1BDF8003003EB4303E386BDF915
:1022C00002305B4203EB43032387BDF8043003EB8A
:1022D0004303638702B010BD07B5012301AAFF21A4
:1022E0000068FFF791FD03B05DF804FBF7B5054604
:1022F0000068FDF7A9FB00230370042304460DEBDF
:1023000003022868FF21FFF77FFD10B9002003B00A
:10231000F0BD286804236A46FF21FFF775FD0028F9
:10232000F4D09DF804309B09023B012BEED9BDF897
:102330000420BDF80630BDF80050BDF8021052BAB6
:1023400043F6FF77C2F30D02BA42DFD0002ADDD098
:102350005BBAC3F34A1340F2FF76B342D6D0002BE8
:10236000D4D06DBAC5F30D05BD42CFD0002DCDD070
:1023700049BAC1F34A11B142C8D00029C6D0561B90
:10238000002EB8BF7642FF2EC0DC5E1A002EB8BF0A
:102390007642FF2EBADC01262A440B4432413341F7
:1023A0002670C4F80520C4F80130B0E773B50646BE
:1023B0000068FDF749FB0323C568044601AA30689D
:1023C0000021FFF721FD98B19DF805309DF804200C
:1023D0001B0243EA02439DF806202D0E43EA020346
:1023E0001BBF2361E36843F0807323F07F43E36006
:1023F00002B070BD37B505460068FDF725FB002328
:102400000370042304460DEB03022868FF21FFF745
:10241000FBFC40B19DF804309B0907D00B4A042116
:102420000320FBF749FB002003B030BDBDF80420BA
:10243000BDF8063052BA5BBA92B2C3F34A13012117
:102440002170C4F80520C4F80130EDE7F0EF06086C
:1024500007B5022301AAFFF7D7FC044B1870BDF89B
:10246000040040BA80B203B05DF804FBF81000200D
:1024700038B515460C4A0B0A82F8103F82F8111F36
:10248000022302F57162FF210446FFF72DFC30B1F3
:1024900001232A46FF212046FFF7B6FC10B96FF052
:1024A0000C0038BD0020FCE7987000202DE9F041B9
:1024B000104D05F571681646002485F8111F02239A
:1024C0004246FF21074685F8104FFFF70DFC18B96B
:1024D0006FF00C00BDE8F08102234246FF21384630
:1024E000FFF792FC0028F3D0B5F8103F5BBA3380B9
:1024F0002046EFE7987000202DE9F341744D046801
:10250000DFF8D8810023064685F8FE302D27B9B2C2
:1025100018F8012B20460137FFF714FC882FF6D15D
:10252000402287212046FFF70DFC00238DF806305E
:102530009DF80630002B6FD0012286212046FFF740
:1025400001FC002287212046FFF7FCFB092208211D
:102550002046FFF7F7FB00220B212046FFF7F2FB96
:10256000002851D137680DF106025E213846FFF789
:102570009DFFBDF80630B3F5D77F00F0A58059D890
:10258000512B00F09F804DD81D2B70D01E2B00F0DA
:102590009980306821214BF068FC34680DF1060207
:1025A000DE212046FFF782FFBDF806309FED497A15
:1025B0002822C3F30903534307EE903AF8EEE77A73
:1025C000454A67EE877A0021FCEEE77A82F8101F11
:1025D00017EE903A6C2182F8111F190E82F8121F23
:1025E000190C82F8131F190A82F8141F82F8153F7C
:1025F000FF2102F5716206232046FFF775FB306864
:1026000040228721FFF79EFBB0FA80F0400985F851
:10261000FE0002B0BDE8F0810DF1060120464BF04E
:10262000B5FC85E7AD2B4FD0D62B01D0602BB0D1B8
:1026300021241DE040F2E132934247D00CD840F211
:10264000D922934242D040F2E122934202D0B3F524
:10265000E67F9ED164240BE040F28F42934203D088
:1026600040F29152934294D14FF4FA7400E00F2457
:1026700000288ED10A224B213846FFF763FB0F2238
:1026800060213846FFF75EFB0D2263213846FFF7D5
:1026900059FBB82269213846FFF754FB40F60D720A
:1026A00078213846FFF766FB40F60E627A213846FD
:1026B000FFF760FB00287FF46CAF214638464BF0F3
:1026C000D4FB66E71424D3E73224D1E7C824CFE74C
:1026D000A05F00209A99893F98700020D04B06088F
:1026E00037B5134D95F8FE300446FBB100680DF187
:1026F00005014BF04BFC9DF805307BB10DF1060256
:1027000020689621FFF7D2FE0A22BDF80630B3FBFF
:10271000F2F3084A9360012385F8FF302068012214
:10272000862103B0BDE83040FFF70CBB03B030BDDD
:10273000A05F0020F810002013B5022301AA044670
:1027400051210068FFF760FB114AE8B1BDF8043081
:102750005BBA9BB2D360D368B3F5C87F02DD4FF09C
:10276000FF33D3600B4B0C4A196852F8E03C32330C
:102770008B4207D242F8E01C20680023E83A51213E
:10278000FFF7B2FA02B010BD6FF00103E9E700BF36
:10279000F8100020042A00209081002007B50223B1
:1027A000006801AA0021FFF72FFB0F4B83F80401FB
:1027B000B0B1BDF804300D4A5BBA9BB2B3F5FA6F05
:1027C0003FBF0A21B3FBF1F307EE903AF8EEE77A48
:1027D0002BBF4FF0FF33FDEEE77A1361C2ED047AB1
:1027E00003B05DF804FB00BFA05F0020F8100020DC
:1027F000F8B5254C05460323006804F118020021B2
:10280000FFF702FB00283CD0A77E04F11706032146
:102810000023013909D19F42286817D06FF00203C5
:102820006361BDE8F8404BF01CBB16F8012F08208F
:1028300053405AB2002ABBBF520082F007025B002D
:10284000D3B2A8BFDBB20138F3D1E2E7238B5BBA86
:102850009BB25A1E92B24FF6FD718A4202D94FF0D6
:10286000FF33DDE707EE903AF8EEE77AF2EE046A1E
:1028700087EEA67AFDEEC77A17EE903A2868636174
:10288000CFE76FF00103F9E7F810002013B502233A
:102890000C46006801AA0021FFF7B6FA60B15CB1EE
:1028A0009DF805309DF90420DB0903EB830302EB5F
:1028B000820203EB4203238002B010BDF8B590F909
:1028C00010301546142253430D4AD75883689A078F
:1028D00004460E4602D440694BF068FD3146384646
:1028E0004DF0E0FD01230022294638464DF072FDEF
:1028F000A3689B0702D42046FFF748F80120F8BDE3
:10290000B400002073B50379012B16460AD0022BC0
:1029100015D18368DB0758BF41F0800102B0BDE8E4
:102920007040CBE7826802F00102CDE900620A46FE
:10293000417C90F91000F8F7A7FB02B070BD0020B1
:10294000FBE713B504466A4600680821FFF7DAFF83
:102950009DF80030DB0602D4002002B010BD2068D4
:1029600006236A460021FFF74FFA0028F4D09DF8AD
:1029700001309DF800209DF80410DFED496A1B022C
:1029800003EB02439DF802201C021A449DF8033019
:1029900048BF02F17F42090201EB034107EE902A92
:1029A0009DF80530F8EEE77A0B44090248BF03F1C1
:1029B0007F4387EEA67A07EE903AF8EEE77A394B36
:1029C000C7EEA63AB3F96A20B3F97410D3ED196AC9
:1029D000D3ED187AB8EEE66A06EE902AB3F96C20C9
:1029E00003EE101AB3F9681005EE902AB3F96E20C1
:1029F00004EE901A2C4905EE102AB3F9702011F854
:102A0000DC1C04EE102AF8EEE44A1129F8EEE77A0D
:102A1000F8EEE66AF8EEE55AB8EEC55AB8EEC44AE2
:102A2000B3F9722064EEA34A67EE232A2CD1B8EEE4
:102A3000C33AA7EE034AE4EE075AA5EE876AE6EE2C
:102A4000077A06EE102AB8EEC66A77EEA47AA7EEE9
:102A5000065AE5EE076AB3F95C20E6EEA27A07EEC5
:102A6000102AB3F95E20C3ED1E7A07EE902AF8EE25
:102A7000E77AB8EEC77A67EEA37AF6EE006AE7EE79
:102A8000267AC3ED1F7A68E7E7EE045AE7EE056A97
:102A9000A5EE876AE6EE077A77EEA47ADBE700BF59
:102AA00000007848A05F0020908100202DE9F341CC
:102AB00016460DF107021D4607468846FFF722FF1E
:102AC0009DF8074006EA0403AB4209D024EA060257
:102AD0002A434146384602B0BDE8F041FEF786BFC2
:102AE00002B0BDE8F0811FB50446002300688DF8F0
:102AF00007300DF107022721FFF704FF60B19DF8B1
:102B000007301B0708D52068062302AA2821FFF7F3
:102B10007BF920B9E086A063002004B010BDBDF9A8
:102B20000830002BB8BF03339B10E386BDF90A3091
:102B3000002BB8BF03339B102387BDF90C30002B4B
:102B4000B8BF03339B106387E7E71FB50021044636
:102B5000C18681630DF107020068FFF7D3FE10B94B
:102B6000002004B010BD9DF807301B07F8D5206881
:102B7000062302AA0121FFF747F90028F0D0BDF88B
:102B800008305BBAE386BDF80A305BBA2387BDF82C
:102B90000C305BBA5B426387E3E730B5002585B054
:102BA0000446C58685630DF1070200680621FFF71C
:102BB000A9FE10B9002005B030BD9DF80730DB0735
:102BC000F8D52068062302AA2946FFF71DF9002838
:102BD000F0D0BDF80830E386BDF80A302387BDF891
:102BE0000C306387E7E707B50DF10702FFF78AFEB0
:102BF000034B18709DF8070003B05DF804FB00BF9D
:102C0000F8100020F8B5144E144F41F001020021D5
:102C10000446FFF739F8356847F8D85C1321204699
:102C2000FFF7E1FF10F007000BD001220B21204637
:102C3000FFF72AF8002220461146FFF725F8012069
:102C400008E057F8D42C002AE8D033689BB25B1B0D
:102C50009A42E3D2F8BD00BF042A002090810020F0
:102C600010B50C460121FFF7BEFFC0F3001323701F
:102C7000C0F3C003A370C0F380036370C0F380137C
:102C8000C0F3C010E370207110BD2DE9F8430F466A
:102C9000502114460546FFF7A6FF01304000C0B2A0
:102CA000208046212846FFF79EFF2C4E23780130D6
:102CB00080B273434FF47A78A08003F5FA734FF42F
:102CC000FA69B3FBF8F25121B3FBF9F300FB0233CD
:102CD0002846B3FBF8F3E360FFF7BAFBC2B2C0F3D8
:102CE0000F2023788240013292B27343E28003F5D1
:102CF000FA732846B3FBF8F1B3FBF9F302FB013397
:102D00007021B3FBF8F32382FFF76DFF0130400021
:102D1000C0B2608071212846FFF79AFBC3B2C0F3AE
:102D20000F2083400133FA789BB2238112B1E288ED
:102D30009B1A2381A3782089734303F5FA734FF418
:102D40007A724FF4FA65B3FBF2F1B3FBF5F300FBD3
:102D50000133B3FBF2F36382BDE8F883002F3A003E
:102D60002DE9F047DB4FDFF87483DFF874934FF4FD
:102D7000FA738AB0044600268921006847F8D43CDB
:102D800088F8FC60FFF72FFF40F00102D2B2206804
:102D90008921FEF779FF324620688821FEF774FF0B
:102DA000206801228021FEF76FFF20680122FF21A9
:102DB000FEF76AFF324631462068FEF765FF912133
:102DC0002068FFF710FF314607F8D00C0122206879
:102DD000FEF75AFF32462068FF21FEF755FF3246C4
:102DE00020688021FEF750FF60212068FFF7FBFE7E
:102DF00040F01202D2B220686021FEF745FF206841
:102E000020224421FEF78FFF2068FF220121FEF7D8
:102E10003BFF2568012280212846FEF735FF01226D
:102E2000FF212846FEF730FF324631462846FEF79E
:102E30002BFF0622FF212846FEF726FF8321284686
:102E4000FFF7D1FE40F00402D2B283212846FEF7FC
:102E50001BFF0722FF212846FEF716FF01228121D2
:102E60002846FEF711FF012280212846FEF70CFFBD
:102E70006B2294212846FEF707FF3246832128461D
:102E8000FEF702FFD9F8006047F8D86C8321284686
:102E9000FFF7A9FE002800F046830122284683217F
:102EA000FEF7F2FE92212846FFF79DFE0022C0F3B6
:102EB000C716814681212846FEF7E6FE06222846EF
:102EC000FF21FEF7E1FE83212846FFF78CFE8321D8
:102ED00000F0FB022846FEF7D7FE28460122FF211C
:102EE000FEF7D2FE284601220021FEF7CDFE28463D
:102EF0000022FF21FEF7C8FE284600228021FEF7AF
:102F0000C3FE062303AAB0212068FEF77DFF2068D8
:102F10000122FF21FEF7B8FE206800224F21FEF7B4
:102F2000B3FE20682C224E21FEF7AEFE2068002260
:102F3000FF21FEF7A9FE2068B422B621FEF7A4FE09
:102F40000025002E18BF0C2609F07F092A46012013
:102F5000C5F3C40C0CF128035FFA85FE0DEB030CDE
:102F600076451CF81C3C05F0070102D8914540F05D
:102F7000E58200FA01F123EA01030CF81C3C01355B
:102F8000302DE5D1062303AAB0212068FEF7ACFE60
:102F9000514B01221870FF212068FEF775FE0022B8
:102FA00011462068FEF770FE20680022FF21FEF720
:102FB0006BFE206800220921FEF766FE20680022D1
:102FC0001021FEF761FE206800221121FEF75CFE51
:102FD000206801222421FEF757FE2068FF222521C8
:102FE000FEF752FE206800227521FEF74DFE206894
:102FF0000122FF21FEF748FE20682C224E21FEF719
:1030000043FE206800224821FEF73EFE2946206844
:103010002022FEF739FE20680022FF21FEF734FE51
:10302000294620680922FEF72FFE2068002254213D
:10303000FEF72AFE206804223121FEF725FE2068D3
:1030400003223221FEF720FE206883224021FEF772
:103050001BFE206825224621FEF716FE206800226E
:103060006021FEF711FE206800222721FEF70CFEEA
:10307000206806225021FEF707FE20680022512119
:10308000FEF702FE206896225221FEF7FDFD206821
:1030900008225621FEF7F8FD2A4620685721FEF740
:1030A000F3FD206800226121FEF7EEFD206800227A
:1030B0006221FEF7E9FD206800226421FEF7E4FDAD
:1030C000206800226521FEF7DFFD2068A02266212E
:1030D00008E000BF90810020F8100020A05F0020D1
:1030E000042A0020FEF7D0FD20680122FF21FEF710
:1030F000CBFD206832222221FEF7C6FD2068142273
:103100004721FEF7C1FD2068FF224921FEF7BCFDE3
:10311000206800224A21FEF7B7FD20680022FF2127
:10312000FEF7B2FD20680A227A21FEF7ADFD206885
:1031300000227B21FEF7A8FD206821227821FEF7DE
:10314000A3FD20680122FF21FEF79EFD20683422A6
:103150002321FEF799FD206800224221FEF794FD0D
:103160002068FF224421FEF78FFD2068262245219A
:10317000FEF78AFD206805224621FEF785FD4022E4
:1031800011462068FEF780FD206806220E21FEF71A
:103190007BFD20681A222021FEF776FD2068402260
:1031A0004321FEF771FD20680022FF21FEF76CFD30
:1031B000206803223421FEF767FD20684422352170
:1031C000FEF762FD20680122FF21FEF75DFD206809
:1031D00004223121FEF758FD206809224B21FEF719
:1031E00053FD206805224C21FEF74EFD2068042285
:1031F0004D21FEF749FD20680022FF21FEF744FD26
:10320000206800224421FEF73FFD2068202245214E
:10321000FEF73AFD206808224721FEF735FD2068B9
:1032200028224821FEF730FD206800226721FEF7A2
:103230002BFD206804227021FEF726FD2068012264
:103240007121FEF721FD2068FE227221FEF71CFD90
:10325000206800227621FEF717FD206800227721E2
:10326000FEF712FD20680122FF21FEF70DFD206808
:1032700001220D21FEF708FD20680022FF21FEF744
:1032800003FD206801228021FEF7FEFC2068F82261
:103290000121FEF7F9FC20680122FF21FEF7F4FC72
:1032A000206801228E21FEF7EFFC20680122002118
:1032B000FEF7EAFC20680022FF21FEF7E5FC20680B
:1032C00000228021FEF7E0FC042220680A21FEF79C
:1032D000DBFC256884212846FFF785FC842100F06B
:1032E000EF022846FEF7D0FC012220680B21FEF7F2
:1032F000CBFC256801A92846FFF7B2FC05AA01A965
:103300002846FFF7C2FC9DF80430002B00F01C811A
:10331000089D05F684559DF80630002B00F01781B6
:10332000089B03F2B22305EB43059DF8073023B158
:10333000BDF8243003F525731D449DF8083023B1F2
:10334000BDF8263003F226231D44E822206847F802
:10335000CC5C0121FEF798FC206829464AF032FE39
:10336000012220681146FEF78FFC20684021FFF7FC
:1033700049FC002800F0DF80206801210222FEF7CE
:1033800083FC20680021FFF73DFC002800F0D3807B
:103390002068DFF8D491E8220121FEF775FC20684F
:1033A00020224421FEF7BFFC256801A92846FFF72B
:1033B00057FC05AA01A92846FFF767FC50225721B0
:1033C0002846FEF761FC082256212846FEF75CFCE1
:1033D000082250212846FEF757FCBDF824004FF480
:1033E0007A7A48F20E660AFB0060B0FBF9F080B210
:1033F000FEF7ECF9512102462846FEF794FC089BA3
:103400000AFB0366574B9E429DBFB6FBF9F202F1E1
:10341000FF32D2B2FF2246212846FEF735FC57F88C
:10342000CC1C28464AF0CEFD01212846FFF7DBFBE5
:103430000222064601212846FEF726FC00212846E6
:10344000FFF7E0FB324601212846FEF71DFC246809
:1034500001A92046FFF704FC05AA01A92046FFF7B1
:1034600014FC482211462046FEF70EFC0822472194
:103470002046FEF709FC032232212046FEF704FC19
:10348000072230212046FEF7FFFB0122FF212046C4
:10349000FEF7FAFB202230212046FEF7F5FB002242
:1034A000FF212046FEF7F0FB062220467021FEF7A2
:1034B000EBFBBDF826304FF47A7246F6440002FB6F
:1034C00003004DF28803B0FBF3F09DF8073080B2A3
:1034D0001BB1BDF81A30184480B2FEF777F971219C
:1034E00002462046FEF71FFC57F8CC1C20464AF047
:1034F00069FD01212046FFF776FB022205460121E6
:103500002046FEF7C1FB00212046FFF77BFB2A4641
:1035100001212046FEF7B8FB642347F8D43C012381
:1035200088F8FC3007E0D9F800309BB29B1BB3F55C
:10353000FA7F7FF6ABAC0AB0BDE8F0870B41DB0742
:1035400044BF0132D2B21AE540F63635E3E69DF8C3
:103550000530002B3FF4E9AE089B03F525731D44AD
:10356000E3E600BF1B280D011C0C0100F8B53B4F22
:1035700097F8FC300446002B37D0394D15F8C86C4D
:10358000012E33D0022E4FD07EBB00680122802155
:10359000FEF77AFB20680122FF21FEF775FB206809
:1035A00032463146FEF770FB15F8D02C2068912189
:1035B000FEF76AFB206801223146FEF765FB2068B2
:1035C0003246FF21FEF760FB206832468021FEF77D
:1035D0005BFB206801223146FEF756FB214B1B683E
:1035E00045F8D83C012305F8C83CF8BD0068002127
:1035F000FFF7F9FAC20711D555F8D42C002AF4D0F8
:10360000184B55F8D81C1B689BB25B1A9A42ECD237
:10361000154B4FF0FF325A600023E4E7114B1B6853
:1036200045F8D83C0223DEE700681321FFF7DBFAF8
:103630004307E1D01E212068FEF70AFF012206465B
:103640000B212068FEF720FB0A23B6FBF3F6064B9E
:10365000B6B25E60012387F8FD30DDE7A05F002091
:1036600090810020042A0020F810002010B5EFF30C
:103670001181102383F312884FF0E023C9B29C69B3
:103680001A6912F4803F0D4A1EBF0120C2F8040FD0
:103690009C690B4B1868D2F8043F81F31188D2F86B
:1036A000081F4FF47A72034402FB01F0001BB0FBC9
:1036B000F1F00021E3FB020110BD00BF9870002073
:1036C000042A0020124B5B68C3F3080330B4EBB943
:1036D000EFF31183D3B90F490F4B4FF0E0250A6880
:1036E000AC6908688242FAD1D3F8000F8442F6D858
:1036F000D3F8081F4FF47A7303FB01F0001BB0FBF3
:10370000F1F00021E2FB030130BC704730BCADE7B3
:1037100000ED00E0042A00209870002010B5074C4E
:1037200014F8BF0C40B1FFF7CDFF54F8B83CC01AF5
:10373000C0F5FA5020EAE07010BD00BF9081002073
:1037400010B5044630B1036823B1DB6813B1BDE89E
:1037500010401847FFF7B6FFD4E90423904299417F
:1037600034BF0120002010BDF8B506460D46FFF716
:10377000A9FF04460F46FFF7A5FF021B61EB0703F5
:10378000B242AB41F7D3F8BD38B50D460446FFF75A
:10379000C5FF011E02DDC917FFF7E6FF064B2068D3
:1037A000002203F8BF2C492113F8BE3C2A46FEF73D
:1037B0002BFB012038BD00BF908100202DE9F34193
:1037C000384C54F8B03CC0F8363034F8AC3C438741
:1037D00014F8C03C012B064600F13608A4F1B007EE
:1037E0000CD0022B26D0A3BB0122022149F027FBDB
:1037F000012304F8C03C14F8AA5C10E0FFF78EFF28
:1038000014F8AA5C58B969463046FFF7BDFF9DF829
:10381000003008B19B0706D1002304F8C03C2846BD
:1038200002B0BDE8F08107220321304649F007FBD2
:103830000223F2E7FFF772FF0028DCD16946304629
:10384000FFF7A2FF9DF80630054610B113F00802FD
:1038500005D0002504F8C05C04F8AA5CDFE734F961
:10386000A81C6846FBF7B6FB404234F9A61CF0865C
:103870000DF10200FBF7AEFB34F9A41C308701A860
:10388000FBF7A8FBD6F8363044F8B03C40427087CE
:10389000B8F80430BB80012304F8C02C04F8AA3C1B
:1038A000BDE700BF9081002010B50446013C00D266
:1038B00010BD4FF47A700021FFF756FFF6E738B5D8
:1038C0000568044600212846FCF77CF8B62214213E
:1038D0002846FEF78BF86420FFF7E6FF81221021CF
:1038E0002068FEF783F80120FFF7DEFF152120682E
:1038F0008022FEF77BF80120FFF7D6FF2068032126
:10390000BDE83840FCF75EB838B5056804460021CC
:103910002846FCF757F8B6227E212846FEF766F8BF
:103920006420FFF7C1FF00227C212068FEF75EF8CB
:103930006420FFF7B9FF04227D212068FEF756F8C6
:103940006420FFF7B1FF8C2240212068FEF74EF87B
:103950000120FFF7A9FF022241212068FEF746F867
:103960000120FFF7A1FF20680221FCF72BF84FF49C
:103970000063A38138BD10B504464069FCF700FC24
:103980000120FFF791FF6069FCF7F5FBBDE81040EF
:103990000A2089E773B50468B6227E2105462046D1
:1039A000FEF724F86420FFF77FFF02212046FCF792
:1039B00009F82046FFF7DFFF00227C212046FEF7B2
:1039C00015F80120FFF770FF002259212046FEF76D
:1039D0000DF80120FFF768FF5E238DF8073094F99A
:1039E0001030142253433D4AD658A3689A0702D494
:1039F00060694AF0DBFC01230DF10702002130462B
:103A00004CF0E8FC4FF4A473354A002130464CF0EA
:103A1000E1FCA3689B0702D42046FDF7B7FF0A200C
:103A2000FFF742FF012259212046FDF7DFFF012069
:103A3000FFF73AFF8C2240212046FDF7D7FF0120F7
:103A4000FFF732FF032241212046FDF7CFFF01207F
:103A5000FFF72AFF234EA96B234A95F83500B6FBE2
:103A6000F1F1032389B2FBF743FC4388B6FBF3F67D
:103A70002E640279422142F0C0022046FDF7B6FFD3
:103A80000120FFF711FF082243212046FDF7AEFF7A
:103A90000120FFF709FF042258212046FDF7A6FF69
:103AA0000120FFF701FF0A2253212046FDF79EFF68
:103AB0000120FFF7F9FE00227C212046FDF796FF4A
:103AC0000120FFF7F1FE06227D212046FDF78EFF43
:103AD000012002B0BDE87040E6E600BFB40000205F
:103AE0002B4C060840420F00744D0608F8B5816B58
:103AF0000468294A294FB7FBF1F10546062389B22C
:103B000090F83500FBF7F4FB00214388B7FBF3F78F
:103B100006462F642046FBF755FF80226B21204686
:103B2000FDF764FF6420FFF7BFFE032268212046F3
:103B3000FDF75CFF6420FFF7B7FE01226B212046F2
:103B4000FDF754FF0F20FFF7AFFE18221B21204680
:103B5000FDF74CFF0F20FFF7A7FE18221C2120467F
:103B6000FDF744FF0F20FFF79FFE32791A21204610
:103B7000FDF73CFF0F20FFF797FE727919212046D1
:103B8000FDF734FF6420FFF78FFE20460321BDE8D8
:103B9000F840FBF717BF00BF864D060840420F00F4
:103BA0002DE9F74305230468816B6C4A6C4EB6FB24
:103BB000F1F1054689B290F83500FBF799FB002139
:103BC0004388B6FBF3F607462E642046FBF7FAFE61
:103BD000002276212046FDF709FF624E0F224E217A
:103BE0002046FDF703FF0F20FFF75EFE16F8A28CBC
:103BF00008F1FF335A425A417B7903F00F034F21FA
:103C00004FEA4219204643EA4212FDF7EFFE0F2029
:103C1000FFF74AFE7A7902F00F0249EA02025021C8
:103C20002046FDF7E3FE0F20FFF73EFE5221FF2264
:103C30002046FDF7DBFE0F20FFF736FE95F8351026
:103C400007293FD04046FBF79FFB0546012276211E
:103C50002046FDF7CBFEAA780C212046FDF7C6FED4
:103C60002A790D212046FDF7C1FEAA79AB88120101
:103C700042EA1322D2B20E212046FDF7B7FE4FF4DE
:103C8000807116F8A20CFBF77FFB05460222762115
:103C90002046FDF7ABFEAA78520002F0FE02032197
:103CA0002046FDF7A3FE2A7904212046FDF79EFE5B
:103CB000AA79AB88120142EA1322D2B2052120462A
:103CC000FDF794FE002276212046FDF78FFE0322A9
:103CD00014212046FDF78AFE0F20FFF7E5FD0022A4
:103CE00063212046FDF782FE6420FFF7DDFD0822F8
:103CF00065212046FDF77AFE0DF10702642120467A
:103D0000FEF700FE9DF8072022F0100242F060024C
:103D1000642120468DF80720FDF768FE0F20FFF78D
:103D2000C3FD0DF106024D212046FEF7EBFD9DF887
:103D3000062002F03F0242F040024D2120468DF85D
:103D40000620FDF753FE0F20FFF7AEFD03212046AE
:103D5000FBF738FE03B0BDE8F08300BFAA4D0608AC
:103D600040420F0090810020F8B5816B04682D4A15
:103D70002D4FB7FBF1F10546062389B290F83500C7
:103D8000FBF7B6FA00214388B7FBF3F706462F642A
:103D90002046FBF717FE80226B212046FDF726FE0A
:103DA0006420FFF781FD072268212046FDF71EFEF3
:103DB0006420FFF779FD00226B212046FDF716FEF7
:103DC0006420FFF771FD01226B212046FDF70EFEF6
:103DD0000F20FFF769FD18221B212046FDF706FE84
:103DE0000F20FFF761FD18221C212046FDF7FEFD84
:103DF0000F20FFF759FD32791A212046FDF7F6FD15
:103E00000F20FFF751FD727919212046FDF7EEFDD5
:103E10006420FFF749FD20460321BDE8F840FBF789
:103E2000D1BD00BF864D060840420F009CE710B58B
:103E30007822044600210068FDF7D8FD0520FFF731
:103E400033FD202201212068FDF7D0FD0520FFF77A
:103E50002BFD002202212068FDF7C8FD6420FFF73A
:103E600023FD012010BD10B5072204460A21006879
:103E7000FDF7BCFD0520FFF717FD24224121206836
:103E8000FDF7B4FD0520FFF70FFDC0224221206899
:103E9000FDF7ACFD0520FFF707FD012010BD10B5B3
:103EA0000122044610210068FDF7A0FD48B114204E
:103EB000FFF7FAFC2068A022BDE810401121FDF7B1
:103EC00095BD10BD13B5044600210068FBF77AFDCF
:103ED0000021204648F09AFF1420FFF7E5FC0F214F
:103EE000204648F093FF0A20FFF7DEFC01AA0323D7
:103EF0001021204648F0B8F80A20FFF7D5FC9DF8BD
:103F00000420174B803223F8A82C9DF8052080321E
:103F100023F8A62C9DF8062000218032204623F8A5
:103F2000A42C48F073FF0A20FFF7BEFC0DF103023A
:103F300001230221204648F097F801230DF10302E6
:103F40000921204648F090F82046122148F05EFFF3
:103F500020680321FBF736FD012002B010BD00BF31
:103F60009081002008B5006801220921FDF73EFD7F
:103F7000BDE80840642097E480B506460A25012183
:103F80000846FCF7B9FC00210846FCF7B5FC771C95
:103F90004FF03208052457EA04030BD14FF47A702E
:103FA000FFF782FC013DEAD101210846F7F792F8BC
:103FB000FDF796FC0120FCF78DFC0020FCF78AFC45
:103FC0000120FDF748FC4046FFF76EFC0120FCF79E
:103FD00081FC0020FCF77EFCFDF73DFC4046FFF72E
:103FE00063FC44B1013CD6D14FF4FA70FFF75CFC9E
:103FF0004FF0FA08CFE7013FCDE737B50568044633
:1040000000212846FBF7DEFC15227E212846FDF71D
:10401000EDFC6420FFF748FC11227E212068FDF7AB
:10402000E5FC0520FFF740FC20680DF107020321A5
:10403000FEF768FC9DF8073003F03C03142B02D018
:104040000620FFF799FF0C2240212068244DFDF740
:10405000CDFC0120FFF728FCA16B224A94F8350023
:10406000B5FBF1F1092389B2FBF742F94388B5FBAF
:10407000F3F52564027920684221FDF7B7FC0120A1
:10408000FFF712FC082241212068FDF7AFFC012058
:10409000FFF70AFC002243212068FDF7A7FC01205E
:1040A000FFF702FC102251212068FDF79FFC012040
:1040B000FFF7FAFB0A2253212068FDF797FC012045
:1040C000FFF7F2FB802256212068FDF78FFC0120CC
:1040D000FFF7EAFB20680321FBF774FC03B030BD57
:1040E00040420F00C84D0608F0B5816B0568514A83
:1040F000514FB7FBF1F185B00446062389B290F821
:104100003500FBF7F5F800214388B7FBF3F70646C7
:1041100027642846FBF756FC80226B212846FDF7D2
:1041200065FC9620FFF7C0FB032268212846FDF7B7
:104130005DFC9620FFF7B8FB03226B212846FDF7B4
:1041400055FC0F200021FFF70FFB10226A212846A3
:10415000FDF74CFC0F200021FFF706FB00226C212D
:104160002846FDF743FC0F200021FFF7FDFA727986
:1041700019212846FDF73AFC0F200021FFF7F4FA39
:1041800018221B212846FDF731FC0F200021FFF7E4
:10419000EBFA18221C212846FDF728FC0F200021ED
:1041A000FFF7E2FA32791A212846FDF71FFC0120B9
:1041B0000021FFF7D9FA03212846FBF703FC20680A
:1041C000062302AA4321FDF71FFED0B1BDF8083037
:1041D000DBBA07EE903ABDF80A30F8EEE77ADBBAC0
:1041E000C4ED077A07EE903ABDF80C30F8EEE77AA6
:1041F000DBBAC4ED087A07EE903AF8EEE77AC4ED40
:10420000097AD4ED087AFDEEE77ACDED017A9DF9D1
:10421000043001330CD1D4ED077AFDEEE77ACDED11
:10422000017A9DF90430013302D10620FFF7A4FE84
:1042300005B0F0BD864D060840420F0018B1036876
:104240005B6803B11847FF20704718B103689B688B
:1042500003B118470020704770B450B106798E4200
:1042600007D34579954204D30368DB680BB170BC72
:10427000184770BC704710B440B184798C4205D3A4
:1042800003681B6913B15DF8044B18475DF8044BD4
:10429000704718B103685B6903B11847704718B1DC
:1042A00003681B6A03B118470020704730B50A46FF
:1042B00058B1041D00F1140320686168154603C558
:1042C00008349C422A46F7D1012030BD10B50C4677
:1042D00070B92D2300202375094B2061C4E900002B
:1042E000C4E90200C4E90633302384F8203010BD4D
:1042F0000368DB6A002BECD098470028E9D0F6E78A
:10430000CD3B070838B5054D441E14F8011F01B90F
:1043100038BD55F8A00CFBF718FBF6E7908100209C
:1043200008B50648FFF7EEFF054B33F89C0C18B1B3
:10433000BDE80840FFF7B8BA08BD00BFD748070876
:104340009081002008B5FFF7DDFFBDE80840E7E7F2
:1043500010B504460948FFF7D5FF2046FFF7D2FF06
:10436000074B13F89A2C3AB1012203F8992C13F851
:10437000982C013203F8982C10BD00BF13F00608EA
:104380009081002010B504460348FFF7BBFF20468C
:10439000BDE81040D6E700BF1FF0060810B5074C77
:1043A00002460B4654F8A00C05494CF093F854F81B
:1043B000A00CFBF7BEFABDE81040B1E790810020E9
:1043C0006BF9000820B10078B0FA80F0400970471E
:1043D00001207047034B9A780021101A997018BF7A
:1043E00001207047C0B8002010B5114B014603F101
:1043F0001C0253F8044B41F8044B9342F9D11B883B
:104400000B800B4900F11E0351F8044B43F8044B99
:104410009142F9D111881980054B3C3053F8041BA7
:1044200040F8041B9342F9D11B88038010BD00BFE4
:10443000044E0608144A92F8301092F831300B43BB
:1044400092F83B100B4392F829100B4392F82A1074
:104450000B4392F82B100B4392F82C100B4392F85D
:1044600036100B4392F842100B4392F84B100B435B
:1044700092F857100B4305D192F86900013818BF24
:104480000120704701207047C0B800200FB413B559
:10449000084C0949206804AB53F8042B01934CF0F5
:1044A00019F82068FBF745FA02B0BDE8104004B0E7
:1044B000704700BFF08000206BF9000870B50D4E0A
:1044C0000D4604460C48FFF71DFF2B460B4930688C
:1044D00022464BF0FFFF3068FBF72BFA084B1B78A6
:1044E00033B1084B01221A70074A13780133137055
:1044F00070BD00BFF080002013F006086BF90008C3
:10450000F6800020F7800020F88000200FB407B567
:1045100004A951F8040B0191FFF7D0FFFFF700FF4A
:1045200003B05DF804EB04B070470148EEE700BF4C
:1045300024F0060813460A4601460148E6E700BF94
:1045400030F0060838B5064D002455F83400013423
:10455000FFF7D8FEFFF7E4FE362CF6D138BD00BFDA
:10456000244E060870B5C379164603F007028CB0D6
:104570000446062A4FD8DFE802F0041417191C1E5F
:1045800049000D7813F0C00347D0402B3CD1294699
:10459000204617F025FE002859D00CB0BDE8704029
:1045A00074E791F90050EDE70D88EBE7B1F90050A1
:1045B000E8E70D68E6E791ED000A6846F9F752FF73
:1045C00001462848FFF762FFF6B1E3793F2B1BD87D
:1045D000204617F05FFD00EE100A6846B8EEC00AEC
:1045E000F9F740FF01462048FFF750FF204617F03B
:1045F00061FD00EE100A6846B8EE400AF9F732FF96
:1046000001461948FFF742FF0CB070BD15480CB0C9
:10461000BDE870403AE70025B4E7042A0CBF134810
:1046200013482946FFF732FF002EEDD0E3793F2BE8
:10463000EAD8204617F02EFD0546204617F03AFD31
:1046400002460C4829460CB0BDE870401EE769469A
:10465000204617F01BFC08486A462946FFF756FF1C
:10466000D2E700BF1CF706081BF7060821F606086C
:1046700052260708C04B07084DF0060838B50D460E
:10468000044617F0FBFC2A4601462046BDE83840A8
:1046900068E72DE9F04F8FB001F02003814688468E
:1046A00000270093384617F069FC484B0446186809
:1046B000FBF73FF994F807B00BF038034B454AD1AC
:1046C000204617F071FCFAF723F98568204617F0A9
:1046D00097FC82462E18204617F0D0FC0BF00702FC
:1046E0000146062A6AD8DFE802F0043E43474C50F0
:1046F0005C0015F80A200978531A5A425A41009B67
:1047000003B142BB02A92046019217F0BFFB18F08B
:10471000400F15D0019A9AB92D4802A9FFF7B6FEAD
:104720002C4902A84CF0CCF8002849D115F80A30E1
:10473000202B45D128483146FFF7A8FEFFF7F0FDB2
:10474000264802A9FFF7A2FE002231462046FFF7C5
:1047500009FFFFF7E5FD013740F292239F42A1D107
:104760000FB0BDE8F08F15F90A2091F90010C3E7EA
:1047700035F80A200988BFE735F90A20B1F9001099
:10478000BAE755F80A200968B6E796ED007AD1ED48
:10479000007AB4EE677AF1EE10FA0CBF0122002223
:1047A000ADE72046019117F085FC0199421C304687
:1047B0004FF0C4FDB0FA80F25209A0E700229EE754
:1047C000002231462046FFF7CDFEB7E7F0800020FB
:1047D0006AF00608834B0708DBF506086BF006084D
:1047E00008B520214FF07DFD0346184623B102781D
:1047F000202A03F10103F8D008BD70B50D46144618
:10480000FFF7EEFF0646A0B1F9F71CFF40F63403B0
:104810009842A8BF1846B0F5617FB8BF4FF46170E9
:10482000A0F561731922B3FBF2F32B7023780133E7
:1048300023703046FFF7D4FF0646A0B1F9F702FF18
:1048400040F634039842A8BF1846B0F5617FB8BF60
:104850004FF46170A0F561731922B3FBF2F36B7032
:10486000237801332370304670BD2DE9F04F87B0B7
:104870000346FFF7A7FD054618B107B0BDE8F04FA6
:1048800053E65E49DFF8A8A1DFF870B105AA184623
:104890004FF0A1FC2F4681462C46A8464FF0FF362C
:1048A000B9F1000F12D14FFA86F9484621F0EEF81F
:1048B00010B14568002D79D1B8F1000F55D150489D
:1048C0003146F9F7C6F807B0BDE8F08F032D07D8D9
:1048D000DFE805F0020E132D4846F9F7B3FE064651
:1048E00005AA594600204FF076FC01358146D7E7EE
:1048F0004846F9F7A7FE8046F2E7424948464FF09E
:1049000052FD20B9404948464FF04DFD08B144F0F2
:104910000104514648464FF046FD28B93B494846F8
:104920004FF041FD0028DBD044F00204D8E74846B0
:104930004BF0D0FF032816D199F80020382A12D165
:1049400099F80120452A0CD04E2A0CD1002299F862
:104950000230312B03D0322B05D142F00202174333
:10496000BEE70422F3E7FF22F9E7002C08BF032487
:104970000023E4B2CDE9008402971A46194648465E
:1049800021F044FA054610B92148314699E72148FB
:1049900042463146F9F75DF831461F48F9F759F8B4
:1049A0001E4B2946D86F46F0F1FF8CE71C48314674
:1049B000F9F74FF85CB16979A14208D0194822464D
:1049C000F9F747F82B68E1B29B69284698475FB131
:1049D000A979B94208D014483A46F9F73AF82B6851
:1049E0003946DB6928469847EB6A002BD4D00F483C
:1049F000F9F72FF80023EB62CEE700BFA4420708C7
:104A000078F00608E2040708752C07081E08070856
:104A1000A0F00608BFF006084DF10608C0B8002057
:104A2000DCF00608F4F0060814F1060837F1060871
:104A300075F0060870B5054608460E464BF04AFF6D
:104A40003146044602462846F9F7A4F960B92B5DC1
:104A5000A3F13002092A06D923F02003413B192B88
:104A600001D90134281970BD0020FCE72DE9F04F71
:104A700085B00546FFF7A6FC044630B100210120B1
:104A800005B0BDE8F04F47F057B885492846F9F71B
:104A90009BF920B905B0BDE8F04F3EF0D9BB814984
:104AA0002846F9F791F928B9012005B0BDE8F04F83
:104AB0003EF02EBD7C492846F9F786F990BB7B4B2A
:104AC00093F92B2E83F8240E194693F8D654012D12
:104AD00009D0033D052D06D90CB181F82B2E05B068
:104AE000BDE8F04F21E593F8D754A52D00F1010062
:104AF00013D1012A0ED181F8242E6D4A81F8250E9A
:104B0000002382F8803081F82B3E05B0BDE8F04FDD
:104B10003EF046BD013A52B20124782803F1140355
:104B2000D3D1D9E72846F9F78DFD614B93F9803051
:104B3000009303FA80F6772E834600F2A78028467A
:104B4000FFF74EFE0746002800F08C80F9F77AFD4B
:104B50000124C5B23846FFF743FE0746002800F09F
:104B60008480F9F76FFD01340190E4B23846FFF715
:104B700037FE804600287AD0F9F764FD01340746F5
:104B8000E4B24046FFF72CFE8146002871D0F9F7C9
:104B900059FD01340290E4B24846FFF721FE8246F7
:104BA000002868D0F9F74EFD01340FFA80F9E4B21D
:104BB0005046FFF715FE824600285ED0F9F742FD09
:104BC00001340FFA80F8E4B25046FFF709FE0028DE
:104BD00055D00390F9F736FD039A0FFA80FA104684
:104BE000FFF7FEFD0346002857D004F0FD04F9F757
:104BF00029FD042C7FF473AFC3B2012D03D9EA1E43
:104C0000052A3FF66CAF23B1A52B02D0482B7FF4C9
:104C100066AF26480EB980F82B6E142202FB0602FE
:104C20000199C2F8C414A52B029982F8D654C2F88F
:104C3000C874C2F8CC14A2F8D094A2F8D284A2F816
:104C4000D4A482F8D7340AD1009B194A01335B44BB
:104C500082F8803090F82B3E013380F82B3E05B06F
:104C6000BDE8F08F0446054674E701907EE70746ED
:104C700087E7029090E781469AE78046A4E75FFACB
:104C800088F382468046062CB7D028E70948772269
:104C9000214605B0BDE8F04F4CE40134E4B2F2E740
:104CA0007BF1060881F10608370307081861002028
:104CB000C0B8002086F106082DE9F3473549DFF832
:104CC000D49001AA4FF087FA4FF0000A4FF0FF3559
:104CD000564654465746A84678B9BAF1040F3DD017
:104CE000BAF1050F44D0BAF1030F13D02A492B466D
:104CF0004246012046F0ACFF0EE0BAF1040F09D89D
:104D0000DFE80AF0030D12171C00F9F79BFC804640
:104D100003281BD9FFF709FC02B0BDE8F087F9F7BB
:104D200091FC0546A828F4E7F9F78CFC07463F28D4
:104D3000EFE7F9F787FC04463F28EAE70378482BBA
:104D400003D0562BE6D1012600E0002601AA4946F1
:104D500000200AF1010A4FF03EFABDE70F4BA922ED
:104D600002FB085203EB4203B3F88260C6F34036FD
:104D7000A92303FB0855A401084B04F47C6407F045
:104D80003F0703EB45033C4344EA4634A3F8824023
:104D9000C2E700BFA442070842B90020C0B8002003
:104DA00008B504460648FFF7ADFA064B1868FAF74F
:104DB000C0FD054BD86F21F075F9204605F092FB38
:104DC0008FF10608F0800020C0B80020034808B525
:104DD000FFF798FA0120FFF7E3FF00BF9BF10608F9
:104DE00008B50C4B93F8CC25012A12D193F8D13594
:104DF000062B0AD00A2B04D00748BDE80840FFF76D
:104E000081BA27F04FFA0548F7E726F027F804485B
:104E1000F3E708BDC0B80020B4F10608C3F10608E6
:104E2000DDF1060808B50A48FFF78CFA094B186847
:104E3000FAF77FFD084B002483F8F045C3F83046AD
:104E4000064B1C7018F0DCFD2046FFF7A9FF00BFE1
:104E5000F6F10608F0800020C0B80020B9730020E9
:104E600038B5224CD4F83C0600283ED0E56F21F03E
:104E700019F9284621F016F9D4F83C0641798B0738
:104E800004D4036841F002019B6998470021084659
:104E9000FBF732FD00210120FBF72EFDD4F83C0684
:104EA000FCF7A5FC78B101210020FBF725FDD4F823
:104EB0003C06FCF7BDFC01462846FCF795FC0021AA
:104EC0000846FBF719FD2846FCF791FC0028E5D0C1
:104ED00001210846FBF710FD2846FCF7A9FC014616
:104EE000D4F83C06FCF780FCD4E738BDC0B80020FD
:104EF00070B51D4990B0052204464FF0FFF970B916
:104F00001A4A13782BB901211170194A1370194AE2
:104F10001370194810B0BDE87040FFF713BA174975
:104F2000032220464FF0EAF9C0B9104E104D3378F5
:104F3000104C7BB12B786BB12278114901A8F8F79E
:104F4000A5FD01A8FFF7E2FA002333702B70237050
:104F500010B070BD0B48FFF7F5F9F5E70A4810B03F
:104F6000BDE87040FFF7D2BAE4000708F6800020E1
:104F7000F7800020F880002020F206085803070878
:104F800036F2060879F206088DF2060870B5124E60
:104F9000337890B0A3B1114D2B788BB1104C1149DF
:104FA000227801A8F8F772FD01A8FFF7AFFA0E48C2
:104FB000FFF7ACFA002333702B70237010B070BD74
:104FC0000A48FFF79FF926F007FFF9F79DFB26F047
:104FD0000DFF0020FFF7E4FEF6800020F7800020A0
:104FE000F880002036F206089CF20608BAF206089D
:104FF00010B5F6F71FFF124CD0B11248FFF7C2F9F7
:105000001148FFF77FF92068FAF793FC4FF47A70A4
:10501000FEF74AFC0D4BD86F21F044F80C4B187882
:10502000FCF740F802210120F6F754F8FCF758FC91
:105030000848FFF767F92068BDE81040FAF779BC27
:10504000F0800020C1F206088FF10608C0B80020E9
:10505000846F0120E1F20608A0F2DC50164BB0F597
:10506000FA7FA8BF4FF4FA70984210B5B8BF18463F
:105070000C46114646F05EFE00B207EE900A9FED28
:105080000F7AF8EEE77AE4B287EE870AFBEE096A58
:10509000E0EE006A07EE904A9FED097AF8EE677A33
:1050A000A7EEA67AF3EE097A20EE070A80EE270A29
:1050B0004DF012F800B210BD0CFEFFFF0000C84218
:1050C00000401C452DE9F043DFF8F491764CD9F807
:1050D0000030D3F82880754B1B6813F0100F87B091
:1050E00040F0A5802378002B00F0A180704E06F2DE
:1050F0006465D6F86C3628469847002800F09780FB
:1051000096F8C336002B43D1022384F82030B6F939
:10511000C43607EE903AB6F9C636F8EEE77AC5ED32
:105120000A7A07EE903AB6F9C836F8EEE77AC5ED96
:105130000B7A07EE903AF8EEE77AC5ED0C7A5D4906
:1051400003AAA1F10C0047F011FB03A996F8A826C9
:10515000084627F079FD03A827F038FD95ED060AEB
:105160005549554D03A847F00EFB05F17807002679
:10517000B5EC010AD4F8003585ED020A38469847A7
:105180000136032E05ED010A07F5C077F0D14EE098
:1051900094F82030012BD2D1EB6903932B6A04934E
:1051A00003A96B6A059304F12000F8F7EFFA94F86D
:1051B0002030012B4FF0000771D0022B68D00397ED
:1051C00004970597DDED037A9DED047ADDED056A20
:1051D000C5ED0A7A85ED0B7AC5ED0C6AFDEEE77A2E
:1051E000BDEEC77AFDEEE66A17EE903A17EE102A8A
:1051F00016EE901A1BB212B209B2A6F8C436A6F87F
:10520000C626A6F8C8160120CDE9002104212B4AA4
:10521000F8F752FCD9F8003000200021C3E90C0156
:10522000C3E91001C3E90E01A760E7602761D4F864
:1052300004355B0629D51E4D95F81C372BB34FEA74
:10524000E876314640464CF0BBF805F5DE6307EEE4
:10525000900AD4ED026A93ED107AD5F83827D5F884
:105260003C17A7EEA67A12EB080246EB0106D4ED36
:10527000036A83ED107A93ED117AC5F83827A7EE0B
:10528000A67AC5F83C6783ED117A07B0BDE8F083D4
:10529000A36B0393236D0493A36E059392E7AF6210
:1052A000EF622F63C0E700BF906F0120E06E012026
:1052B000C0B800204CBF0020986F012010F30608F2
:1052C000806F01200CB4830607B500D551B904984E
:1052D00005A90191FFF762F8012003B05DF804EB26
:1052E00002B070470020F8E7024B01461868FAF751
:1052F0002CBB00BFF080002030B5274885B0FFF7F9
:1053000001F8F6F7D5FA28B9244805B0BDE83040D1
:10531000FFF718B8F6F798FD08B92148F5E7F6F752
:10532000C9FD0268037D81790446407C0290207C9F
:105330000190608A009052081A48FFF7A7F8E51D0F
:105340000C3415F8010BFFF7CFFFA542F9D1164C2D
:105350001648FEF7D7FF6378022B06D007D9032B38
:1053600010D11348FEF7CEFF0CE01248FAE704F51F
:1053700080541148FEF7C6FF94F8B431022B06D0D2
:10538000032B06D005B0BDE83040FEF7C9BF0B487F
:10539000E8E70B48E6E700BF37F3060841F30608E5
:1053A0004FF306085EF30608784D00208CF30608DC
:1053B0009CF30608A2F30608AFF30608B5F3060847
:1053C000CEF306080CB407B510F0400009D069B957
:1053D0002320FFF789FF049805A90191FEF7DEFF5E
:1053E000012003B05DF804EB02B070470020F8E73D
:1053F0002DE9F04F834689B090460C4616460027AB
:105400004FF0190A4FF46179B8F1000F4BD03078A2
:1054100025787178B378F278854242D165788D42EB
:105420003FD1A5789D423CD1E578A5EB020CDCF19B
:10543000000545EB0C05CDE90632059115F0A8F8FD
:10544000079A069B059901911AFB02921AFB039396
:105450000392029343790093144A3B4629465846E7
:10546000FFF7B0FF207815F093F8E3780F4A1AFBA6
:1054700003930393A3781AFB039302936378019336
:105480004379009329463B4658460137FFF71AFFF8
:10549000282F04F1040406F10406B5D109B0BDE8D3
:1054A000F08F0025C7E74546DCE700BFE0F30608BC
:1054B000F7B50746FEF786FF044630B12E490022B5
:1054C000012003B0BDE8F04092E73846F9F7BAF89A
:1054D0002728054648DC8600781C8DF80740FFF732
:1054E0007FF9074690B1F9F7ADF8031E0EDB234AAA
:1054F0002146DBB202F5E87404EBC10CC8009CF84D
:1055000005C09C4525D001313D29F5D13846FFF72E
:1055100067F9044660B1F9F795F81D2808D8184BCB
:10552000334483F849079DF8073001338DF807307D
:10553000114FB11C0DF1070239442046FFF75DF908
:105540009DF80730042B02D0002347F8253003B024
:10555000F0BD0B4B0244334492F8D42183F8482722
:1055600001238DF80730D1E706482722214603B0F2
:10557000BDE8F040FEF7DEBF08C00020044E06087C
:10558000C0B80020F6F406082DE9F04F3F4FDFF8D1
:1055900004A189B0814690460C46164602F1300BB4
:1055A00094F9045000230C22394802FB03F10956F8
:1055B000A94266D00133042BF6D10C36B34504F171
:1055C0000C04EDD109B0BDE8F08F96F90430D6F89F
:1055D00000E07279B179307A96F807C007939D425E
:1055E0004DD1256875454AD16579954247D1A57950
:1055F0008D4244D1257A854241D1E579A5EB0C0352
:105600005D425D4107EB820207EB8C0C07EB8000EB
:1056100007EB8101D2F8B823DCF8B833D0F8B8032F
:10562000D1F8B8130493CDE900E203900291079BEF
:10563000524629464846FFF7C5FEE27994F9043000
:1056400007EB82022946D2F8B8230492227A07EBAC
:1056500082024846D2F8B8230392A27907EB82026D
:10566000D2F8B8230292627907EB8202D2F8B8230B
:105670000192226800925246FFF724FE9DE7002522
:10568000C0E7B8F1000FA0D14546D6E7044E0608A2
:10569000A8C00020F3F306082DE9FF410346FEF7FA
:1056A00091FE30B145490022012004B0BDE8F0412F
:1056B0006AE718465E1CF8F7C5FF044640B220F0C2
:1056C00061FB054630B93E48214604B0BDE8F041D3
:1056D000FEF71CBF0068696801AB03C3A8681860C7
:1056E0003046FFF77DF80446002853D003782B2B73
:1056F00005D02D2B43D0F8F7A5FF019009E0013428
:105700002046F8F79FFF012303FA00F0019B0343B3
:10571000019302262B4F4FF000082046FFF760F858
:10572000044628B3F8F78EFF274A002352F8041BDB
:10573000884231D00133112BF8D1002307EB8302CB
:10574000D2F8B823904213D1B8F1020F26D0B8F1A5
:10575000030F26D0B8F1010F14BF8DF809308DF872
:105760000A3008F101080136B8F1040FF6B2D4D1BD
:10577000012E19D804B0BDE8F041FEF7D6BE0134C1
:105780002046F8F75FFF012303FA00F0019B23EAAC
:105790000003BDE70126BDE7DBB2CFE78DF80C3093
:1057A000DFE78DF80B30DCE701AB03CB286018682E
:1057B0006960A86004B0BDE8F08100BFD8C00020D7
:1057C00010F40608044E0608BC5106082DE9F04FF7
:1057D000834687B090460C46164600274FF0190ABC
:1057E0004FF46179B8F1000F4DD0B078A5783378D7
:1057F000727896F803C096F804E07179854240D13A
:1058000025789D423DD1657895423AD1E578654548
:1058100037D12579754534D165798D4214BF00257E
:1058200001251AFB02921AFB0393CDE901030392AF
:105830000091CDE904CE154A3B4629465846FFF76C
:10584000C1FD23790593E378049363780F4A1AFB2B
:105850000393039323781AFB03930293A378019392
:105860006379009329463B4658460137FFF72AFDE6
:10587000142F04F1060406F10606B3D107B0BDE803
:10588000F08F0025CDE74546DBE700BF23F406088F
:105890002DE9F3478246FEF795FD064630B13E49B5
:1058A0000022012002B0BDE8F0478FE75046F8F72C
:1058B000C9FE1328054663DC062747430AF10100A9
:1058C0008DF80760354CFEF78BFF04F6480909EBAD
:1058D0000708064648B1F8F7B5FE03289FBFE3194D
:1058E00083F84D0801238DF807303046FEF778FF26
:1058F000064668B1F8F7A6FE1D2809D8062303FB63
:10590000054383F84A089DF8073001338DF80730C6
:105910000DF1070241463046FEF76FFFFEF760FFCC
:10592000064668B1F8F78EFE3C2809D89DF8073086
:10593000062202FB0542013382F84B088DF807303E
:105940003046FEF74DFF68B1F8F77CFE1D2809D8F8
:105950009DF80730062202FB0544013384F84C0809
:105960008DF807309DF80730062B11D0002349F839
:105970000730A8F8043002B0BDE8F047FEF7D5BD07
:1059800007481322314602B0BDE8F047FEF7D2BD0A
:1059900002B0BDE8F08700BF08C10020C0B80020F9
:1059A000F6F406082DE9F04F2DED088BDFF814A171
:1059B00097B0074690460C461546002694ED008A9F
:1059C000B5EE408AF1EE10FA73D0D4ED019A94ED61
:1059D000029AD4ED038AB8F1000F40D095ED000A89
:1059E00095ED01BAD5ED02AA95ED03AAB4EE408A71
:1059F000F1EE10FA62D1F4EE4B9AF1EE10FA5DD1AD
:105A0000B4EE6A9AF1EE10FA58D1F4EE4A8AF1EE49
:105A100010FA0CBF4FF001094FF0000912A8F8F777
:105A200021FDB0EE4B0A83460EA8F8F71BFDB0EE41
:105A30006A0A05900AA8F8F715FDB0EE4A0A049024
:105A400006A8F8F70FFD059B049A0390CDE900B373
:105A500002923346524649463846FFF7B3FCB0EE51
:105A6000480A12A8F8F7FEFCB0EE690A81460EA8B3
:105A7000F8F7F8FCB0EE490A83460AA8F8F7F2FCFA
:105A8000B0EE680A049006A8F8F7ECFC049B0390BB
:105A9000CDE901B3CDF80090334652460021384697
:105AA0000136FFF70FFC0C2E04F1100405F1100570
:105AB00084D117B0BDEC088BBDE8F08F4FF0000922
:105AC000ACE700BF41F40608F8B50546FEF77AFCDE
:105AD000064660B146498B784FF4D67202FB03113B
:105AE00001F6D4010022BDE8F84001205AE74149FF
:105AF00005222846F8F74EF978B93D4A02F50C63BD
:105B000092784FF4D67101FB0233002201300C2849
:105B10005A6103F11003F9D1F8BD2846F8F792FD58
:105B20000B2804465CD82846FEF75AFE0546002896
:105B300040D0F8F7FBFC2E4B03F50C629B784FF43A
:105B4000D670611C434303EB0113134483ED010A38
:105B500001262846FEF744FE054678B1F8F7E6FC34
:105B6000234B03F50C629B784FF4D670611C4343C2
:105B700003EB0113134483ED020A01362846FEF7B6
:105B80002FFE054670B1F8F7D1FC194B03F50C62F6
:105B90009B784FF4D6714B4303EB0413134483ED0E
:105BA000070A01362846FEF71BFE28B9BDE8F84073
:105BB000FEF7BBBC0646CCE70D4FBD78F8F7B6FC48
:105BC0004FF4D6736B4307F50C6103EB04140C44DC
:105BD000032E84ED080AE9D114330022194482E728
:105BE00031460548BDE8F8400B22FEF7A3BC00BFD4
:105BF000C0B800207BF10608F6F406082DE9F3474B
:105C0000DFF868A081460E4617464FF002080024D0
:105C100057B337F8243036F8241037F80820994263
:105C200020D136F80850A91A4D424D41CDE9003235
:105C30002946234652464846FFF7C4FB36F808304B
:105C4000019336F8243000935246234629464846AD
:105C50000134FFF737FB042C08F10408D8D102B057
:105C6000BDE8F0870025E1E73D46E7E755F4060883
:105C7000F8B50446FEF7A6FB054628B1BDE8F84096
:105C80002A4900220120B9E729492046F8F79CF863
:105C9000A8B9284B4FF47A714FF4FA62A3F86C1A42
:105CA000A3F86E2AA3F8701AA3F8722AA3F8741A3C
:105CB000A3F8762AA3F8781AA3F87A2AF8BD204622
:105CC000F8F7C0FC0328064628D82046FEF788FDD2
:105CD000044670B1F8F7B6FC012705462046FEF7EA
:105CE0007FFD10B1F8F7AEFC37B9BDE8F840FEF71C
:105CF0001CBC05460746F1E7A5F2EE2240F2DC5354
:105D00009A42F2D8A0F2EE229A42EED8094B03EB67
:105D10008603A3F86C5AA3F86E0ACFE72946064813
:105D2000BDE8F8400322FEF705BC00BF2CC30020ED
:105D30007BF10608C0B8002066F406082DE9F04F94
:105D400091B0174607900C461546002604F1150938
:105D50000DF1240B0422494658464EF001FB002366
:105D60008DF82830D4E90232082B72F100010DF1D0
:105D70002C0A55D22F491A465046F7F787FE002FB6
:105D800056D095F80080237843454ED1D4E90202DD
:105D9000D5E902139A4208BF884246D1227D2B7D65
:105DA0009A4242D1042205F1150148464EF058FAB4
:105DB00000283AD121692B69CB1AD3F1000949EBAC
:105DC00003091D4B059300230493B5F91230039387
:105DD000B5F910300293194B194A0798CDE90083A1
:105DE00049463346FFF7EEFACDF814B0237D04930D
:105DF000B4F912300393B4F91030114A0798CDE981
:105E000001A314F8203B0093494633460136FFF7BF
:105E100059FA082E05F1200598D111B0BDE8F08F90
:105E200008495046F7F732FEA9E74FF00009C8E7E6
:105E3000B946D9E75226070862160708BC3007089A
:105E400079F406086EF406082DE9F74F0446FEF7CC
:105E5000B9FA074630B170490022012003B0BDE80D
:105E6000F04F6BE76D492046F7F7AEFF014638B9B2
:105E700069484FF4807203B0BDE8F04F4EF01ABA93
:105E80002046F8F7DFFB83B2072B054600F2BB8004
:105E90002046FEF7A5FC804600284CD0F8F7D2FB40
:105EA00001240FFA80FB4046FEF79AFC68B14FF0E0
:105EB000000A411E00F1100C564611F8013F13F084
:105EC000DF0F3BD101270134E4B2FEF789FC8046A5
:105ED00000284CD0F8F7B6FB01340FFA80F9E4B291
:105EE0004046FEF77DFC0346002842D00190F8F7BB
:105EF000A9FB0134019B0FFA80F8E4B21846FEF7C3
:105F00006FFC0346002836D00190F8F79BFB013464
:105F1000019B41B2E4B218460191FEF761FC019980
:105F2000024650B30134E4B2032C28D803B0BDE8D4
:105F3000F04FFEF7FABA04468346B4E76145C2D093
:105F4000A3F13002D2B2092A05D9A3F16102052AD0
:105F500007D8573BDAB2360146EA1A7642EA0A1AFD
:105F6000ABE7A3F14102052AADD8373BF2E7814602
:105F7000B6E78046C2E70146CDE7294AD4E71FFAD3
:105F80008BF3022BD2D809F226239BB2B3F5E16F33
:105F9000CCD808F226239BB2B3F5E16FC6D8CCB2B9
:105FA000062CC3D8104601924AF094FC0428BDD8B0
:105FB000002FBBD01B4B019A2DB203EB451103F50B
:105FC000286303EB4510C0E902A60346164D81F88D
:105FD00080BAA1F8909AA1F8928A81F8944A143371
:105FE000511E033211F8010F2C5C04F00304022C43
:105FF00008BF203803F8010F087808B18A42F1D1B0
:1060000003B0BDE8F08F09480722394603B0BDE868
:10601000F04FFEF78FBA00BF40C300207BF10608A7
:1060200062160708C0B80020C15007089AF4060895
:106030002DE9F04FDFF8AC9087B0834690460C46D0
:1060400016460027B8F1000F49D0707A617AB6F988
:106050000AC0B6F90CE096F808A08142D6E90032F1
:106060003BD12168994238D16168914235D1B4F968
:106070000A10614531D1B4F90C1071452DD1257A42
:10608000A5EB0A014D424D41CDE90032CDE9020CAC
:10609000CDE904EA3B464A4629465846FFF792F9BD
:1060A000237A0593B4F90C300493B4F90A300393BE
:1060B000637A02936368019354F8103B00934A4655
:1060C0003B46294658460137FFF7FCF8112F06F1E9
:1060D0001006B7D107B0BDE8F08F0025D4E74546DC
:1060E000DEE700BFA7F406082DE9F74F0446FEF7E8
:1060F00069F9054630B14F490022012003B0BDE8DF
:10610000F04F95E74C492046F7F75EFE30B94FF067
:10611000FF3003B0BDE8F04F3FF002BF2046F8F774
:1061200091FAC3B2102B834607D94448102229465E
:1061300003B0BDE8F04FFEF7FDB92046FEF750FB77
:106140000646E8B1F8F77EFA012482463046FEF7AB
:1061500047FB0646B8B1F8F775FA01348146E4B258
:106160003046FEF73DFB064600285CD0F8F76AFA99
:106170000128804609D903B0BDE8F04FFEF7D5B934
:1061800004468246E2E78146EAE70134E4B230465B
:10619000FEF726FB0646002847D0F8F753FA00F52D
:1061A000B473B3F5347F0746E5D80134E4B2304622
:1061B000FEF716FB0346002839D00190F8F742FAA3
:1061C00000F5B472B2F5347F0646D4D80134019B91
:1061D000E4B21846FEF704FB034640B10190F8F71D
:1061E00031FA0134051E019B18BF0125E4B218469F
:1061F000FEF7F6FA08B10134E4B2062CBBD1104B1D
:106200004FFA8BFB03EB0B13C3F880ABC3F8849BF3
:1062100083F8898BA3F88A7BA3F88C6B83F8885B5F
:1062200003B0BDE8F08F8046B1E70746BFE70646FA
:10623000CFE700BF40C400207BF10608C7F4060882
:10624000C0B800202DE9FF47DFF870908046174660
:106250000D4616464FF0000A77B3337829789942F5
:10626000D6E9012026D16968914223D1AC68211A70
:106270004C424C41CDE9012000934A465346214609
:106280004046FFF79FF8AB6802936B68019315F8DF
:106290000C3B00934A465346214640460AF1010A08
:1062A000FFF710F8BAF1080F06F10C06D4D104B0CC
:1062B000BDE8F0870024DDE73C46E4E7D8F40608B3
:1062C0002DE9F8430446FEF77DF8054628B1BDE800
:1062D000F8432E4900220120B4E72D492046F7F764
:1062E00073FD014628B9BDE8F843284860224DF007
:1062F000E1BF2046F8F7A6F9C3B2072B064606D938
:1063000029462448BDE8F8430722FEF713B9204682
:10631000FEF766FA074628B3F8F794F9051E18BF8A
:10632000012501243846FEF75BFA0746E0B1F8F78D
:1063300089F901348046E4B23846FEF751FA07463F
:10634000A0B1F8F77FF901348146E4B23846FEF790
:1063500047FA08B10134E4B2032C09D0BDE8F84390
:10636000FEF7E3B80446DDE78046E5E78146EDE762
:10637000094B76B20C2202FB063686F8905CC6F812
:10638000948CC6F8989CBDE8F88300BF50C50020E7
:106390007BF10608EDF40608C0B800202DE9F04FA7
:1063A000DFF8849091B007468846164600240DF128
:1063B0002C0A04EB840508EB050358F805001B794B
:1063C0000290514602A88DF80C3045F063FB4EB3A5
:1063D000731970591B790490052204A902A88DF83D
:1063E00014304DF03DFF0DF1180BB0FA80F5594611
:1063F00004A86D0945F04EFBCDF800B023464A468F
:1064000029463846FEF7DEFF2346CDF800A04A466F
:10641000294638460134FEF755FF802CC9D111B00A
:10642000BDE8F08F3546EFE7FCF406082DE9F04FA4
:1064300089B00546FDF7C6FF044630B16349002226
:10644000012009B0BDE8F04FA8E72846F8F7FAF8B0
:106450007F28064600F3B2802846FEF7C1F9B30054
:106460005A4A039306EB8603D118D450584B0C714B
:10647000CDE901430546A346A146A2462746A046CC
:10648000029B05AA13F8010B029394460023AE4623
:1064900015F8011B19B1884201D00A2B0CD1203309
:1064A0006B444FF00005884203F80C5C08D009B03B
:1064B000BDE8F04FFEF739B80CF8011B0133E6E7F1
:1064C00008F1FF330EF10105032B31D8DFE803F0AB
:1064D000591B026E4FF0010C12F8011B61B33D48CD
:1064E000002310F801EB8E455AD00133082BF8D168
:1064F0003948002310F801EB714553D10CFA03F32E
:1065000049EA0309E8E7012112F8013BA3B14E2B48
:106510003CD0452B3CD0532B3CD0572B3CD0552B5B
:106520003CD0442BF0D1052301FA03F31F43EBE7E2
:1065300005A8F8F787F8834608F101085FFA88F89C
:10654000B8F1050F9CD10399244B019A3144581896
:1065500003F54F630B4402F00F0204F00F0444EA0A
:10656000071442EA0B123F1180F8F02C80F8F1ACCE
:1065700080F8F29CDC701F7109B0BDE8F04F2FF07D
:10658000EFBD05A8F8F75EF80190D5E70023CBE74B
:106590000123C9E70223C7E70323C5E70423C3E7B1
:1065A0009A46A5E70133072BA4D195E705A8F8F78C
:1065B00049F810280446A8BF0024BDE708487F22F8
:1065C000214609B0BDE8F04FFDF7B4BFB0C50020CB
:1065D00000520608055206080D520608C0B80020F1
:1065E000F6F406082DE9FF47DFF86C908046174661
:1065F0000D4616464FF0000A67B333882A889A4240
:1066000026D16C887288A21A54425441F2780292C0
:10661000B2782146CDE90032404653464A46FEF75D
:10662000D1FEEB780293AB78019335F8043B0093ED
:106630004A465346214640460AF1010AFEF742FE09
:10664000BAF1100F06F10406D6D104B0BDE8F08708
:106650000024DBE73C46E4E706F506082DE9F041B7
:106660000546FDF7AFFE044628B1BDE8F0412449D8
:1066700000220120B6E72846F7F7E4FF0F28064678
:1066800036DC2846FEF7ACF81E4FDFF8848005465E
:10669000A0362846F7F7D6FF37F8023B98421FDCB2
:1066A000012C08EB860311D0022C12D0A3F8F00CB9
:1066B00028462C214DF015FE054668B10135012311
:1066C00001346BB1032CE4D1BDE8F08183F8F20C06
:1066D000EEE783F8F30CEBE7A21E53425341EFE7DA
:1066E000094B002243F82620BDE8F041FDF71DBF0D
:1066F00021460648BDE8F0410F22FDF71BBF00BF51
:1067000030C8002014520608B0C50020F6F4060870
:10671000C0B800202DE9F04FDFF8B49085B00646F0
:10672000884614464FF0000B062303FB0BF505F5D6
:106730003075002718F805A0002C44D0625DAAEB44
:10674000020041424141CDE900725B464A46304673
:106750000391FEF737FE0399CDE9007A5B464A467E
:1067600030460137FEF7AEFD062F05F10105E1D1F8
:106770000BF1010BBBF1070FD6D1DFF8549040F2BB
:10678000EA2518F805B0A5F2EA2AF4B1635DABEB8F
:10679000030257425741CDE900A34A460723394631
:1067A0003046FEF70FFE0723CDE900AB4A463946D7
:1067B0003046FEF787FD013540F2F3239D42E0D1DC
:1067C00005B0BDE8F08F2146C6E72746EBE700BFDE
:1067D00018F506082DE9FF47DFF898908046174620
:1067E0000C4616464FF0000A002F41D0B6F9003093
:1067F000B4F90010B6F90220B6F9040096F906C003
:10680000994233D1B4F9021091422FD1B4F9041056
:1068100081422BD194F90610A1EB0C056942694124
:10682000CDE90032CDE9020C53464A4640460D46BA
:10683000FEF7C8FD94F906300393B4F904300293CF
:10684000B4F90230019334F9083B00934A465346A9
:10685000294640460AF1010AFEF734FDBAF1120F4B
:1068600006F10806C0D104B0BDE8F0870021D7E7E3
:106870003D46DFE72CF5060830B585B00546FDF747
:10688000A1FD044610B32E490022012005B0BDE849
:1068900030409FE72D2B03D0A3F13002092A4AD8BC
:1068A000042C04DD05B0BDE83040FDF73EBE2846AF
:1068B000F7F7C8FE04AB621C03EB440424F80C0C8D
:1068C00015F8013F303B092BFAD914462B78002BE1
:1068D000E0D1052CE6D1BDF80430BDF90450112BF0
:1068E000E0D8BDF90600A0F5FA739BB2B3F5FA6FD4
:1068F000D8D8BDF90810A1F5FA739BB2B3F5FA6FB9
:10690000D0D8BDF90A209042CCDC9142CADBBDF957
:106910000C4004F17D039BB2FA2BC3D8094B03EB67
:10692000C503A3F8E40FA3F8E61FA3F8E82F83F844
:10693000EA4F05B030BD202BB4D101352246C4E763
:10694000A4C80020C0B800202DE9F04F80468FB0C9
:1069500017460C4616464FF0000A23780793B4F901
:10696000029063782068A2880893237994F905B08F
:106970000A90ADF82C200993B9F1000F3DD0002FFB
:1069800040D03068BDF828500C9080B2B288ADF885
:106990003420854231787378B6F9022096F804E005
:1069A0002ED191452CD1BDF82C50BDF83400281AB9
:1069B00045424541CDE901320091CDE903EB124A50
:1069C000534629464046FEF7FDFC099B0E4ACDF88A
:1069D00010B0CDE90293089B0193079B00932946D1
:1069E000534640460AF1010AFEF76CFCBAF1240F47
:1069F00004F1060406F10606AFD10FB0BDE8F08F32
:106A00000025D7E73D46E0E741F50608F0B589B037
:106A1000044649F05FFF10F0FF020CD13A498B7831
:106A20004FF4D67000FB031101F69411012009B058
:106A3000BDE8F04088E7354905222046F7F7AAF976
:106A4000A8B9314B9A784FF4D67101FB0233304A22
:106A50001568948803F69413062606FB00F299182D
:106A6000013024289D508C80F7D109B0F0BD20461C
:106A70002849284E01AA4DF0AEFB4FF0FF33079393
:106A800002AD002478B1062C02D1FDF74EFDECE7F3
:106A9000F7F7D8FD01AA45F8040B31460020013470
:106AA0004DF099FBEEE7042CEFDD029F232FECD88D
:106AB000039E112EE9D8049D3C2DE6D8059C04F5D3
:106AC0007A73B3F5FA6FE0D80698FF28DDD80799F6
:106AD0004B1C402BD9D80C4B9A784FF4D67C0CFB2E
:106AE00002F24FF0060C0CFB0722134483F89809BE
:106AF000094883F8946983F89559A3F8964983F86F
:106B00009919FFF783FFB0E7C0B800207BF10608B2
:106B10001A520608A4420708621607082DE9F04F2A
:106B20009BB091460E900F930C46154600260F9B86
:106B30005A1C01D0B34266D1A446BCE80F0010AF86
:106B40000FC7DCF800303B6023790993237C0B935B
:106B500094F911300C93A37C94F80C8094F813A052
:106B60000A9207460D93B9F1000F5AD0AE46BEE81F
:106B70000F000DF1540CACE80F00DEF80020149B60
:106B8000CCF80020534033F07F43864695F804B09C
:106B9000A96895F80CC0E87C3FD1099A5A453CD1C8
:106BA00077453AD1E04538D10A9A8A4237D1AAEBE3
:106BB0000003594259410A9B1B4A0E98CDF81CA06C
:106BC000CDE90583099B03930D9B02930C9B0193D5
:106BD0000B9B0093049733468B46FEF7F3FB0A9B0F
:106BE000114A0E98CDF81CA0CDE90583099B0393AB
:106BF0000D9B02930C9B01930B9B009304973346D0
:106C00005946FEF75FFB0136402E04F1140405F1EE
:106C100014058CD11BB0BDE8F08F0021CBE71946DD
:106C2000C9E7CB46DBE700BF58F506082DE9F04180
:106C30008AB004460D4649F04DFE10F0FF000FD11A
:106C40003E4B1A783AB94FF0FF333D4901200AB064
:106C5000BDE8F04162E76B1C6DD02B460246F4E7BD
:106C6000384905222046F7F795F838B934484FF4EB
:106C70007E710AB0BDE8F04147F0C2BB2046324900
:106C8000314E6A464DF0A7FA01AD002478B1092CC7
:106C900002D1FDF74AFC4EE0F7F7D4FC6A4645F80E
:106CA000040B3146002001344DF095FAEEE7092C33
:106CB000EFD101993F29ECD8DDF808E0BEF1010FD2
:106CC000E7D8DDF80CC00CF10103402BE1D8049F9C
:106CD000382FDED8059E072EDBD8069D1B4A05F50A
:106CE000742303F510739342D3D8079C072CD0D894
:106CF000089800F5742303F510739342C9D8099AD4
:106D0000FF2AC6D8124B4FF0140808FB013309B212
:106D100043F87C0C0F4803F874EC03F873CC03F8C9
:106D2000727C03F8806C43F8845C03F8784C03F8B9
:106D3000712CFFF77BFF0AB0BDE8F081F6800020E0
:106D400034C900207BF10608A442070880841E0095
:106D5000B8C90020621607084FF0FF3166E72DE939
:106D6000F04F074687B016460C4615464FF0000B0D
:106D7000D4E9009AD4F8088066B3A8688045D5E9BC
:106D8000002125D1914523D1AAEB01035942594154
:106D9000CDE9019A104ACDF800805B46384605914E
:106DA000FEF710FB05990C4ACDF800805B46CDE953
:106DB000019A38460BF1010BFEF784FABBF1080F7C
:106DC00004F10C0405F10C05D2D107B0BDE8F08F39
:106DD0000021DDE73146E6E779F5060870B586B0B3
:106DE000044649F077FD10F0FF0205D1214901204A
:106DF00006B0BDE87040B2E71F4905222046F6F70D
:106E0000C9FF38B91B4840F2FF3106B0BDE87040F9
:106E100047F0F6BA20461949184E01AA4DF0DBF9A1
:106E200002AD002478B1042C02D1FDF77EFB1FE0F7
:106E3000F7F708FC01AA45F8040B3146002001349D
:106E40004DF0C9F9EEE7042CEFD1029A072AECD8ED
:106E50000B4B0C480C2101FB0233039AC3F884242A
:106E6000049AC3F87C24059AC3F88024FFF7B6FF80
:106E700006B070BD34CE00207BF10608A44207089E
:106E8000B8C90020621607082DE9F04FA1B01746D7
:106E900010900C4615460026A646BEE80F000DF1E0
:106EA000480CACE80F0023680B939EE80700238A88
:106EB0000C93638A0D93A38A0E93E38A94F804805B
:106EC000D4F808B094F80CA094F818900F938CE8BC
:106ED0000700002F5CD0AE46BEE80F000DF1640C39
:106EE000ACE80F009EE807008CE8070095F818C092
:106EF00029682879AB682A7BCC4547D1804545D1A4
:106F00000B98884242D1924540D19B453ED1169A7A
:106F10001D9B9A423AD117991E9BCB1A594259414F
:106F20000F9B08930E9B07930D9B06930C9B194A8E
:106F30001098CDF80CA0CDE904B30B9BCDF80090D0
:106F4000CDE9018333461191FEF73CFA11990F9B6D
:106F500008930E9B07930D9B06930C9B0D4A10986C
:106F6000CDF80CA0CDE904B30B9BCDF80090CDE992
:106F7000018333460136FEF7A5F9042E04F11C0403
:106F800005F11C0588D121B0BDE8F08F0021C7E7CD
:106F90003946DCE78AF506082DE9F0438DB0044652
:106FA00049F098FC10F0FF0205D13F4901200DB0D7
:106FB000BDE8F04368E73D4905222046F6F7EAFEC2
:106FC00038B939484FF47E710DB0BDE8F04347F051
:106FD00017BA20463649364E01AA4DF0FCF802ADEC
:106FE000002478B10A2C02D1FDF79FFA59E0F7F797
:106FF00029FB01AA45F8040B3146002001344DF06D
:10700000EAF8EEE70A2CEFD1DDF80880B8F1030FBB
:10701000EAD8DDF80CE0BEF1010FE5D8DDF810C0CC
:10702000BCF1070FE0D8059F224A07F5742303F54A
:1070300010739342D8D8069E072ED5D8079D05F524
:10704000742303F510739342CED8089CB4F5004F17
:10705000CAD20998B0F5004FC6D20A99B1F5004FCF
:10706000C2D20B9AB2F5004FBED2134B4FF01C099F
:1070700009FB0833A3F8EE0483F8F4E483F8E0C4D2
:10708000C3F8DC7483F8E864C3F8E454A3F8EC4470
:10709000A3F8F014A3F8F22423F090FE0748FFF7BA
:1070A0007BFF0DB0BDE8F08394CE00207BF1060895
:1070B000A442070880841E00B8C900206216070891
:1070C0002DE9F04FA1B0CDE90C011546002414AE16
:1070D0000D9A02EB441263010DF1400C02F1200EF7
:1070E00010685168674603C708327245BC46F7D13D
:1070F000002D00F081802B4418AF03F1200C18689C
:1071000059683A4603C2083363451746F7D19DF8DC
:1071100040300B939DF860100B98BDF842709DF8BD
:107120004480BDF846909DF848A0BDF84AB09DF84F
:107130004C30BDF84E2081425CD1BDF86210B9429E
:1071400058D19DF86410414554D1BDF866104945A9
:1071500050D19DF8681051454CD1BDF86A10594581
:1071600048D19DF86C10994244D1BDF86E109142FF
:1071700040D11CA914A8CDE90E3249F0A1FBDDE9EC
:107180000E32B0FA80F14909CDE905B30B9B0093AB
:10719000CDE90726CDE9039ACDE90178174A0C9885
:1071A0000B912346FEF70EF90B99BDF84E3007936D
:1071B0009DF84C300693BDF84A3005939DF8483051
:1071C0000493BDF8463003939DF844300293BDF814
:1071D000423001939DF840300093084A0C9808967D
:1071E00023460134FEF76EF8082C7FF471AF21B00E
:1071F000BDE8F08F0021C7E72946D6E7ACF50608C1
:107200002DE9F04190B0044649F064FB10F0FF0214
:1072100005D14549012010B0BDE8F04150E7434990
:10722000434F01AA20464CF0D6FF41496A464CF034
:10723000D2FF06AE0024354600286ED0092C61D15D
:107240003A4901AA00204CF0C6FF0646002869D042
:1072500049F040FB044638B10F2828BF0F242246CE
:10726000314602A84CF0E2FF04F14003DDF818803B
:107270000DEB0304B8F1070F4FF0000304F8383C9E
:107280004DD8DDF81CE0BEF11C0F48D8DDF820C059
:10729000BCF1FF0F43D8099F1C2F40D80A9EFF2E38
:1072A0003DD80B9C1C2C3AD80C98FF2837D80D9948
:1072B000022934D80E9AFF2A31D81E4B03EB48130B
:1072C00003F25C5303F8084C03F810EC23F80ECCDF
:1072D00003F80C7C23F80A6C23F8060C03F8041C52
:1072E00023F8022C02AC224603CAAA421860596055
:1072F000144603F10803F6D10F48FFF781FF10B0E1
:10730000BDE8F081F7F79EF96A4646F8040B394666
:10731000002001344CF05FFF8EE7092C90D0FDF780
:1073200004F9ECE704469FE704CF0020C0160708E5
:10733000A4420708B8C90020621607082DE9F04FDB
:10734000DFF864A0DFF864B085B0064689461546CC
:107350001F460024002F01DBA7421DD119F804802D
:1073600005B32B5DA8EB03020AEB83035142D3F86C
:107370001C340093514123465A4630460391FEF790
:1073800021F803990AEB88085A46D8F81C34009370
:1073900030462346FDF796FF01340E2CDAD105B0B6
:1073A000BDE8F08F2946EDE7044E0608E0F5060833
:1073B0002DE9F3412649DFF8988001AA4CF00BFF34
:1073C000002504462F464FF0FF366CB9022F0BBF45
:1073D000204920498D55334612BF22463346224666
:1073E0000120FFF7ABFF04E037B1012F12D0FDF70A
:1073F0009CF802B0BDE8F0812046F7F723F90D288C
:107400000646F4D801AA414600204CF0E4FE0137BC
:107410000446DAE710482146F6F7D6FC0546002870
:10742000F0D00E482146F6F7CFFC60B10C4821465B
:10743000F6F7CAFC48B10B482146F6F7C5FC002810
:10744000D5D10325DEE73D46DCE70225DAE700BFBC
:10745000A4420708307F0020F8F50608930C0708BF
:10746000AF390708D93E07080FB407B504A951F88A
:10747000040B0191FCF792FF03B05DF804EB04B03C
:107480007047F8B5C47914F0C003064602D0402B0B
:1074900015D0F8BD14F00EFE04F00704062C0546C6
:1074A00004D10146BDE8F8401348DDE7304614F04A
:1074B000F1FD2A460146BDE8F8401048D4E714F033
:1074C0007EFE05460E480F4E0F4FFCF71BFF0024B3
:1074D0002B79A34203D8BDE8F840FCF721BF14B1D3
:1074E0003046FCF70FFF2B68384653F82410FCF7A2
:1074F000CDFF0134ECE700BFFDF506080DF60608E8
:1075000024F6060834F606081BF706082DE9F047AE
:107510008CB0074610F8013B202BFAD00024DFF88E
:107520008480DFF88490DFF884A02646204614F09B
:1075300025FD6946054614F0A9FC394668464CF01D
:1075400032FFE0B169464046FCF7A0FF4946684675
:1075500049F0B6F9F0B9284614F090FD104B0146F9
:107560000078202814BF50461846FCF78FFFFCF720
:10757000D7FE2846FFF785FFFCF7D2FE013601341F
:1075800040F292239C42D1D10EB944F067FA0CB07C
:10759000BDE8F08700212846FDF770F8E7E700BF57
:1075A000DBF506086FF00608834B07081CF7060892
:1075B0002DE9F04F2DED028B8DB00578202D06467C
:1075C00000F10100F9D0304649F084F9044618B1C1
:1075D000012822D12A2D20D19748DFF87C82FCF7A0
:1075E000B1FE002540F29227284614F0C7FC6946F8
:1075F000064614F04BFC69464046FCF747FF013550
:1076000021463046FDF73AF8FCF78AFEBD42EBD141
:107610000DB0BDEC028BBDE8F08F3D2130464CF043
:1076200060FE002800F000810346994613F8012D02
:10763000202AFAD0A9EB060901308046074610F847
:10764000013B202BF9D04FF0000A5FFA89F9504630
:1076500014F094FC6946054614F018FC684649F09D
:1076600039F96946024683463046F6F793FB40F205
:107670009223044638BBCB4525D1EB7903F00706AE
:10768000062E2DD14046F6F773FB6C49684649F04B
:1076900017F920B16A49684649F012F9D0B998F84B
:1076A0000030222B16D1404649F014F908EB0003B4
:1076B00013F8013C222B0DD1821E08F1010128464E
:1076C00014F09AFDA4E70AF1010A9A45BFD144F0EB
:1076D000C5F99DE7404649F0FDF841460246EEE710
:1076E00013F0C0030AD0402B6AD05648FCF730FE96
:1076F0002846FFF7C6FEFCF713FE89E798F800302E
:10770000002BF2D0504940464CF03DFE0446404626
:1077100049F0E0F88442E8D14046F6F707FF2846F2
:10772000B0EE408A14F0B6FC07EE900AF8EEE77A65
:10773000F4EEC87AF1EE10FAD7D8284614F0BAFC65
:1077400007EE900AF8EE677AF4EEC87AF1EE10FAD6
:10775000CBDB052E1AD118EE104A3C49684649F099
:10776000AFF848B93A4B93F85716E2B2914203D0BA
:10777000002C45D183F8BB46284614F07FFC052E2B
:1077800043D8DFE806F041414B4B4D4F042E12D158
:107790003A4617F8013B202BFAD0092BF8D0013AD2
:1077A00000240A2112F8013F303BDBB2092BD4D868
:1077B00001FB0434F6E74046F6F744FF0446CCE705
:1077C000284614F0FCFC90F804B081462746234676
:1077D000A246BB4500D91BB1BAF1000F85D0BCE76A
:1077E000D9F80030414653F82700F6F7EDFA0028A3
:1077F00005BF3C46012300234FF0010A0137E8E7AB
:10780000012283F8BB26B7E7047069461148FCF7EC
:107810003DFE00212846FCF731FFF9E60480F4E73D
:107820000460F2E70460F0E730460DB0BDEC028B77
:10783000BDE8F04F6AE600BF36F60608834B07083E
:1078400048F6060882F6060853F6060861F60608AA
:10785000B8C9002077F606086FF006087FB5034622
:10786000FCF7B0FD044638B119490022012004B0EC
:10787000BDE87040FEF74EBF1649164E6A461846E0
:107880004CF0A9FC01AD80B1032C03D1FCF74DFEF7
:1078900004B070BDF6F7D6FE6A4645F8040B3146D3
:1078A000002001344CF097FCEDE7032CEED1DDE92C
:1078B0000145039E29463246E0B22EF0B1FD002874
:1078C000E4D0054833462A462146FFF7CDFDDFE7E1
:1078D000B0C50020A442070818F5060810B50346F5
:1078E000FCF770FD30B1F9F761F9BDE810400748C9
:1078F000FCF728BD1846F6F7A5FE044680B2F9F756
:1079000029F921460248BDE81040ADE592F6060887
:107910009EF6060808B50346FCF754FD38B10B4B3C
:107920000B4800221A80BDE80840FCF70BBD184642
:10793000F6F788FE014628B1044B1880BDE80840E0
:10794000044891E5BDE80840FCF7EFBDF480002055
:10795000B0F60608C6F606082DE9F84F054648F0C9
:10796000B9FFDFF8EC800446D8F80090C0B9304881
:10797000304D314FFCF7C6FC012655F8041B59B1B8
:107980000B783BB106FA04F313EA090F02D038462C
:10799000FCF77CFD0134F0E7BDE8F84FFCF7C0BC14
:1079A000024626492846F6F7F5F978B92448214CCD
:1079B000214DFCF7A7FC54F8041B0029ECD00B78F0
:1079C000002BF8D02846FCF761FDF4E72B78DFF8B0
:1079D00064B02D2B03BF013504F1FF344FF0010AD1
:1079E0004FF0000A00265BF8047B1FB9BDE8F84F92
:1079F00044F034B8224639462846F6F7CBF9A0B908
:107A00000120B040BAF1000F09D0F6F777FF0D481A
:107A1000FCF778FC39460C48BDE8F84F24E540EA0D
:107A20000900C8F800000948F2E70136DBE700BFAB
:107A3000DDF606083452060812490708E7F606087C
:107A4000ECF60608F8F606081BF7060801F7060824
:107A5000543D00202DE9F84F054648F03BFFDFF884
:107A6000F4800446D8F80C67C8B93148314DDFF8C6
:107A7000D480FCF747FC0127E3B205EB8302D2F880
:107A8000B41441B107FA03F3334202D04046FCF785
:107A9000FDFC0134F0E7BDE8F84FFCF741BC0246BD
:107AA00025492846F6F776F960B92448244C254D37
:107AB000FCF728FC54F8041B0029ECD02846FCF7FE
:107AC000E5FCF7E72B78DFF878B02D2B03BF013505
:107AD00004F1FF344FF0010A4FF0000A4FF00009A3
:107AE0005BF8047B1FB9BDE8F84F43F0B7BF2246EF
:107AF00039462846F6F74EF9B0B9012303FA09F3DF
:107B0000BAF1000F0BD026EA03030F48C8F80C3770
:107B1000FCF7F8FB39460D48BDE8F84FA4E43343C1
:107B20000B48C8F80C37F3E709F10109D8E700BFA3
:107B3000DDF60608044E0608E7F60608ECF6060829
:107B4000B852060812490708F8F606081BF7060897
:107B500001F70608B8C900202DE9F047814648F032
:107B6000B9FE484E0446376800BB4748474D484E6B
:107B7000FCF78CFC4FF00C0808FB04F35A5D012362
:107B8000013A93403B4206D020461CF083FB01465D
:107B90003046FCF77BFC0134182CEDD117B93D4879
:107BA000FCF7B0FBBDE8F047FCF7BABB02463A4928
:107BB0004846F6F7EFF8054678B93848FCF7A2FBD7
:107BC0002C46334D20461CF065FB01340146284607
:107BD000FCF75CFC1A2CF5D1E4E799F800302D2B6A
:107BE00003BF09F1010904F1FF344FF0010A4FF01E
:107BF000000A002528461CF04DFB2246804601461F
:107C00004846F6F7C7F8002835D1BAF1000F1BD067
:107C1000182D16D0192D09D1736821483360FCF74F
:107C200071FB41461F48BDE8F0471DE41E4B0C2286
:107C300002FB053393F8F0240123013A93403B43C0
:107C4000EBE76FF07F43E8E7182D03D1C6F800A0FB
:107C50001648E4E7192D01D17760F9E7124B0C22A1
:107C600002FB053393F8F0240123013A934027EAFD
:107C700003033360ECE701351A2DBBD1BDE8F047B3
:107C800043F0ECBE7C7F002009F70608F45206089A
:107C90001AF7060813F70608E7F606081FF706089E
:107CA000F8F606081BF70608044E060801F7060852
:107CB0002DE9F341044648F00DFE04283DD1661E2F
:107CC0002546E71C16F8010FF6F74CF8BE42307057
:107CD000F8D1DFF87880271D15F8016B4046314652
:107CE0004CF0FFFA20B1314628464CF0FAFA20B1A8
:107CF00002B0BDE8F041FCF718BCBD42ECD1204613
:107D000024F086F80F48FCF7FDFA0F490F480023CE
:107D100011F8012F10F8014B08326A440133042B8B
:107D200002F8084CF4D1002309488DF80430694664
:107D3000FFF79AFB02B0BDE8F0810028E2D0FCF723
:107D4000F4FBDFE72AF706088CBE00202C54060857
:107D50001CF7060830B585B00346FCF733FB054633
:107D600020B105B0BDE83040FCF7DFBB1846F6F7A0
:107D700069FC0728044607D923480722294605B08D
:107D8000BDE83040FCF7D6BB40B21DF07FFE88B1A5
:107D900042687AB11D4BD3F814178A4214D0D3F835
:107DA000F0178A4229D0D3F8CC188A4209D103F6B9
:107DB000CC030BE01648214605B0BDE83040FCF787
:107DC000A5BB14482146F7E703F2147300228DF88F
:107DD0000D20ADF80E200222009203A9042243F2E6
:107DE00001008DF80C401FF0CDFD0028214607DD75
:107DF0000948FFF739FB05B030BD03F5FE63E5E741
:107E00000648FCF783FBF6E730F70608B8C9002000
:107E100035F7060850F7060879F706089DF70608B3
:107E2000F7B50346FCF7CEFA044620B103B0BDE82F
:107E3000F040FCF77ABB20491F4F01AA18464CF0CE
:107E4000CAF92646254640B90B2D18D901461B48CC
:107E50000B22FCF76FFB03B0F0BD44B1012C0AD03C
:107E600001AA3946002001344CF0B5F9EBE7F6F7EA
:107E7000E9FB0546F4E7F6F7E5FB0646F0E7022CDA
:107E80000FD1A6F57A73B3F57A7F05D90C484FF474
:107E9000FA624FF47A71DCE70A4B03EB4503A3F86F
:107EA0000865084B084803EB45032946B3F9082544
:107EB000FFF7DAFACFE700BFA4420708F6F4060896
:107EC000151A0708906F0120CBF7060870B5034616
:107ED000FCF778FAC0B11F4B1E68013630461CF023
:107EE000D9F934460546E8B901341A2CA8BF002454
:107EF00020461CF0CFF90546A0B9B442F4D1BDE844
:107F000070401548FCF71EBA1846F6F79BFB04466E
:107F10001CF0C0F9054628B921461048BDE870405C
:107F2000FFF7A2BA0B4B1C601EF0EAFB2A460C4876
:107F30002146FFF799FA192C9DBF0A4B0C2202FB30
:107F400004330020BDE8704098BF93F8F0041EF0A1
:107F5000EFBB00BF14120020D8F70608ECF70608A4
:107F600002F80608044E06082DE9F04F2DED028BAD
:107F7000A5B0C04B0393C04B0293C04B0193C04BC1
:107F8000C04AC149C1480093C14BC24DC24CC34F06
:107F9000FFF76AFAC249C348FFF766FAC24BC34803
:107FA00019684FF47A73B1FBF3F1FFF75DFA08A893
:107FB000F6F702F808A918A846F02EFA18A9BC4846
:107FC000FFF752FA24F08EFC6423B0FBF3F103FBBD
:107FD000110095F8A93904EB830382B2D3F8303647
:107FE000009395F8A839B34889B2FFF73DFAB24B30
:107FF000B2481968B24BB1FBF3F1FCF747FAD7F876
:108000000485002604F5C86905F6AA1A04F25C6B1B
:108010000123B34013EA080F0BD059F8263043B1BF
:108020001AF806205BF8261053F82220A548FCF722
:108030002DFA0136072EEBD1FCF772F9A248A04EBB
:10804000FCF780F90BA8F2F73AFB0B999F48B1FBBC
:10805000F6F1FFF709FA0C999D48B1FBF6F1FFF72D
:1080600003FA0D999B48B1FBF6F1FFF7FDF90E9964
:108070009948B1FBF6F1FFF7F7F924F03FFE04EB66
:108080008000D0F88436069324F042FE04EB800092
:10809000D0F8848624F04CFE04EB8000D0F884965F
:1080A00024F06AFE04EB8000D0F884A624F088FE59
:1080B00004EB8000D0F884B624F0D0FE04EB8000FE
:1080C000D0F8846624F09AFE04EB8000D0F8841681
:1080D000079124F0A9FE04EB80000799D0F88436BC
:1080E0000493CDE902614B464246CDE900AB0699C7
:1080F0007A48FFF7B9F97A4B1B68DA031CD5794B3C
:1081000093F80080B8F1000F16D07748DFF834926A
:10811000DFF834A24146FFF7A7F90026B9F902209B
:10812000314650460136FCF7B1F9F3B2434509F147
:108130001009F3D3FCF7F4F80020FDF7DDF86B4BE2
:108140006B4A1E886B4B6C491B686C48DFF8FCA1BE
:10815000DFF8FC91DFF8FC81DFF8FCB1C3F50073B8
:108160009B00FFF781F9664A664B6748D31A674A56
:10817000B6B231461288FFF777F96548FCF7E2F8A6
:1081800004265AF8041B6348FCF780F96248FCF7A0
:10819000B9F819F8011B002940F0D7815F48FCF7B6
:1081A000B1F85F48FCF7AEF858F8041B002940F01E
:1081B000D0815A48FCF7C6F8013EE2D1B7F8201545
:1081C0005848FCF763F958490A6F5AB107EE902AEC
:1081D000DFED566AF8EEE77A86EEA77AFDEEC77A0B
:1081E00017EE902AD1F800315BB107EE903ADFED3F
:1081F0004F6AF8EEE77A86EEA77AFDEEC77A17EEB9
:10820000903A896A59B107EE901ADFED486AF8EEA4
:10821000E77A86EEA77AFDEEC77A17EE901A0091FC
:10822000B5F8B8194248434F434EDFF83091FFF795
:108230001BF94248FCF766F83B684FF001081E4006
:10824000002E40F08A81FCF76BF83B685B0140F13F
:1082500087800FA813F046FF002840F081800F9818
:1082600013F08CFE18A913F011FE354818A9FCF77D
:108270004DF975E0621607081DF8060826F806088D
:108280002FF8060890EB0608A3EB060896FD0608F3
:1082900017F80608B8C90020044E0608906F0120A0
:1082A0003BF80608B1FD0608042A00204BF8060832
:1082B00065F8060876F80608040100209BF8060811
:1082C00040420F00ABF80608B3F80608C8F80608E5
:1082D000DAF80608ECF80608FEF8060810F90608B1
:1082E000886F0120846F01206DF90608F0320020AC
:1082F000000002202033002000180000A1F9060829
:108300000080000800400008D9F90608523D00200E
:1083100013FA060826FA06082EFA060815F70608C4
:1083200044FA06084EFA0608D008002000247449D2
:108330005EFA0608E06E0120C0FFFD7F9BFA06088A
:10834000B2FA06087C3C002092F906089854060808
:1083500069D30020A05F00203DFA06081BF706083D
:108360003E68370509D500203DF0F6F9042840F0B5
:10837000078191499148FFF777F89148FBF7C2FFD1
:10838000D5F8BC19002900F00E810B7B4A7B8D4883
:108390008968FCF77BF8FBF7C3FF8B48FBF7B2FF5C
:1083A000D5F8C009FBF751FF002800F000810FA9A4
:1083B000D5F8C009FBF78AFF9DF850109DF85C3096
:1083C000169A8248FCF762F8139911B18048FCF7BD
:1083D0005DF8119911B17F48FCF758F8FBF7A0FF41
:1083E0007D4B1B68180640F1A1802CF0D5FB0028BE
:1083F00000F09C807948FBF785FF794890F840367B
:1084000090F84126453BDBB2052B96BF04EB830376
:108410007449D3F8081790F8423690F844060728B4
:1084200096BF04EB80000020D0F8200700906E4833
:10843000FCF72CF800210F202CF0BAFB10B16B4890
:10844000FCF724F86A4E9FED6B8AFBF769FFF17920
:108450006948FFF709F8738C07EE903AF8EEE77A6F
:10846000C7EE887A17EE900A48F0A0FB02460B464A
:108470006248FEF7F9FFF38B07EE903AF8EEE77AE1
:10848000C7EE887A17EE900A48F090FB02460B463A
:108490005B48FEF7E9FF338C07EE903AF8EEE77A97
:1084A000C7EE887A17EE900A48F080FB0B4602462A
:1084B0005448FEF7D9FF5448FEF7D6FF5348FBF760
:1084C00041FF5348FBF73EFF95F8C43919070AD519
:1084D00095F8CC2995F8CD194E48C2F3C002C1F3E6
:1084E000C001FEF7C1FF95F8C4395A070AD595F8BF
:1084F000CC2995F8CD194848C2F38002C1F3800118
:10850000FEF7B2FF95F8C4399B070AD595F8CC2938
:1085100095F8CD194148C2F34002C1F34001FEF77E
:10852000A3FF95F8C8193E48FEF79EFF3D4B1B7808
:1085300033B104EB83043C48D4F84017FEF794FFB2
:1085400025B0BDEC028BBDE8F08F5846FBF79EFFCF
:1085500027E65846FEF788FF2EE696FAA6F3B3FA0A
:1085600083F308FA03F2052B26EA02067FF768AECA
:1085700004EB83034846D3F88C16FBF787FF5FE6CE
:10858000012801D12949F5E6022807D1760303D550
:108590002748FEF769FFF0E62649EBE603287FF45B
:1085A000ECAE2548F5E72548FBF7ACFEF3E624489A
:1085B000FBF7A8FE12E700BFC6FA06081AF706087E
:1085C0003BFB060841FB06085AFB060860FB060851
:1085D0007EFB060887FB0608543D0020A3FB060827
:1085E000C0B800208BFE0608A9FB0608D0FB0608D1
:1085F000E46F00200000C842F0FB0608FBFB060801
:1086000006FC060813FC060820FC060835FC0608D4
:1086100056FC060862FC060874FC060885FC060881
:1086200097FC06083E7F0020AEFC0608E2FA06082A
:10863000F6FA06080FFB060828FB06084EFB06089C
:1086400096FB06082DE9F04F2DED028B4D484E4D5F
:108650009FED4E8A8BB0FEF707FF0027B946BA465A
:108660004B4B4C4AD3F8241500238B4227DB0137B0
:108670001D2F05F14805F3D14749484BD1E90021A9
:10868000520942EAC1624649186809684FF47A7390
:10869000B0FBF3F34348FEF7E7FE0A2299FBF2F33F
:1086A00002FB139000909AFBF2F13F4802FB11A2EB
:1086B000FEF7DAFE0BB0BDEC028BBDE8F08F52F88E
:1086C000040BA84201D00133CFE7AC6A4CB107EEEE
:1086D000904AB8EEE77AC8EE077AFDEEE77A17EE31
:1086E000904AAB6B0893D5E90C637609E96B46EACF
:1086F000C3665B090993089B4FEAE47B6143A4FBD3
:10870000030C03FB0B1141F28833C01841EB0C0141
:108710004FF47A72002348F0E9FE099A804604FB80
:1087200002F1A4FB060C41F28833C01806FB0B11C2
:1087300041EB0C014FF47A72002348F0D7FE2B6C0A
:108740000196042F4FF47A72B3FBF2F306934FF0C5
:108750000A0318BF814490FBF3F203FB1200CDE93A
:10876000042098FBF3F203FB1283CDE90223089B5C
:1087700000932A680D482346394618BFC244FEF7C5
:1087800073FE74E7C8FC0608D00800200024744972
:10879000906F0120E86E0120606F0120686F01205A
:1087A000706F012044FD060866FD06080FFD0608EF
:1087B0001FB50A4B03930A4B02930A4B01930A4BD2
:1087C00000930A4A0A4B0B490B48FEF74DFE0B4932
:1087D0000B4805B05DF804EBFEF746BE62160708CD
:1087E0001DF8060826F806082FF8060890EB06087C
:1087F00017F80608A3EB060894FD06083BF80608E0
:10880000AFFD0608F8B50C480C4E0D4F0D4DFEF7A8
:108810002BFE0D4B1A68C2F500729200002422B1A3
:1088200056F824103846FEF71FFE0134222C02D0E1
:1088300055F82420F3E7F8BDB8FD06085C55060896
:10884000CEFD0608243B0020203300202DE9F34113
:108850001A481B4C1B4E1C4FDFF87080FEF704FEBD
:108860000025E2792168A37994F808C006EB82021A
:1088700001F13F41D2F8E007A28806EB830301F53E
:108880007E01890AB2FA82F2D3F858374131C2F137
:108890001F02BCF1000F0CD0CDE900C04046FEF72E
:1088A000E3FD0135312D04F10C04DAD102B0BDE84D
:1088B000F08100903846FEF7D7FDF2E7DCFD0608B0
:1088C000D4730020044E060808FE0608F8FD0608CA
:1088D00070B5124B93F8D029D2B1192A94BF104B1E
:1088E00010491148114D124E98BF03EB82034FF00F
:1088F000000498BFD3F85C18FEF7B6FD214655F882
:10890000042B30460134FEF7AFFD082CF6D170BDC4
:10891000BDE870400748FBF715BD00BFB8C900208F
:10892000044E060816FE06081EFE06088CD300201C
:1089300036FE060845FE06082DE9F8432CF02CF912
:1089400020B9BDE8F8434948FBF7DCBC4848494C2E
:10895000494E4A4FDFF87081FBF7F4FC002563783D
:10896000FF2BA94605F1010576D02278FF2A73D0A6
:1089700029463046FEF778FD2378A178062B5AD891
:10898000DFE803F004343A42594A5200072954D828
:108990003B4B03EB8103D3F8C4283846FEF764FD54
:1089A000A1794046FEF760FDE1793648072997BF77
:1089B000334B354A03EB8103D3F84829FEF754FDC6
:1089C000324B334803EB091303F6FC19B3F8FE19D5
:1089D000FEF74AFDB9F8021001F00301012936D073
:1089E000022940D02B48FEF73FFD33E02A4A2B4BAB
:1089F000002908BF1A46D0E7062920D8204B03EBF0
:108A00008103D3F8E428C8E707291AD81C4B03EBE5
:108A10008103D3F80029C0E7092914D8184B03EBC8
:108A20008103D3F82029B8E779B11D4A1D4B0229EB
:108A300018BF1A46B1E71C4AAFE71C4AADE71C4A0B
:108A4000ABE71C4AA9E71C4AA7E71C4AA5E71C4854
:108A5000FBF778FCFBF764FC402D04F110047FF475
:108A60007EAFBDE8F8831748F2E700BFEBFE0608CB
:108A70001AFF0608ACD300202AFF06083EFF0608AE
:108A8000044E060866FF06088BFE0608B8C90020DB
:108A900077FF0608AEFF060886FE06087BFE06087E
:108AA000CDFE0608DBFE06085CFE06086FFE060823
:108AB00093FE0608A3FE0608B2FE0608BFFE0608DF
:108AC0008CFF06089CFF06084DFF06082DE9F843B9
:108AD000274DDFF8B89004460020FBF77BFC2548C3
:108AE000FBF750FCA97824480131FEF7BDFC214674
:108AF0002020FBF7CEFD2148FBF744FCAB78204A51
:108B000009F6F4564FF4D67707FB0363D3ED057AE5
:108B1000F5EE407AF1EE10FA0CBF0121002120465B
:108B2000FCF7D0FBA978794305F50C68143108EB04
:108B3000010220463144FCF735FF1248FBF722FCC6
:108B4000AB78114A07FB03992046B9F9CA1EB1FA5E
:108B500081F14909FCF7B6FBA9787943D43108EBD8
:108B6000010220463144BDE8F843FDF7EDBE00BFE9
:108B7000C0B80020C5FF0608D3FF0608E6FF0608B8
:108B8000F9FF0608080007081B000708B8C90020FD
:108B900008B50448FBF7B6FB034B1868BDE808406E
:108BA000F6F7C7BE1FF00608F0800020034B012235
:108BB00083F8A02F022283F8A12F7047B8C90020A4
:108BC00070B50D4E35782D1A18BF012503280446BF
:108BD00034BF044600242046F5F7DEFE074A347011
:108BE00002F6A873C4EB041403EB4403C2F8A43FD9
:108BF0001BF0F6F8284670BDC0B80020B8C90020A8
:108C0000022810B50C4618D8FFF7DAFF0B48FBF71F
:108C1000B9FB0B4B0B4819780131FEF725FC2146B7
:108C20000820FBF736FD21461020FBF732FD2146D8
:108C30002820BDE81040FBF72CBD10BD2800070818
:108C4000C0B800203800070838B5154C154DAC42A7
:108C500013D30020F5F7A0FE134823F0D9F8134AE8
:108C6000136843F48003136000BF114B1878FFF7BB
:108C7000A7FFBDE838402DF073BAB4F90230002BDD
:108C80004FF00001204607DAF5F776FE0121204675
:108C9000F5F772FE02212046F5F76EFE1434D6E792
:108CA000C4510708145707084D000708543D002019
:108CB000C0B8002010B504460A48FBF723FBFFF7B5
:108CC000C3FF23F089F8F5F71FFD23F08FF8064B5B
:108CD0000649002220461A70FBF7ACFE08B9FCF7E3
:108CE0005FF810BD56000708F78000201C01070838
:108CF00010B5064B5C78241A18BF0124032828BF3E
:108D00000020587023F0B0FD204610BDC0B80020F0
:108D1000022810B50C4610D8FFF7EAFF0748FBF70A
:108D200031FB074B074859780131FEF79DFB21467F
:108D30001820BDE81040FBF7ACBC10BD6C00070864
:108D4000C0B800207C0007082DE9F04F0D468DB01B
:108D5000B6490746FBF76EFE0646002840F0B7808E
:108D6000B3493846FBF766FE0646002840F0B1805E
:108D7000B0493846FBF75EFE0646002840F0AB805F
:108D8000AD493846FBF756FE0646002840F0A58060
:108D9000AA493846FBF74EFE002806460ABF0124C2
:108DA00010243E466D4205F020052C43A44DA54FEE
:108DB00095F800A095F8029095F80180DFF8F8B2D8
:108DC0005F45C0F08C80FFF73FFF5046FFF7F8FE8D
:108DD0004846FBF7FFFA4046FFF78AFF9A493046BC
:108DE000FBF728FE08B144F0400414F0110301938E
:108DF00000F05A829548FBF7C5FA0020FFF7D8FC2F
:108E00009348FBF7BFFA9348FBF79CFA04F0300352
:108E1000302B02D19048FBF7B5FA9048904FFBF702
:108E2000B1FA9048FBF7AEFA4FF0FF338E4A8F4904
:108E30002046FEF783FA8E48FBF7A4FA8D4A8E4946
:108E40002046FDF7C7FC8D48FBF79CFA8C4A8D49FC
:108E50002046FDF7F7F98C48FBF794FA8B4A8C49CA
:108E60002046FDF7E5F88B48FBF78CFA8A4B1E6825
:108E70008A4BD3F800908A4B00939B4669EA06031D
:108E80004FF0000A02935BF8043B002B34D01A78B1
:108E9000D2B1029A03934FF0010808FA0AF812EAD5
:108EA000080F14BF012100213A462046FCF78AFA38
:108EB00066EA090212EA080F039B3A4614BF012131
:108EC00000212046FCF7FEF90AF1010ADBE7012444
:108ED00068E7022466E7082464E7042462E77B88E5
:108EE000C3F30B021B04D7E9011048BF02EB420297
:108EF0004BF09CF9143763E71F46DFF8C0A169EA1D
:108F000006030293009B53F804BB0093BBF1000FD0
:108F100025D09BF8002002B34FF0010808FA07F8AB
:108F200019EA080F0BD066EA090212EA080F5B463D
:108F3000524614BF012100212046FCF743FA16EAED
:108F4000080F0AD0029B13EA080F52465B4614BF73
:108F5000012100212046FCF7B5F90137D2E751483D
:108F6000DFF85CA1FBF70EFA4F4AD2F800804F4AB7
:108F7000126888EA02025E46D343DFF848B10093E4
:108F8000009B0127B7403B4214BF4FF001094FF04F
:108F9000000918EA07070CBF52465A4630460392AA
:108FA0001BF078F9039A0290034649462046FCF7E5
:108FB00009FA0136002F0CBF5A465246029B494619
:108FC0002046FCF77FF9182EDAD13948DFF8F8A0EF
:108FD000DFF8F880DFF8F890FBF7D4F9354BD3F8D9
:108FE00014710026F3B20AEB8302D2F8B4B4BBF1D9
:108FF000000F6FD00121994039405B460CD04A46A2
:1090000000212046FCF75EF95B464A4600212046D7
:10901000FCF7D8F90136E5E7424620460091FCF717
:1090200051F900995B464246F1E700BFA6000708E8
:1090300028000708C5FF06086C000708AD000708F0
:10904000C0B80020C4510708B1000708BE000708D7
:10905000C6000708DE000708EA0007082501070820
:10906000750107082F010708307F002008810020C4
:109070003F010708A4C80020BAD900204F01070803
:1090800050C500204CDA00205801070840C40020D9
:10909000ACDA00206C010708583D0020543D002048
:1090A000345206088C010708FC8000207C7F0020D9
:1090B00093010708B0DA0020145707088101070858
:1090C0009B00070891000708044E0608A80107083E
:1090D0009C0107089748FBF755F9DFF828C3964825
:1090E000964ACDF820B0CDF810B0042601271CF820
:1090F000013F10F801EB03F13001694401F820EC65
:1091000012F8011F01F13008E84408F810EC002FB4
:1091100000F0ED805F1A79427941013E0F46E6D1B9
:10912000874A8DF8146008AB2046FCF74BF904AB76
:109130003946834A2046FCF7C5F88248FBF722F9F6
:10914000814A82492046FCF71FFA8148FBF71AF949
:10915000804A81492046FDF721F98048FBF712F942
:109160007F4A80492046FDF73DFA7F48FBF70AF920
:10917000784A79492046FDF7CDFA7C48FBF702F999
:109180007B4A7C492046FCF733F97B48FBF7FAF829
:109190007A4A7B492046FCF719FB7A48FBF7F2F83C
:1091A000794A7A492046FCF729FD7948FBF7EAF825
:1091B000784A79492046FCF7C1FD7848FBF7E2F888
:1091C0007749204642F0B8FC7648FBF7DBF84FF0D1
:1091D000FF331A467449204642F03AFD7348FBF7C4
:1091E000D1F84FF0FF33724A72492046FDF796FCE2
:1091F0007148FBF7C7F8714A71492046FDF7AFFD8A
:109200007048FBF7BFF8704A70492046FDF73CFEF6
:109210006F48FBF7B7F86F4A6F492046FDF750FFDC
:109220006E48FBF7AFF821463046FBF732FA14F0F0
:10923000100F2F785DD02146304695F8029095F8B2
:109240000180FFF7DDFC21460120FFF7D9FC214614
:109250000220FFF7D5FC2046FFF738FC21463046B8
:10926000FFF756FD21460120FFF752FD214602205F
:10927000FFF74EFD3846FFF7A3FC4846FBF7AAF878
:109280004046FFF735FD5648FBF77CF85548791CFA
:10929000FEF7EAF8544809F10101FEF7E5F85348F2
:1092A00008F10101FEF7E0F80026A00703D52878B1
:1092B0002146FFF7A5FC210704D5AB7813B920465A
:1092C000FFF704FC620703D568782146FFF720FD0D
:1092D000019B13B14648FBF755F82EB14548FBF703
:1092E00051F84548FBF72EF8444C454D1CE03946F3
:1092F00013E721463846FFF783FCAB7813B92046C5
:10930000FFF7E4FB68782146FFF702FD0126CCE772
:109310006388C3F30B021B04D4E9010148BF02EBCD
:1093200042024AF083FF1434AC42F1D30DB0BDE8E1
:10933000F08F00BFB50107082C5406088CBE002032
:10934000CB010708D2010708D8C00020F0DB0020BD
:10935000D8010708B0C5002020DC0020DD01070887
:1093600030C80020A0DE0020E7010708F60107084A
:1093700008C0002014DF00200202070808C10020F6
:10938000B4DF0020190207082CC300202CE00020C5
:109390002A02070840C3002040E0002036020708E8
:1093A00040E1002055020708A0EA002066020708F5
:1093B00034C90020E8EF00207902070834CE0020ED
:1093C000E8F400209702070894CE002048F500201A
:1093D000B402070804CF0020B8F50020A600070853
:1093E000C9020708EC020708FF0207081003070874
:1093F000230307083C03070852030708C451070862
:1094000014570708CCDB002000219DE401219BE4D8
:109410002DE9F04FD24CDFF884A385B0D14B9C42AC
:10942000C0F08D81D04DD14C2878FFF7C9FB68780A
:10943000FFF75EFCA878FAF7CDFFB5F8D426B5F8AB
:10944000B036CB4804329A42A4BF5A1FA5F8D4269E
:10945000B5F8D626043A9342A8BF053394F8212BD9
:10946000A8BFA5F8D63694F8203B9A4224BF002323
:1094700084F8203BF5F742FABE4B1A68BE4B934383
:1094800012D100212520F0F731FD064660B1002100
:109490002720F0F72BFD38B1026833689A4203D1D8
:1094A0004FF48030F5F72AFA0027DFF8D0823E46E5
:1094B0004FF0FF0948F2B83A58F8270043088108EE
:1094C00001F0333103F077330B44C10801F011315F
:1094D000C31A5B1A03EB131310F0010203F00F33EE
:1094E000B3FBF9F1C1EB012118BF0136A3EB010376
:1094F00018BFF6B2012B40F29981022B00F08D814A
:109500009E480D2144F07CFFB4F8503BB4F84E2B3C
:10951000643B9342A8BF1346A4F84E3B00BF94F8A7
:10952000C63B13B9082384F8C63B002012F0DAFDCD
:10953000DFF86CB2DBF80030002800F0808123F007
:109540008063CBF800308E4BD3F8A42F019214F037
:109550002BFA804614F0CEF9019A1FFA88F311789D
:109560000093A0EB08034B43642193FBF1F385497F
:1095700013FA88F3A4F8DC3B00271678A7EB06095A
:109580000FFA89F9B9F1000FB24640F35B81C6F1D9
:109590006406F6B253780391CDE9013214F0AAF9CA
:1095A000019B039909FB09FC03FB0CFCC3F1640359
:1095B00016FB06F60AEB8A0A9CFBF6F633440A22EF
:1095C00009FB03F393FBF2F303EB4A0A0FFA8AFA5F
:1095D000A0EB08004FF47A73174400FB0AFA9AFBD9
:1095E000F3FA009B029ABFB29A446E2F21F802ABA5
:1095F000C3D123F053F91AF09FF9302200216248B9
:109600004AF058FE12F070FB94F8143C4BBB95F8EE
:109610006610C4F8203C6422C82012FB0101C4F883
:10962000181C95F86710C4F8243C12FB0102C4F81A
:109630001C2CC4F8283C95F86920C4F82C3CC4F8CC
:10964000303CC4F8343C84F8413C84F8423C84F813
:10965000153CC4F8443C4FF07A7384F8402CC4F8AD
:10966000483CDBF8003049499B060A6800F1ED8070
:10967000B4F8160BB4F8143B0343B4F8180B0343C7
:109680001BB2002B40F0E180B4F91A3BB3F5805FC8
:1096900040F0DB80B4F91C3BB3F5805F40F0D5802F
:1096A000B4F91E3BB3F5805F40F0CF8022F4007226
:1096B0000A6023F011F8B4F84C3C9FED357AB4F809
:1096C0004E1C344A06EE903AF8EEE66A02F5A863BC
:1096D000C6EE877A06EE901AF8EEE66AB4F8501CE9
:1096E000C3ED007A86EE876A06EE901AF8EEE66A17
:1096F000B4F8521C83ED016A86EE876A06EE901A72
:10970000F8EEE66A77EE867AC6EE875A94F8541C2D
:1097100082F854159FED207A83ED026A67EE877A0E
:10972000B6EE007A67EE877AC3ED035AC3ED047A8A
:1097300019F092FE05B0BDE8F04F3CF0B7B8B4F9AF
:109740000230DFF86080002BA7BF002637460326D3
:10975000012700257919C9B28E4225D214345DE65D
:10976000C451070814570708C0B80020A8EB002010
:1097700020631406543D002040000100D8C00020A2
:10978000B8C90020B874012088F70020886F012034
:1097900000401C46906F012035FA0E3D0140000844
:1097A000E06E012000800008534603F1060BC3451C
:1097B0004ED21A88002A4BD003EB020CC44547D284
:1097C000052A45D92088B3F802E0C0F30B0086458E
:1097D00021D1587900F0030088421CD12946204647
:1097E00093F804900092F5F7C7F82188009AB9EB36
:1097F000113F0ED161886068C1F30B03063A9A42AB
:10980000A8BF1A46090448BF03FB050059464AF0A1
:109810000DFD01359EE76346C7E712B110EA0A0F56
:1098200004D143F08BFC00283FF46AAE03370C2FC1
:109830007FF442AE013E022E7FF666AE60E643F054
:1098400080637EE608BF0126A4E642F400722FE79B
:1098500029462046F5F790F8DBE710B5144C94F84C
:10986000A13F022B18D122F0B7FAF4F74DFFFFF712
:10987000CFFD22F0BBFA01201CF098FF0D4B0E49E2
:109880001B6803F59C530022083384F8A02FC1F80D
